:100000000C94891B0C94BA1B0C94BA1B0C94BA1B4D
:100010000C94BA1B0C94BA1B0C94BA1B0C94BA1B0C
:100020000C94BA1B0C94BA1B0C94BA1B0C94BA1BFC
:100030000C94BA1B0C94BA1B0C94BA1B0C94BA1BEC
:100040000C94BA1B0C94C7A40C94BA1B0C94BA1B46
:100050000C94BA1B0C94BA1B0C94858B0C942577CA
:100060000C94BA1B0C94F6EF0C94ECEF0C94BA1BA6
:100070000C94BA1B0C94BA1B0C94BA1B0C94BA1BAC
:100080000C94EFC50C94BA1B0C94BA1B0C94BA1BBD
:100090000C94BA1B0C94BA1B0C94BA1B0C94BA1B8C
:1000A0000C94BA1B0C94BA1B0C94C1C50C94BA1BCB
:1000B0000C94BA1B0C94BA1B0C94BA1B0C94BA1B6C
:1000C0000C94BA1B0C94BA1B0C94BA1B0C94A4C6C7
:1000D0000C946EC60C94BA1B0C94BA1B0C94BA1BED
:1000E0000C94BA1B084AD73B3BCE016E84BCBFFDC3
:1000F000C12F3D6C74319ABD56833DDA3D00C77FF8
:1001000011BED9E4BB4C3E916BAAAABE0000008090
:100110003F05A84CCDB2D44EB93836A9020C50B91F
:10012000918688083CA6AAAA2ABE000000803F004B
:100130000D94541A0D94F62B0D94F3160D946B0C2C
:100140000D94860B0C94BB720C94D3740C949CF09D
:100150000D94CE0E0D9454170C949C720C94F4458F
:100160000D945C1C0C94DD730D94241A0C94BF4305
:100170000C943EC70C94AD720C94C9730D94111677
:100180000D944C100C94A7F00C94BAF00D94BC167E
:100190000D94A8160C9411C70C9472F00C94B345EE
:1001A0000C94B7720C94DA6F0C9474740C945B76A4
:1001B0000C9436C70C9455C70C94A7720C947B759D
:1001C0000D94142C0C943AC70D942C140D947C1A95
:1001D0000C94E2C60C9490F00C941C750C949C73D7
:1001E0000D947F160D94DF160C9460750C944AC71D
:1001F0000D94AF140C94D3730C94BF730C9434F01F
:100200000D947B140C94CD720C9420C70C940B7637
:100210000C9457730D949A1A0D94881B0C94987231
:100220000C94C9720C94E7730C9438760D943C1FAF
:100230000C94F1730D944B150C948A730C94BB437E
:100240000C9488F00C9464730C945D700C9460C7EB
:100250000D94861A0D9412170C9468C70D94650AB4
:100260000C9481F00C9481720D9417180C94827385
:100270000C94C5720C945C700D945F140C944EC772
:100280000C94A6730C9498F00C942FC70C946E7376
:100290000D94A71A0C945F730C9446C70D94DB154C
:1002A0000C94F9750D94511A0D944B1A0C947873A3
:1002B0000C94A0720C9457740C94B0730C948672C6
:1002C0000C946C430C94A0F00C942C460C94A472E7
:1002D0000C94D3720C948CF00C94BF720D946D1A24
:1002E0000D94FD0D0D94991B0C9494F00C9463F0F7
:1002F0000D94950C0D9467170C94B2F00C94B17298
:100300000C94D7720C9487450C9492730C9442C74A
:100310000D94E6124E414E494E495459494E46CD30
:10032000CCCC3D0AD7233C17B7D13877CC2B3295AC
:1003300095E6241FB14F0A000020410000C842008A
:10034000401C4620BCBE4CCA1B0E5AAEC59D740054
:10035000407A10F35A00A0724E18090010A5D4E894
:100360000000E87648170000E40B54020000CA9A27
:100370003B000000E1F50500008096980000004079
:10038000420F000000A086010000001027000000BE
:1003900000E803000000006400000000000A000004
:1003A0000000000100000000002C76D888DC674FB8
:1003B0000823DFC1DFAE59E1B1B796E5E3E453C6E8
:1003C0003AE651997696E8E6C28426EB898C9B62E0
:1003D000ED407C6FFCEFBC9C9F40F2BAA56FA5F48A
:1003E00090055A2AF75C936B6CF9676DC11BFCE0B2
:1003F000E40D47FEF520E6B500D0ED902E03009405
:100400003577050080841E080000204E0A00000099
:10041000C80C333333330F986E12831141EF8D21A3
:1004200014893BE65516CFFEE6DB18D1844B381B0A
:10043000F77C1D901DA4BBE424203284725E2281CF
:1004400000C9F124ECA1E53D27434F4D4D554E49E0
:10045000434154494F4E0044525952554E00455263
:10046000524F525300494E464F004543484F004FAC
:100470004646004F4E0020204D61783A2000200073
:1004800020204D696E3A2000536F667420656E64BB
:1004900073746F70733A20003D3D4F6E506F7765F7
:1004A000724C6F7373526573756D653D3D004D32CF
:1004B000342053256C642054256C64004739322E57
:1004C00039204525730047312046256400473932DD
:1004D0002E39205A2573004731205A3020463230B9
:1004E000300047312058257320592573204633307A
:1004F0003030004D34323020532569205A257300A6
:100500004D3130362050256920532569004D323059
:10051000302044257300473238523058590047394B
:10052000322E39204530205A300A47315A2573007F
:100530004D31303920532569004D31393020532554
:1005400069004D343230205330205A300020496E3B
:1005500076616C69642065787472756465722000D8
:1005600047322F47332062616420706172616D658C
:10057000746572730A00536C6565702E2E2E005AD6
:100580002050726F62652050617374204265640A66
:10059000005A2050726F626520506173742042656A
:1005A00064004732384C30004D3131372050726F83
:1005B0006265206661696C65642E0A4732380A00FC
:1005C00070726F62655F7265776970650047323976
:1005D000205265747279696E670050726F62696E3D
:1005E00067204661696C6564004D31313720426592
:1005F00064206C6576656C696E67206661696C6500
:10060000642E0A4730205A31300A4D3330302050A2
:10061000323520533838300A4D33303020503530A1
:100620002053300A4D333030205032352053383883
:10063000300A4D333030205035302053300A4D339E
:1006400030302050323520533838300A4D33303076
:10065000205035302053300A473420533100707217
:100660006F62655F6661696C6564004D313137208A
:10067000426564206C6576656C696E6720646F6E98
:10068000652E00205A3A200020593A200042656425
:1006900020583A20004D65736820706F696E742091
:1006A0006F7574206F662072616E67650A004D3049
:1006B0002053746F70004D312053746F7000436F7E
:1006C0006E74696E756500436C69636B20746F208E
:1006D000526573756D652E2E2E004E6F204D6F7610
:1006E000652E00456E642066696C65206C697374C4
:1006F0000A00426567696E2066696C65206C6973E3
:10070000740A004E6F206D656469610A005265735A
:10071000756D696E6720534400286E6F2066696CA2
:1007200065290043757272656E742066696C653A5E
:1007300020005072696E742074696D653A20000A59
:1007400053746174733A2046696C616D656E7420F0
:10075000757365643A20002C204C6F6E6765737466
:10076000206A6F623A2000546F74616C2074696D66
:10077000653A200053746174733A20002C2046615E
:10078000696C65643A20002C2046696E697368655F
:10079000643A20005072696E74733A200053746199
:1007A00074733A2000436F6F6C696E672E2E2E00B3
:1007B00048656174696E672E2E2E00452025530012
:1007C0006F6B006F6666006A0465045E0457044937
:1007D0000444454255473A004D31313320530042DD
:1007E000656420436F6F6C696E672E2E2E00426524
:1007F000642048656174696E672E2E2E00544D3357
:100800004420453520506C7573204F46462E002FEE
:100810002F004D32303620580046523A0020466CA8
:100820006F773A20003A200020536572766F2000DF
:10083000206F7574206F662072616E67650A0053C1
:100840006572766F200020643A0020693A002070BB
:100850003A00496E76616C696420657874727564DB
:1008600065720A0020643A0020693A0020703A005C
:1008700064697300656E0043290A0061626C6564F7
:1008800020286D696E2074656D702000436F6C6464
:1008900020657874727564657320617265200050FC
:1008A0004944204175746F74756E65005049442049
:1008B0004175746F74756E65206661696C6564213D
:1008C00020426164206865617465722069640A0071
:1008D00046696C616D656E742072756E6F757420FB
:1008E00064697374616E636520286D6D293A200018
:1008F00046696C616D656E742072756E6F757420DB
:10090000004D34323120696E636F727265637420FA
:10091000706172616D657465722075736167650AD7
:10092000004D65736820706F696E74206F75742058
:100930006F662072616E67650A004F666673657444
:1009400073204170706C696564004572723A20547E
:100950006F6F206661722100546F6F206661722094
:1009600066726F6D207265666572656E6365207074
:100970006F696E740A00454550524F4D204F4B0A27
:10098000002E0A002028302D313029002076616C9D
:100990007565206F7574206F662072616E676500E3
:1009A000416476616E6365204B3D00506F776572E0
:1009B0002D6C6F7373207265636F7665727920009A
:1009C0004D383400446F6E65207072696E74696EC4
:1009D000672066696C650A004D3737004D3331007A
:1009E0004361703A004D4541545041434B00434FE1
:1009F0004F4C45525F54454D504552415455524518
:100A0000004348414D4245525F54454D5045524187
:100A10005455524500424142595354455050494E55
:100A2000470041524353004D4F54494F4E5F4D4F85
:100A300044455300544845524D414C5F50524F5429
:100A4000454354494F4E004C4F4E475F46494C4535
:100A50004E414D45004155544F5245504F52545F01
:100A600053445F5354415455530053445F575249C4
:100A7000544500524550454154005344434152446B
:100A80000050524F4D50545F535550504F525400E8
:100A9000454D455247454E43595F5041525345528B
:100AA00000434153455F4C494748545F42524947D0
:100AB00048544E45535300544F47474C455F4C49AB
:100AC0004748545300534F4654574152455F504F87
:100AD000574552004255494C445F50455243454E9C
:100AE00054004C4556454C494E475F4441544100E3
:100AF0005A5F50524F42450052554E4F5554004197
:100B000055544F4C4556454C005052494E545F4A3F
:100B10004F420050524F4752455353004155544F96
:100B20005245504F52545F54454D5000564F4C550E
:100B30004D455452494300454550524F4D0042499E
:100B40004E4152595F46494C455F5452414E5346BF
:100B500045520053455249414C5F584F4E5F584FE4
:100B60004646004649524D574152455F4E414D451C
:100B70003A4D61726C696E20322E302E375F4457C9
:100B8000372E3320544D334420453550534D444285
:100B900042202841707220323420323032312031EC
:100BA000393A34383A35362920534F555243455F48
:100BB000434F44455F55524C3A68747470733A2FF2
:100BC0002F6769746875622E636F6D2F496E73614C
:100BD0006E6974794175746F6D6174696F6E2F4DB4
:100BE00061726C696E2F747265652F437265616CFA
:100BF0006974794477696E5F322E302050524F54B9
:100C00004F434F4C5F56455253494F4E3A312E3069
:100C1000204D414348494E455F545950453A544D43
:100C2000334420453520506C757320455854525537
:100C30004445525F434F554E543A3120555549442F
:100C40003A63656465326132662D343161322D3428
:100C50003734382D396231322D633535633632669B
:100C600033363766660A0050726F6265204F6666DB
:100C7000736574205A0050726F6265204F66667308
:100C80006574205A00290A0020746F20003F5A2002
:100C90006F7574206F662072616E67652028002969
:100CA0000A0020746F20003F59206F7574206F6612
:100CB0002072616E676520282D00290A0020746F5C
:100CC00020003F58206F7574206F662072616E6738
:100CD0006520282D0050726F6265204F666673652F
:100CE0007420580043616E6E6F74206F70656E20C3
:100CF00073756264697220002569730025696D202F
:100D0000256973002569682025696D2025697300B0
:100D1000256964202569682025696D20256973008F
:100D200025697920256964202569682025696D2059
:100D3000256973003D3D4477696E20496E697420D2
:100D4000436F6D706C6574653D3D002A2A2A4E6FB5
:100D50007A7A6C6554656D705374617475735B3227
:100D60005D203D003D3D48656174696E6720446FBC
:100D70006E65204368616E67652046696C616D65CC
:100D80006E743D3D002020737461727470726F67E1
:100D90007265737320003D3D7761697477617920D6
:100DA000353D3D003D3D7761697477617920343D83
:100DB0003D003D3D7761697477617920333D3D00A9
:100DC0003D3D7761697477617920313D3D003D3D5E
:100DD0006F6E5072696E7454696D657253746F7082
:100DE0007065643D3D003D3D6F6E466163746F729A
:100DF0007952657365743D3D00270A0A000027207B
:100E000027002027002D006E6F7469666963617486
:100E1000696F6E200063616E63656C005072696E6D
:100E2000742041626F72746564004469736D697304
:100E3000730055492041626F727465640072657376
:100E4000756D65004D3234002A2A2A43506C617951
:100E500020546F6E652A2A2A003D3D6F6E507269DC
:100E60006E7454696D65725061757365643D3D00C3
:100E7000486F6D696E67204661696C6564006F70CC
:100E8000656E00545249474745524544003A200098
:100E900066696C616D656E74007A5F6D696E00796C
:100EA0005F6D617800785F6D6178005265706F7278
:100EB00074696E6720656E6473746F7020737461FB
:100EC0007475730A0020746F6F206C6F6E672065F5
:100ED0007874727573696F6E2070726576656E7462
:100EE00065640A0020636F6C6420657874727573A2
:100EF000696F6E2070726576656E7465640A00486D
:100F00006F6D652025732573257320466972737490
:100F1000005761726E696E673A20486F6D696E673F
:100F20002042756D702044697669736F72203C2091
:100F3000310A000202040000B4430000B443000080
:100F400000000000B4430000B4430000C8430000A8
:100F5000004100000041000000400101FF000000CE
:100F600001000000010000800055555500000040C0
:100F70000033333300AAAA2A00499224000000203B
:100F800000C7711C0099991900D1451700555515D6
:100F9000003BB11300244912001111110000001090
:100FA000000F0F0F00E3380E0043790D00CCCC0C7E
:100FB00000C3300C00E8A20B0064210B00AAAA0AAF
:100FC00000703D0A009DD80900427B090092240967
:100FD00000DCD308008888080010420800000008E0
:100FE00000F0C107008787070075500700711C07D4
:100FF000003EEB0600A1BC0600699006006666068E
:1010000000703E06006118060017F4050074D10553
:10101000005BB00500B290050062720500555505F1
:101020000078390500B81E0500050505004EEC04E2
:101030000087D40400A1BD040090A70400499204D5
:1010400000C17D0400EE690400C756040044440456
:10105000005C320400082104004110040000000478
:10106000003FF00300F8E0030026D20300C3C303EF
:1010700000CCB503003AA803000A9B0300388E0396
:1010800000C08103009F750300D0690300505E0318
:10109000001D53030034480300913D030033330324
:1010A0000016290300381F030097150300300C03B6
:1010B00000030303000BFA020049F10200BAE80240
:1010C000005CE002002DD802002DD0020059C802B9
:1010D00000B0C0020031B90200DAB10200AAAA02CF
:1010E00000A0A30200BC9C0200FA9502005C8F02E3
:1010F00000DF88020082820200457C02002776021F
:101100000027700200436A02007C640200D05E0285
:10111000003F590200C8530200FFFDFCFAF8F6F444
:10112000F2F0EEECEAE9E7E5E3E1E0DEDCDAD9D77C
:10113000D5D4D2D0CFCDCBCAC8C7C5C3C2C0BFBD1E
:10114000BCBAB9B7B6B4B3B2B0AFADACAAA9A8A691
:10115000A5A4A2A1A09E9D9C9A99989795949392DC
:10116000908F8E8D8B8A8988878684838281807F09
:101170007E7D7B7A797877767574737271706F6E15
:101180006D6C6B6A696867666564636261605F5E07
:101190005D5C5B5A595858575655545352515050EC
:1011A0004F4E4D4C4B4A4A494847464645444342B8
:1011B0004241403F3E3E3D3C3B3B3A393838373672
:1011C0003535343332323130302F2E2E2D2C2B2B1F
:1011D0002A292928272726252524232322212120BF
:1011E000201F1E1E1D1C1C1B1B1A19191818171650
:1011F00016151514131312121111100F0F0E0E0DD8
:101200000D0C0C0B0A0A0909080807070606050554
:101210000404030302020100003D3D6F6E50726939
:101220006E7454696D6572537461727465643D3D8A
:10123000000000B4430000B4430000C843000000B5
:101240000000000000000000003D3D6F6E53746F11
:10125000726553657474696E67733D3D003D3D6F03
:101260006E436F6E66696775726174696F6E5374F1
:101270006F72655772697474656E3D3D0053657495
:1012800074696E67732053746F726564000A206915
:101290006E6974207A70726F62655F7A6F666673CA
:1012A0006574203D20003D3D6F6E436F6E6669673B
:1012B00075726174696F6E53746F726552656164A3
:1012C0003D3D00454550524F4D20496E697469615E
:1012D0006C697A65640A003B20003A0A0020204DC0
:1012E000363033200020440020204D34313220534A
:1012F0000046696C616D656E742072756E6F7574F1
:101300002073656E736F723A002055004C00466979
:101310006C616D656E74206C6F61642F756E6C6F9F
:101320006164206C656E677468733A0020204D39E3
:101330003030204B004C696E6561722041647661EB
:101340006E63653A0020204D3835312058005A2D03
:1013500050726F6265204F66667365740020204D81
:10136000343133205300506F7765722D4C6F737397
:10137000205265636F766572793A002044002049F7
:101380000020204D333034205000204400204900FC
:1013900020204D3330312050005049442073657473
:1013A00074696E67733A00204A0020204732392062
:1013B0005720490020204D343230205300417574AD
:1013C0006F20426564204C6576656C696E673A00F3
:1013D00020204D323036205800486F6D65206F66F2
:1013E000667365743A0020580020530020204D3267
:1013F0003035204200416476616E6365643A204274
:101400003C6D696E5F7365676D656E745F74696D61
:10141000655F75733E20533C6D696E5F66656564FC
:10142000726174653E20543C6D696E5F74726176C2
:10143000656C5F66656564726174653E20583C6DDD
:1014400061785F785F6A65726B3E20593C6D6178A8
:101450005F795F6A65726B3E205A3C6D61785F7A96
:101460005F6A65726B3E20453C6D61785F655F6ABF
:1014700065726B3E0020540020520020204D323017
:1014800034205000416363656C65726174696F6EEE
:101490002028756E6974732F7332293A20503C707E
:1014A00072696E745F616363656C3E20523C726565
:1014B00074726163745F616363656C3E20543C7455
:1014C000726176656C5F616363656C3E0020204DE0
:1014D0003230312058004D6178696D756D2041635F
:1014E00063656C65726174696F6E2028756E6974CE
:1014F000732F7332293A0020204D323033205800A8
:101500004D6178696D756D2066656564726174659D
:10151000732028756E6974732F73293A00537465AC
:1015200070732070657220756E69743A00204400F3
:1015300020204D3230302053002044697361626CAA
:1015400065640A0046696C616D656E74207365742C
:1015500074696E67733A0020286D6D29002020475A
:101560003231202020203B20556E69747320696E33
:10157000206D6D003D3D6F6E4C6F616453657474FA
:10158000696E67733D3D0000803B4400803B440032
:10159000002041000096420000A0420000A042004E
:1015A0000048440000BE42D0070000D0070000649D
:1015B0000000004B00000024F4D43050C38E20C241
:1015C000A24017828B7011127A910D816CD90AA8F2
:1015D00061E108C7586607615143061E4B5D05C1AE
:1015E00045A7041A411104093D980371393103409C
:1015F00036DB0265339102D4305402802E1D026323
:101600002CEE01752AC501B028A001102781018F99
:101610002564012B244B01E0223401AC211F018DF4
:10162000200D01801FFC00841EED00971DDF00B817
:101630001CD200E61BC600201BBC00641AB200B21C
:1016400019A8000A19A0006A189900D11791004042
:10165000178B00B516840031167E00B31579003A59
:10166000157300C7146F0058146A00EE13660088E3
:1016700013630025135E00C7125B006C1257001540
:10168000125400C111510070114F0021114B00D6AE
:101690001049008D1047004610440002104200C05F
:1016A0000F4000800F3E00420F3C00060F3B00CB76
:1016B0000E3800930E37005C0E3500270E3400F311
:1016C0000D3200C10D3100900D3000600D2E003242
:1016D0000D2D00050D2C00D90C2B00AE0C2900851A
:1016E0000C29005C0C2700350C27000E0C2600E8A6
:1016F0000B2400C40B2400A00B23007D0B23005AF5
:101700000B2100390B2100180B2000F80A1F00D90B
:101710000A1E00BB0A1E009D0A1D00800A1D0063F0
:101720000A1C00470A1B002C0A1B00110A1A00F7AA
:10173000091A00DD091900C4091900AB0919009242
:101740000917007B091800630917004C09160036B9
:10175000091600200916000A091500F5081500E011
:10176000081400CC081400B8081400A40814009051
:101770000813007D0812006B081300580812004679
:10178000081200340811002308110012081100018A
:10179000081100F0071000E0071000D0071000C08B
:1017A000071000B0070F00A107100091070E00837B
:1017B000070F0074070F0065070E0057070E00495A
:1017C000070E003B070D002E070E0020070D00132B
:1017D000070D0006070D00F9060C00ED060D00E0F0
:1017E000060C00D4060C00C8060C00BC060C00B0A9
:1017F000060C00A4060B0099060C008D060B008257
:10180000060B0077060B006C060B0061060A0057FA
:10181000060B004C060A0042060A0038060A002E93
:10182000060A0024060A001A060A00100609000724
:10183000060A00FD050900F4050900EB050900E2B0
:10184000050900D9050900D0050900C7050900BE32
:10185000050900B5050800AD050800A50509009CAF
:10186000050800940508008C050800840508007C24
:10187000050800740508006C050700650508005D93
:10188000050700560508004E0507004705070040FC
:1018900005080038050700310507002A0507002361
:1018A0000507001C050600160507000F05070008C0
:1018B00005060002050700FB040600F5040700EE1C
:1018C000040600E8040600E2040700DB040600D575
:1018D000040600CF040600C9040600C3040600BDC8
:1018E000040600B7040600B1040500AC040600A617
:1018F000040600A00405009B040600950405009062
:101900000406008A04050085040500800406007AA8
:1019100004050075040500700405006B04050066ED
:10192000040500610405005C04050057040500522D
:101930000405004D04050048040500430405003E6D
:101940000404003A04050035040500300404002CAA
:1019500004050027040400230405001E0404001AE3
:1019600004040016040500110404000D0404000919
:101970000405000404040000040400FC030400F84F
:10198000030400F4030400F0030400EC030400E883
:10199000030400E4030400E0030400DC030400D8B3
:1019A000030400D4030400D0030400CC030400C8E3
:1019B000030300C503030024F404D9201BC40C5CFA
:1019C0000E9804C4095F0265077101F405F900FB74
:1019D00004B30048048700C103690058035500039D
:1019E000034500BE023A008402310053022A002956
:1019F00002250004022000E4011C00C8011900AF08
:101A00000117009801140084011300710110006196
:101A100001100051010E0043010D0036010B002B97
:101A2000010B0020010B00150109000C0109000346
:101A3000010800FB000800F3000800EB000700E4C9
:101A4000000600DE000600D8000600D2000600CC2A
:101A5000000500C7000500C2000500BD000400B974
:101A6000000400B5000400B1000400AD000400A9AA
:101A7000000400A5000300A20003009F0004009BD7
:101A800000030098000300950002009300030090FB
:101A90000003008D0002008B000300880002008616
:101AA00000020084000300810002007F0002007D2C
:101AB0000002007B0002007900020077000100763E
:101AC0000002007400020072000100710002006F49
:101AD0000002006D0001006C0002006A0001006954
:101AE000000200670001006600010065000100645B
:101AF0000002006200010061000100600001005F5F
:101B00000002005D0001005C0001005B0001005A62
:101B10000001005900010058000100570001005663
:101B20000001005500010054000100530000005363
:101B30000001005200010051000100500001004F5F
:101B40000001004E0000004E0001004D0001004C5D
:101B50000001004B0000004B0001004A0001004959
:101B60000001004800000048000100470001004655
:101B7000000000460001004500000045000100444F
:101B80000001004300000043000100420000004249
:101B90000001004100000041000100400001003F41
:101BA0000000003F0001003E0000003E0001003D3B
:101BB0000000003D0001003C0000003C0000003C33
:101BC0000001003B0000003B0001003A0000003A29
:101BD0000001003900000039000100380000003821
:101BE0000000003800010037000000370001003617
:101BF000000000360000003600010035000000350E
:101C00000000003500010034000000340000003402
:101C100000010033000000330000003300010032F7
:101C200000000032000000320001003100000031ED
:101C300000000031000100300000003000000030E2
:101C40000001002F0000002F0000002F0000002FD7
:101C50000001002E0000002E0000002E0001002DCB
:101C60000000002D0000002D0000002D0001002CC0
:101C70000000002C0000002C0000002C0001002BB4
:101C80000000002B0000002B0000002B0001002AA8
:101C90000000002A0000002A0000002A000100299C
:101CA0000000002900000029000000290000002990
:101CB0000001002800000028000000280000002883
:101CC0000000002800010027000000270000002776
:101CD0000000002700000027000100260000002669
:101CE000000000260000002600000026000100255C
:101CF0000000002500000025000000250000002550
:101D00000000002500010024000000240000002441
:101D10000000002400000024000100230000002334
:101D20000000002300000023000000230000002327
:101D30000000002300010022000000220000002219
:101D4000000000220000002200000022000100210B
:101D500000000021000000210000002100000021FF
:101D600000000021000000210001002000000020F0
:101D700000000020000000200000002000000020E3
:101D800000000020000000200001001F0000001FD4
:101D90000000001F0000001F0000001F0000001FC7
:101DA0000000001F0001001E0000001E0000001EB9
:101DB0000000001E000000232C0000B82200005686
:101DC0001800003A0F0000B8080000B104000071CC
:101DD0000200003E01000020436F756E7420583AE7
:101DE0000023646566696E652044454641554C5440
:101DF0005F0000626564004B6420004B6920004B6B
:101E0000702000504944204175746F74756E6520D0
:101E100066696E6973686564212050757420746802
:101E200065206C617374204B702C204B6920616EAF
:101E300064204B6420636F6E7374616E74732066EC
:101E4000726F6D2062656C6F7720696E746F2043CE
:101E50006F6E66696775726174696F6E2E680A00CD
:101E6000504944204175746F74756E6520666169D0
:101E70006C6564212074696D656F75740A00504942
:101E800044204175746F74756E65206661696C6578
:101E900064212054656D706572617475726520747B
:101EA0006F6F20686967680A00204B643A20002041
:101EB0004B693A2000204B703A200020436C61733C
:101EC00073696320504944200A00204E6F206F76CA
:101ED000657273686F6F740A002054753A20002091
:101EE0004B753A2000206D61783A2000206D696EB4
:101EF0003A200020643A200020626961733A200091
:101F0000504944204175746F74756E652073746117
:101F100072740A00504944204175746F74756E657F
:101F2000206661696C6564212054656D706572611D
:101F30007475726520746F6F20686967680A004263
:101F4000656400453100626564002C207379737408
:101F5000656D2073746F70706564212048656174CD
:101F600065725F49443A200048656174696E672074
:101F70004661696C65640048656174696E672066D6
:101F800061696C6564004D31313220536875746449
:101F90006F776E001000C90210012C014001220170
:101FA00070011801B0010E01F00104015002FA00A5
:101FB000B002F0003003E600D003DC009004D20051
:101FC0007005C800A006BE000008B400B009AA0051
:101FD000D00BA000600E960060118C0000158200EE
:101FE00020197800C01D6E00A0226400B0275A009E
:101FF000902C500000314600E0343C001038320094
:10200000903A2800603C1E00A03D1400803E0A006B
:10201000203F0000544845524D414C2052554E41FE
:1020200057415900546865726D616C2052756E613C
:10203000776179004572723A204D415854454D50B0
:10204000004D415854454D50207472696767657260
:102050006564004572723A204D494E54454D50001A
:102060004D494E54454D50207472696767657265DD
:102070006400202F002042403A0020403A002057C0
:102080003A0020573A00496E76616C6964206578A1
:102090007472756465720A007C3C3E5E2B3D3F2F76
:1020A0005B5D3B2C2A225C0043616E6E6F74206F77
:1020B00070656E2073756264697220005344204914
:1020C0006E6974204661696C0053442063617264D8
:1020D000206F6B0A006F70656E526F6F74206661BF
:1020E000696C65640A00766F6C756D652E696E6942
:1020F00074206661696C65640A004E6F2053442049
:10210000636172640A000A4D3234004D3233202577
:1021100073002E0A006F70656E206661696C6564DD
:102120002C2046696C653A200046696C6520736511
:102130006C65637465640A002053697A653A20000F
:1021400046696C65206F70656E65643A2000454E87
:102150004420535542524F5554494E450A002220BF
:10216000706F73002220706172656E743A220053A2
:102170005542524F5554494E452043414C4C2074D2
:1021800061726765743A220053756263616C6C20FA
:102190004F766572666C6F77004578636565646538
:1021A00064206D617820535542524F5554494E4535
:1021B0002064657074683A002E0A0044656C65748A
:1021C000696F6E206661696C65642C2046696C6578
:1021D0003A200046696C652064656C657465643AF4
:1021E000005344207072696E74696E67206279745E
:1021F0006520004E6F74205344207072696E7469BC
:102200006E670A0057726974696E6720746F206682
:10221000696C653A2000667265736800646F696E68
:1022200067002066696C653A20004E6F7720002FAA
:102230006175746F25632E67002020506C616E6E8F
:10224000657242756666657242797465733A2000FC
:102250002046726565204D656D6F72793A200043A6
:102260006F6D70696C65643A204170722032342061
:10227000323032310A00204C617374205570646131
:102280007465643A20323032312D30342D313820AB
:102290007C20417574686F723A2054696E794D6183
:1022A0006368696E657333440A00322E302E375FDF
:1022B0004457372E330A004D61726C696E0020530B
:1022C0006F6674776172652052657365740A0020C9
:1022D0005761746368646F672052657365740A00A0
:1022E0002042726F776E206F75742052657365742B
:1022F0000A002045787465726E616C2052657365C2
:10230000740A00506F77657255700A0073746172B9
:10231000740A004732385859004D31303031006569
:1023200072726F722077726974696E6720746F20A1
:1023300066696C650A00446F6E6520736176696E2C
:10234000672066696C652E0A004D323900456E645F
:1023500073746F7073002553202563202563202537
:102360006320256300205A3A0020593A0020583A49
:1023700000656E6473746F7073206869743A20002E
:1023800000000A0B02090C0D0E08070304010000EF
:10239000000000000000000000000000000000003D
:1023A00000000000000000000000000012111000FA
:1023B000000000000000000000000000000000001D
:1023C0000000000000004572726F7220777269741D
:1023D000696E6720746F20454550524F4D210A00A9
:1023E00053544F505045442E20005072696E74650E
:1023F000722073746F707065642064756520746FEB
:10240000206572726F72732E204669782074686539
:10241000206572726F7220616E6420757365204D45
:1024200039393920746F20726573746172742E208B
:102430002854656D706572617475726520697320CA
:1024400072657365742E205365742069742061660B
:102450007465722072657374617274696E67290A9B
:10246000004E6F20436865636B73756D20776974E8
:1024700068206C696E65206E756D6265722C204CEB
:10248000617374204C696E653A20004E6F2043687A
:1024900065636B73756D2077697468206C696E6510
:1024A000206E756D6265722C204C617374204C69CE
:1024B0006E653A2000636865636B73756D206D69A6
:1024C000736D617463682C204C617374204C696E69
:1024D000653A20004C696E65204E756D626572200C
:1024E0006973206E6F74204C617374204C696E6543
:1024F000204E756D6265722B312C204C61737420F7
:102500004C696E653A20004D313130005365726977
:10251000616C20737461747573206D69736D61747F
:1025200063680A00776169740A0053442072656128
:1025300064206572726F720A002121204B494C4C55
:102540002063617573656420627920746F6F206DFC
:1025500075636820696E6163746976652074696D5E
:1025600065202D2063757272656E7420636F6D6DCA
:10257000616E643A2000486F74656E642049646C33
:10258000652054696D656F757400486F74656E647D
:102590002049646C652054696D656F75740A003D4F
:1025A0003D6F6E46696C616D656E7452756E6F75C8
:1025B000743D3D007061757365004D36303000200C
:1025C00066696C616D656E745F72756E6F7574208F
:1025D0000066696C616D656E745F72756E6F75749F
:1025E00020540046696C616D656E7452756E6F752E
:1025F000742054002A2A2A496E6974696E67206320
:10260000617264206973204F4B2A2A2A004D656449
:10261000696120496E736572746564004D65646913
:10262000612052656D6F766564004D3130303053F6
:1026300000627573793A2070617573656420666F06
:102640007220696E7075740A00627573793A207031
:10265000617573656420666F7220757365720A0018
:10266000627573793A2070726F63657373696E6710
:102670000A002A2A2A6B696C6C2A2A2A00706F7752
:1026800065726F6666004B494C4C45442E200050E5
:1026900072696E7465722068616C7465642E206B5B
:1026A000696C6C28292063616C6C6564210A005395
:1026B000544F505045442E20005072696E7465721C
:1026C0002073746F707065642064756520746F206A
:1026D0006572726F72732E20466978207468652067
:1026E0006572726F7220616E6420757365204D395A
:1026F000393920746F20726573746172742E2028CA
:1027000054656D70657261747572652069732072AD
:10271000657365742E205365742069742061667436
:1027200065722072657374617274696E67290A003C
:102730006563686F3A004572726F723A0042696C65
:10274000696E656172204C6576656C696E672047BD
:102750007269643A0A0021212053544F502063616A
:102760006C6C65642062656361757365206F6620BB
:10277000424C546F756368206572726F72202D2011
:10278000726573746172742077697468204D393989
:10279000390A0021212053544F502063616C6C652D
:1027A000642062656361757365206F6620424C54D6
:1027B0006F756368206572726F72202D2072657369
:1027C000746172742077697468204D3939390A0050
:1027D0002F2F616374696F6E3A0070726F6D707441
:1027E0005F00656E640053656E64204D31303820A3
:1027F000746F20726573756D650A00496E7365723A
:10280000742066696C616D656E7420616E642073FE
:10281000656E64204D3130380A0052656865617418
:102820002066696E69736865642E0052656865612B
:102830007420446F6E6500526568656174696E67E7
:102840002E2E2E00526568656174004865617465BE
:10285000722054696D656F75740053656E64204D08
:1028600031303820746F2068656174206E6F7A7A19
:102870006C650A004E6F7A7A6C65205061726B65E8
:102880006400486F74656E6420746F6F20636F6CB2
:10289000640A00706175736564005061757365004A
:1028A00044697361626C6552756E6F757400507522
:1028B0007267654D6F726500506175736564007372
:1028C000686F7700627574746F6E00626567696E19
:1028D000004C6F61642046696C616D656E74004CDC
:1028E0006F61642046696C616D656E7420540049A7
:1028F0006E736572742066696C616D656E742061BB
:102900006E642073656E64204D3130380A00726544
:1029100073756D656400526573756D696E670057F8
:10292000616974696E6720666F722068656174758D
:10293000702E0A004C656176696E6720473236005A
:102940003F53706563696669656420582C5920633C
:102950006F6F7264696E617465206F7574206F6645
:1029600020626F756E64732E0A003F2852296570CD
:102970006561742076616C7565206E6F7420706C73
:1029800061757369626C653B206D75737420626557
:10299000206174206C6561737420312E0A003F2819
:1029A00052296570656174206D75737420626520AD
:1029B000737065636966696564207768656E206E0B
:1029C0006F74207573696E6720616E204C43442ECE
:1029D0000A003F537065636966696564206E6F7AAB
:1029E0007A6C652074656D706572617475726520AE
:1029F0006E6F7420706C61757369626C652E0A006D
:102A00003F5370656369666965642066696C616DD2
:102A1000656E742073697A65206E6F7420706C61C6
:102A2000757369626C652E0A003F53706563696651
:102A3000696564207072696D65206C656E67746885
:102A4000206E6F7420706C61757369626C652E0AFC
:102A5000003F5072696D65206C656E677468206D0B
:102A60007573742062652073706563696669656457
:102A7000207768656E206E6F74207573696E6720AD
:102A8000616E204C43442E0A003F537065636966B3
:102A9000696564206E6F7A7A6C652073697A652047
:102AA0006E6F7420706C61757369626C652E0A00BC
:102AB0003F52657472616374696F6E204D756C74FA
:102AC00069706C696572206D75737420626520731E
:102AD00070656369666965642E0A003F53706563BB
:102AE00069666965642052657472616374696F6EAA
:102AF000204D756C7469706C696572206E6F7420FE
:102B0000706C61757369626C652E0A003F53706565
:102B1000636966696564206C6179657220686569BE
:102B2000676874206E6F7420706C61757369626C75
:102B3000652E0A0043292E0A003F537065636966BB
:102B4000696564206265642074656D706572617486
:102B5000757265206E6F7420706C61757369626C3C
:102B600065202834302D004732362073746172742A
:102B7000696E672E2E2E0A004F46460A0046616493
:102B800065204865696768742000426564204C656B
:102B900076656C696E6720004661696C65642074B7
:102BA0006F20656E61626C6520426564204C6576BD
:102BB000656C696E670A00496E76616C6964206DA8
:102BC0006573682E0A0050726F62696E6720506FDD
:102BD000696E740025532025692F2569002E0A008F
:102BE0002F0050726F62696E67206D657368207088
:102BF0006F696E742000202844525952554E2900A6
:102C0000473239204175746F20426564204C6576E7
:102C1000656C696E67003F20284C2C522C462C4274
:102C200029206F7574206F6620626F756E64732E35
:102C30000A003F2856296572626F7365206C6576BD
:102C4000656C20696D706C61757369626C652028B4
:102C5000302D34292E0A00426164205A2076616C9E
:102C600075650A004E6F2062696C696E656172203D
:102C7000677269640A004163637572616379204415
:102C8000656372656173696E67210044656372658F
:102C90006173696E67204163637572616379204473
:102CA000657465637465642E0A00473238004732E4
:102CB000385A0041636375726163793A2000206F6E
:102CC00066200044696420004733342061626F72DB
:102CD0007465642E0A0041636375726163792041F3
:102CE0006368696576656400546172676574206124
:102CF0006363757261637920616368696576656491
:102D00002E0A004469666673205A312D5A323D25D9
:102D100073000A444946464552454E4345205A31C0
:102D20002D5A323D0050726F62696E6720466169AC
:102D30006C65640050726F62696E67206661696CD1
:102D400065640A0047333420497465726174696FA1
:102D50006E3A202569000A47333420497465726150
:102D600074696F6E3A20003F2841296D706C696666
:102D700069636174696F6E206F7574206F6620627D
:102D80006F756E64732028302E352D322E30292E2B
:102D90000A003F2854296172676574206163637576
:102DA00072616379206F7574206F6620626F756E33
:102DB00064732028302E30312D312E30292E0A0018
:102DC0003F2849297465726174696F6E206F75744C
:102DD000206F6620626F756E64732028312D33304A
:102DE000292E0A003F285929206F7574206F66200C
:102DF000626F756E64732E0A003F285829206F7524
:102E000074206F6620626F756E64732E0A003F280F
:102E100053292050726F62652D706F736974696FEA
:102E20006E20696E64657820696E76616C69642EC7
:102E30000A003F28532920697320726571756972F1
:102E400065642E0A004D34323220530044657669A1
:102E50006174696F6E0025533A2025730046696ED0
:102E60006973686564210A003A207A3A2000206F6D
:102E7000662000476F696E6720746F3A20580043E0
:102E8000570A00206469723A0020616E676C653AE7
:102E9000005374617274207261646975733A004DF5
:102EA000343820506F696E740025533A2025642F02
:102EB000256400506F736974696F6E696E67207462
:102EC00068652070726F62652E2E2E0A003F4C6579
:102ED0006773206F66206D6F76656D656E7420690F
:102EE0006D706C61757369626C652028302D3135A9
:102EF000292E0A003F2028582C5929206F7574204C
:102F00006F6620626F756E64732E0A0050726F6276
:102F100065206F7574206F6620626F756E64730034
:102F20003F53616D706C652073697A65206E6F74B4
:102F300020706C61757369626C652028342D3530A2
:102F4000292E0A004D3438205A2D50726F626520A8
:102F50005265706561746162696C69747920546549
:102F600073740A003F2856296572626F7365206C7E
:102F70006576656C20696D706C61757369626C65EE
:102F80002028302D34292E0A005374616E6461723A
:102F90006420446576696174696F6E3A200020523E
:102FA000616E67653A2000204D61783A2000204D1F
:102FB000696E3A2000205369676D613A20004D65C3
:102FC000616E3A2000205200416363656C65726156
:102FD00074696F6E3A2050005741524E494E472156
:102FE000204C6F77205A204A65726B206D617920E2
:102FF0006C65616420746F20756E77616E746564B2
:10300000207061757365732E0A0070012C019001A8
:103010002701B0012201C0011D01F00118011002B9
:10302000130130020E016002090190020401C00286
:10303000FF000003FA004003F5008003F000D00316
:10304000EB002004E6007004E100E004DC00400531
:10305000D700C005D2004006CD00D006C8008007CA
:10306000C3003008BE00F008B900C009B400B00ABF
:10307000AF00B00BAA00D00CA500000EA000500FAE
:103080009B00C01096005012910000148C00C015D7
:103090008700B0178200B0197D00D01B7800001E99
:1030A000730040206E0090226900F02464004027E5
:1030B0005F0090295A00E02B5500102E5000203060
:1030C0004B0010324600E033410090353C00103791
:1030D000370070383200A0392D00B03A2800A03BEC
:1030E0002300603C1E00103D1900903D1400103E6E
:1030F0000F00703E0A00C03E0500003F0000403F48
:10310000FBFF803FF6FFC03FF1FF50726F62696EB8
:1031100067204661696C656400205A3A2000205996
:103120003A200042656420583A20003D3D6F6E55BC
:10313000736572436F6E6669726D526571756972FF
:1031400065643D3D00220A00556E6B6E6F776E2000
:10315000636F6D6D616E643A202200204200205042
:10316000006F6B00204500205A00205900204D3987
:103170003220580020453A00205A3A0020593A009F
:10318000583A0020746F6F206C6F6E6720657874FA
:10319000727573696F6E2070726576656E746564A2
:1031A0000A0020636F6C6420657874727573696FB0
:1031B0006E2070726576656E7465640A0043616E98
:1031C0006E6F7420656E74657220737562646972C7
:1031D0003A20004D323520500A4D3234005265738A
:1031E000756D65005549205061757365004E6F20FF
:1031F0004D61746368203A00506755700050674411
:103200006F776E0049732046696C65200049732012
:103210004469722000476F557044697200486173B9
:10322000204D656469610046696C656E616D65205D
:1032300053656C6563746564004D31303030430014
:103240004D313030300046696C616D656E742053CD
:103250007461742030202D20330046696C616D65E7
:103260006E7420537461742030202D203200466922
:103270006C616D656E7420537461742030202D2054
:1032800031002046696C616D656E74205265737003
:103290006F6E7365204E6F00526573756D652059B2
:1032A000657320647572696E67207072696E740050
:1032B0000A204E6F2046696C616D656E7400496E20
:1032C00076616C6964204F7074696F6E004D3530A3
:1032D000300053746F72652053657474696E677340
:1032E00000426564205049442053746172746564DF
:1032F000004D3939390A4D3238305030533136307B
:1033000000424C546F756368205265736574004DBC
:103310003530320A4D35303000496E6974204545EC
:1033200050524F4D00486F74656E642050494420E0
:103330005374617274656400456E676C69736820CC
:10334000416C726561647920536574004368696EED
:10335000657365204E6F7420537570706F7274655D
:103360006400496E4C616E6743686F696365000A6B
:10337000202A2A2A7265636461742E646174615B19
:10338000305D203D004732380A4731204631303029
:1033900030205A313000556E737570706F727465DD
:1033A00064204F7074696F6E2053656C656374653B
:1033B000640047323652323535004D31393053359D
:1033C000350A4732380A47333449380A4732390A0E
:1033D0004D3430300A4D313034533231350A4732B2
:1033E000380A4D313039533231350A4D3432305389
:1033F000310A47315831303059313030463530306C
:10340000300A47315A300A4D3530300A4D313137A4
:1034100020536574205A204F6666736574004731E7
:10342000204631303030205A302E30004732380AB2
:103430004731204631303030205A302E30004D3563
:103440003030005A204F6666736574203A20257329
:10345000004D353030005A204F6666736574203A4F
:10346000202573004732380A473146313530305A0B
:10347000302E30004732385A0A4731463135303025
:103480005A302E30004D383400473146313030301C
:103490005A302E30004732380A473146313030300A
:1034A0005A302E30004D616E75616C5365745465F1
:1034B0006D70005A204F6666736574203A2025733C
:1034C0000053746F70205472696767657265640099
:1034D00053746F70204E6F0053746F705072696E2A
:1034E000740048616E646C652044617461204164BD
:1034F0006A75737420322053657474696E67205343
:10350000637265656E200048616E646C652044617D
:103510007461205072696E7446696C652033205363
:10352000657474696E672053637265656E20004828
:10353000616E646C652044617461205072696E74C0
:1035400046696C6520322053657474696E67205338
:10355000637265656E20004D38340048616E646C9E
:10356000652044617461205072696E7446696C65AF
:1035700020506F73740048616E646C652044617400
:1035800061205072696E7446696C652050726500E6
:10359000426567696E537769746368003D3D2043F7
:1035A0006865636B6B65793D3D007265636461744A
:1035B0002E61646472203D3D007265636461742E07
:1035C000646174615B305D203D3D007761697477B3
:1035D0006179203D3D0020202A2A2A2A2A2A2A52BF
:1035E00054535F48616E646C65446174612A2A2A91
:1035F0002A2A2A2A2A2000526573656E643A20001E
:1036000000002200250028002B002E00310034008D
:1036100002010000050108010B0100002100240047
:1036200027002A002D0030003300010100000401B2
:1036300007010A0105050505070508080808020233
:1036400002020A0A0808040404040101010101013C
:1036500001010303030303030303040707070C0C1F
:103660000C0C0C0C0C0C02020202060606060606E6
:1036700006060B0B0B0B0B0B0B0B0102102020088B
:1036800008102040102040800201020108040201BD
:10369000010204081020408080402010080402012C
:1036A0008004020180402010080402010804020185
:1036B000010204081020408001020408102040800C
:1036C000544D334420453520506C7573205265614C
:1036D00064792E005072696E74696E672E2E2E000A
:1036E0005072696E7420506175736564006E6F74FA
:1036F000696669636174696F6E20005049442054A3
:10370000756E652046696E69736865640000E00047
:103710009A0011241FBECFEFD1E2DEBFCDBF00E083
:103720000CBF14E0A0E0B2E0EEE4FAE702E00BBF69
:1037300002C007900D92A832B107D9F726E1A8E29E
:10374000B4E001C01D92AF3CB207E1F71BE1C8E84D
:10375000DBE100E006C021970109802FFE010F94F4
:103760005439C738D10780E00807A9F70F94A62677
:103770000D94153D0C9400009F92AF92BF92CF9292
:10378000DF92EF92FF920F931F93CF93DF9300D0BE
:103790001F921F92CDB7DEB7E9E1F1E10027BB2709
:1037A000462F572FA82FAA2341F4A52F542FB85FD7
:1037B000AA2319F4A52F5527B85FA03138F45295E4
:1037C000A295452F4F70507FA42BBC5FA03428F4E6
:1037D000550FAA1F550FAA1FBE5FA03818F4550F2A
:1037E000AA1FB395550FAA1FEA0FF01F449151E08D
:1037F000AA27B85081F1C8F0B0FF02C0440F551F8E
:10380000B1FF04C0440F551F440F551FB2FF06C03F
:1038100052954295142F1F70407F512BB3FF1BC050
:10382000A52F542F44270C942B1CB195B0FF02C038
:1038300055954795B1FF04C05595479555954795C2
:10384000B2FF05C05295407F4295452B5F70B3FF94
:1038500002C0452F5527DD24CC24BB24B2E0649F51
:10386000D018C108B00AB00B749FC018B108B00BD3
:10387000849FB018B109659FC018B108B00B759F3F
:10388000B018B109859FB0196A9FB018B1097A9F25
:10389000B0194D9DA12C99243327992722275D9D8E
:1038A000A00C911C301F901F201FAD9D900C311D4E
:1038B000901F201F4C9DA00C911C301F901F201F9B
:1038C0005C9D900C311D901F201FAC9D300D911DF3
:1038D000201F4B9D900C311D901F201F5B9D300DB4
:1038E000911D201FAB9D900D211D4B9F300D911DF3
:1038F000201F5B9F900D211DAB9F200DB1E0BB24CD
:10390000CC24DD24639FD018C108B00AB00B739F8C
:10391000C018B108B00B839FB018B109699FC018D7
:10392000B108B00B799FB018B109899FB019629F97
:10393000B018B109729FB019D61AC70AB80A20F098
:10394000B1E03B0F901F201F1124792F632F90E0CF
:10395000822F0F900F900F900F900F90DF91CF91CB
:103960001F910F91FF90EF90DF90CF90BF90AF909D
:103970009F900895AF92BF92CF92DF92EF92FF9205
:103980000F931F93CF93DF93CDECDCE000E219E0BF
:103990008DEDA82E8CE0B82EC12CD12C7601C394CD
:1039A00069917991899199910F94923228893989F5
:1039B0004A895B890F94F3320F94D03AF8016193EE
:1039C0007193819391938F01C616D706E806F90685
:1039D00010F46B017C01AC16BD0611F76FEF7FEFA1
:1039E000CB01A70196010F94D13820933009309371
:1039F00031094093320950933309DF91CF911F91E0
:103A00000F91FF90EF90DF90CF90BF90AF9008950F
:103A1000CF93DF9324E0829FC0011124EC01CD5E9F
:103A2000D64FFC01E75BF74F835C974FDC012D918C
:103A30003D914D915C9160817181828193810F9460
:103A40005D39688379838A839B83DF91CF91089561
:103A50008091181390911913891B877089F48091B4
:103A6000200E81110DC08091150D9091160D892B9E
:103A700039F481E09091DE05911103C080E0089552
:103A800081E0089590E080E00895282F9091370814
:103A9000833021F495FD0FC094FD0FC0892F90E075
:103AA000B0E0A0E004C0B695A795979587952A95B4
:103AB000D2F78170089581E0089580E00895CF9352
:103AC000C82FCB010E94B4C78DE89EE00E94B4C706
:103AD0008EE79EE0CC2311F083E89EE00E94B4C7FD
:103AE0008AE0CF910C948CC70F931F93CF938C01D6
:103AF000C62F80EE99E00E94B4C7C8010E94B4C7E7
:103B00008AE30E948CC780E38C0F0E948CC78AE0F6
:103B1000CF911F910F910C948CC783E69BE00E947C
:103B2000B4C760E083E59BE00E94741D60E08EE313
:103B30009BE00E94741D61E087E39BE00E94741D7E
:103B400061E08CE29BE00E94741D61E08CE19BE0EF
:103B50000E94741D60E083E19BE00E94741D61E09F
:103B600089E09BE00E94741D61E08FEF9AE00E9463
:103B7000741D61E088EF9AE00E94741D61E080EF9F
:103B80009AE00E94741D61E082EE9AE00E94741D2A
:103B900061E084ED9AE00E94741D60E085EC9AE09B
:103BA0000E94741D60E087EB9AE00E94741D60E043
:103BB00081EA9AE00E94741D61E080E99AE00E9427
:103BC000741D61E081E89AE00E94741D61E08AE75B
:103BD0009AE00E94741D60E083E79AE00E94741DE1
:103BE00061E08AE69AE00E94741D61E085E59AE052
:103BF0000E94741D61E087E49AE00E94741D61E0F8
:103C000084E39AE00E94741D60E087E29AE00E94DB
:103C1000741D61E082E29AE00E94741D61E085E11A
:103C20009AE00E94741D60E081E09AE00E94741D99
:103C300060E08EEE99E00E94741D60E083ED94E1F7
:103C40000E94421D682F617085EE99E00C94741DEE
:103C5000CF93DF938091181390911913891B80954E
:103C6000877019F40E94C3DFF5CF809118138F5F1E
:103C70008770A091181397E6A99FD0011124FD0128
:103C8000E35BF64FEF0119929A95E9F798E090837C
:103C9000AE59B64F90E1EAE2F3E101900D929A95A8
:103CA000E1F72091181390911913291303C094E69A
:103CB0009093151380931813DF91CF910C94C7C282
:103CC0002F923F924F925F926F927F928F929F922C
:103CD000AF92BF92CF92DF92EF92FF920F931F931A
:103CE000CF93DF93D62FC72FFC0180809180A280D5
:103CF000B380C501B40120E831E541E050E00F9404
:103D0000D138C9016DE671E00F9440396B017C0137
:103D1000C501B40120E13EE040E050E00F94D1380D
:103D2000CA01B90128E130E040E050E00F94D138F9
:103D3000362E272E062F172F8CE3482E512C612C60
:103D4000712CC501B401A30192010F94D138B62E94
:103D5000A72ECA01B901A30192010F94D138CB015A
:103D6000C114D10479F1AF92BF927F936F932F92D8
:103D70003F92FF92EF92DF92CF9280E29DE09F937D
:103D80008F93CF93DF930F9424328DB79EB70E9607
:103D90000FB6F8949EBF0FBE8DBF8D2F9C2FDF9165
:103DA000CF911F910F91FF90EF90DF90CF90BF9038
:103DB000AF909F908F907F906F905F904F903F90CB
:103DC0002F900895E114F104C9F0AF92BF927F9350
:103DD0006F932F923F92FF92EF9280E19DE09F932D
:103DE0008F93CF93DF930F942432EDB7FEB73C96B9
:103DF0000FB6F894FEBF0FBEEDBFCFCF012BB9F0C9
:103E0000AF92BF927F936F932F923F9284E09DE099
:103E10009F938F93CF93DF930F9424328DB79EB7E8
:103E20000A960FB6F8949EBF0FBE8DBFB6CF892BF2
:103E3000A9F0AF92BF927F936F938CEF9CE09F931A
:103E40008F93CF93DF930F942432EDB7FEB738965C
:103E50000FB6F894FEBF0FBEEDBF9FCFAF92BF92DB
:103E600088EF9CE09F938F93CF93DF930F9424323E
:103E70000F900F900F900F900F900F908ECFCF93C9
:103E8000DF9300D01F92CDB7DEB784EF91E0A0E0C2
:103E9000B0E089839A83AB83BC83BE016F5F7F4FA1
:103EA0008CE30E9450C58BEA9EE00E94B4C78CB19F
:103EB00065EA7EE085FB882780F90E945F1D80917E
:103EC00003016FE97EE0869581700E945F1D89B1D4
:103ED00069E97EE083FB882780F90E945F1D8CB131
:103EE00060E97EE0829581700E945F1D4B9909C058
:103EF0000E948BC50F900F900F900F90DF91CF9184
:103F000008950E9470C50F900F900F900F90DF9151
:103F1000CF91089580911E06882319F010921E06F5
:103F2000089540E070E060E080E79EE00E94F2DEED
:103F3000CF93C091AF04CF7739F50E94E3C38823B4
:103F400019F18091C8149091C914A091CA14B0912C
:103F5000CB140097A105B105B9F0BC01CD016D5995
:103F60007F4F8F4F9F4F24E630E040E050E00F94AA
:103F7000D1386091CC147091CD148091CE14909171
:103F8000CF140F94D138C22F8C2FCF910895CF9397
:103F9000DF93EB010E9481BE882319F00E94D1BDFE
:103FA000EB01CE01DF91CF9108954F925F926F9216
:103FB0007F928F929F92AF92BF92CF92DF92EF92B9
:103FC000FF921F93CF93DF9300D01F92CDB7DEB740
:103FD00019821A821B821C82CE0101964C0187EB4A
:103FE000C82E87E0D82E99E6E92E92E0F92E23E13B
:103FF000A22E29E0B22E10E088E5810F0E9481BE3A
:10400000F40181934F01882309F4E0C00E9409BEA6
:104010002B013C01812F0E94451D882309F4CCC04F
:10402000F7012081318142815381C301B2010F9494
:104030005D39F60160837183828393831F5FF4E0AF
:10404000CF0ED11C84E0E80EF11C94E0A90EB11C47
:10405000133091F685E40E9481BE8C83882309F495
:10406000C0C00E9409BE6B017C0183E00E94451D17
:10407000882371F020917502309176024091770289
:1040800050917802C701B6010F945D396B017C0134
:10409000C092C307D092C407E092C507F092C6074A
:1040A0008091F004882359F18091D01482FF27C0B9
:1040B0008C81882321F18981811103C08A81882321
:1040C000F1F02DEC3CEC4CE45DE360915E08709106
:1040D0005F0880916008909161080F945D399B01A1
:1040E000AC016091710270917202809173029091A3
:1040F00074020F94BD3B181614F40F94002140E095
:1041000050E0BA0186E40E94EEBE20E030E0A90152
:104110000F94BD3B181684F40E9409BE20E030E0E5
:1041200040E752E40F94573A6093490270934A0271
:1041300080934B0290934C028091850C83FD28C0A4
:104140008091C905882321F1209175023091760272
:1041500040917702509178026091C3077091C40733
:104160008091C5079091C6070F945C392091D605C0
:104170003091D7054091D8055091D9050F945D39FC
:104180006093D6057093D7058093D8059093D90591
:104190000F900F900F900F90DF91CF911F91FF9094
:1041A000EF90DF90CF90BF90AF909F908F907F90D7
:1041B0006F905F904F900895F50120813181428189
:1041C0005381C301B2010F945C3933CFF701808171
:1041D0009181A281B381F60180839183A283B3830D
:1041E0002DCF8091750290917602A0917702B091C7
:1041F00078028093C3079093C407A093C507B09338
:10420000C6074ECFCF9384E50E9481BEC0E08823CD
:10421000D9F00E94E1BDC82F1816B4F40E9418DC32
:104220008DE40E948CC78091A0049091A1040E940B
:1042300054F26C2FCC0F770B8DE495E00E947BCA73
:104240008AE00E948CC7CFEF8C2FCF910895CF9238
:10425000DF92EF92FF920F931F93CF93DF93CDB72F
:10426000DEB7A0970FB6F894DEBF0FBECDBF0E9499
:10427000022187FDCCC085E40E9433BE882309F467
:10428000D5C00E9409BE6B017C0120E030E0A9018D
:104290000F94BD3B87FF04C0F7FAF094F7F8F09451
:1042A000F7FAF094F7F8F094CD8EDE8EEF8EF8A248
:1042B0008CE0E3E9F2E0DE01119601900D928A951F
:1042C000E1F78AE50E9481BE882351F040E050E08A
:1042D000BA018AE50E94EEBE69877A878B879C8740
:1042E00088E50E9481BE882351F040E050E0BA0189
:1042F00088E50E94EEBE69837A838B839C8389E57F
:104300000E9481BE882351F040E050E0BA0189E567
:104310000E94EEBE6D837E838F83988785E50E9421
:1043200033BE882309F489C00E9409BE6B017C0159
:1043300020E030E0A901C701B6010F94BD3B87FF23
:1043400004C0F7FAF094F7F8F094F7FAF094F7F85D
:10435000F094C98EDA8EEB8EFC8E1D8A1E8A1F8A1F
:10436000188E8CE40E9433BE882309F46FC00E942B
:1043700009BE6B017C0120E030E0A901C701B60154
:104380000F94BD3B87FF04C0F7FAF094F7F8F09460
:10439000C98ADA8AEB8AFC8A62E070E082E40E94D1
:1043A00005BFF82E8091B211811131C021E0AE011C
:1043B000475E5F4FBE016F5F7F4FCE014D960E94FB
:1043C00072EE882321F16F2D81E00E9444EF82E597
:1043D0000E9481BE882309F442C00E9405BE40E0CD
:1043E00050E060EA71E44D875E876F87788B20919B
:1043F000B211222361F08C012F2DAE01435F5F4F7C
:10440000BE016F5E7F4FCE0145960E942FEDA096B4
:104410000FB6F894DEBF0FBECDBFDF91CF911F91D5
:104420000F91FF90EF90DF90CF900895C12CD12C89
:1044300080E8E82E80E4F82E33CFC090E804D090D6
:10444000E904E090EA04F090EB0472CFC090EC0431
:10445000D090ED04E090EE04F090EF048CCF90E06B
:1044600080E0BDCFCF92DF92EF92FF920F931F9328
:10447000CF93DF93CDB7DEB76C970FB6F894DEBF5E
:104480000FBECDBF8CE40E9433BE882309F4B0C0B8
:104490000E9409BE6B017C0120E030E0A9010F946D
:1044A000BD3B87FF04C0F7FAF094F7F8F094F7FAF1
:1044B000F094F7F8F094C98EDA8EEB8EFC8E8CE0D7
:1044C000E3E9F2E0DE01119601900D928A95E1F7A1
:1044D00088E50E9481BE8823A1F040E050E0BA0147
:1044E00088E50E94EEBE2091130930911409409195
:1044F0001509509116090F945C3969837A838B836F
:104500009C8389E50E9481BE8823A1F040E050E0B1
:10451000BA0189E50E94EEBE209113093091140979
:1045200040911509509116090F945C396D837E8373
:104530008F8398878AE50E9481BE882351F040E0EE
:1045400050E0BA018AE50E94EEBE69877A878B87C0
:104550009C871D861E861F86188A8091B211811144
:1045600038C020E0AE01435F5F4FBE016F5F7F4FF9
:10457000CE0149960E9472EE882359F18091F00491
:1045800081110F94002160E080E00E9444EF898D4A
:104590009A8DAB8DBC8DB0588D8B9E8BAF8BB88FA9
:1045A000198A1A8A1B8A1C8A1D861E861F86188AEB
:1045B0008091B211882369F010E000E020E0AE01A4
:1045C0004B5E5F4FBE016F5E7F4FCE010D960E9426
:1045D0002FED6C960FB6F894DEBF0FBECDBFDF9106
:1045E000CF911F910F91FF90EF90DF90CF900895A2
:1045F000C12CD12C80E8E82E80E4F82E58CF84E638
:1046000090E09093E7048093E604109217051092CF
:1046100016050C9420AF0F93AB010091150521E016
:10462000022726E135E0BC0186EE94E00E940DC42D
:104630000F910895CF93DF9300D01F92CDB7DEB7CF
:104640008091C9058823C1F083E390E09C838B832C
:104650001A8219829E012F5F3F4F40E150E06AECC1
:1046600075E0CE0103960E9482DE8DE592E10E9404
:10467000B4C78AE00E948CC70F900F900F900F90E4
:10468000DF91CF910895CF93DF9300D01F921F92B7
:10469000CDB7DEB781E08093C90580E1EAECF5E0B3
:1046A000DF011D928A95E9F70E941A2386E18D8326
:1046B00082E390E09C838B831A8219829E012F5F94
:1046C0003F4F41E050E0BE016B5F7F4FCE0103964C
:1046D0000E9482DE0F900F900F900F900F90DF914D
:1046E000CF910895CF92DF92EF92FF92CF93DF9315
:1046F000EC0108960E94F1B96B017C0120E030E0EA
:10470000A9010F948D3220E030E0A901882359F0EF
:10471000CE010E94DABF9B01AC01C701B6010F9424
:10472000F3329B01AC01688579858A859B850F945E
:104730005C39688779878A879B87DF91CF91FF9063
:10474000EF90DF90CF9008958C3221E0920714F023
:104750008CE291E090937D1280937C120C9411F185
:104760000F931F93CF93DF9301EE1CE0C5EFD1E1D0
:10477000F80121913191419151918F0160E070E0F8
:1047800080E89FE30F94573A6993799389939993BB
:10479000F2E1C530DF0761F70F943F1FDF91CF9142
:1047A0001F910F910C94BA1C9091181380911913BA
:1047B000981306C080914B0990914C09892B21F0E8
:1047C00080E00E94C3DFF0CF08959091181380918C
:1047D0001913981308C080914B0990914C09892BAB
:1047E00011F40C94C9C380E00E94C3DFEECFCF92D6
:1047F000DF92EF92FF92CF93DF932091C80C222398
:1048000029F1EC0108960E94F1B96B017C0120E0CE
:1048100030E0A9010F948D3220E030E0A901882317
:1048200059F0CE010E94DABF9B01AC01C701B6016D
:104830000F94F3329B01AC01688579858A859B854D
:104840000F945D39688779878A879B87DF91CF913D
:10485000FF90EF90DF90CF900895CF92DF92EF928C
:10486000FF9280913C08882309F457C0C090380813
:10487000D0903908E0903A08F0903B0820E030E012
:10488000A901C701B6010F948D32882309F445C0F0
:1048900020E030E040E05FE3C701B6010F94F3325F
:1048A0009B01AC010F94F3322BED3FE049E450E45F
:1048B0000F94F3329B01AC0160E070E080E89FE36D
:1048C0000F94573A6B017C01C092C90CD092CA0C6C
:1048D000E092CB0CF092CC0C60917D0270917E0244
:1048E000072E000C880B990B0F9494322AE037EDB9
:1048F00043E25CE30F94F332A70196010F94F33285
:104900006093790270937A0280937B0290937C0289
:10491000FF90EF90DF90CF900895C12CD12C80E8CC
:10492000E82E8FE3F82ED0CF0F931F93CF93DF9312
:1049300050E0FC01E40FF51F8081440F551F440F28
:10494000551F4A535B4FEA01882329F188819981D9
:10495000AA81BB81EB01088119812A813B810097E3
:10496000A105B10569F40C591F4F2F4F3F4FDA01D4
:104970000D931D932D933C9313978FEF808306C067
:10498000081B190B2A0B3B0B37FDF7CFDF91CF919B
:104990001F910F910895188219821A821B82F6CFF7
:1049A0002F923F924F925F926F927F928F929F923F
:1049B000AF92BF92CF92DF92EF92FF920F931F932D
:1049C000CF93DF93CDB7DEB76C970FB6F894DEBF09
:1049D0000FBECDBF8C015B015A834983FC01EF5AA6
:1049E000FF4F208131814281538129873A874B874C
:1049F0005C87CA01B9010F9492326B017C01D50129
:104A00002D913D914D915C910F94F3320F943B3A6F
:104A10002B013C01E981FA8120813181428153815E
:104A2000C701B6010F94F3320F943B3A4B015C017E
:104A3000C301B2010F94D03A698B7A8B8B8B9C8B1C
:104A4000683771058105910540F428E730E040E0C2
:104A500050E0298B3A8B4B8B5C8BC501B4010F94D2
:104A6000D03A6D877E878F87988B6837710581056F
:104A7000910540F448E750E060E070E04D875E87C4
:104A80006F87788BF801E35AFF4F40805180628036
:104A90007380C301B2010F94943269837A838B834C
:104AA0009C8369897A898B899C890F9492326D8B5A
:104AB0007E8B8F8B988F20E030E0A90169817A810D
:104AC0008B819C810F948D32882309F4E1C1A70169
:104AD0009601C701B6010F94F3324B015C012D8999
:104AE0003E894F89588DCA01B9010F94F3329B0159
:104AF000AC01C501B4010F945C394B015C01298103
:104B00003A814B815C81CA01B9010F945D399B01E7
:104B1000AC01C501B4010F94573A0F943B3A0F947E
:104B2000D03A6D837E838F83988766277727CB0162
:104B300064197509860997090F9494324B015C0139
:104B40006D857E858F8598890F9492322B013C016B
:104B500020E030E0A901C501B4010F948D32882313
:104B600009F49AC1A3019201C301B2010F94F33277
:104B7000698F7A8F8B8F9C8FA7019601C701B60131
:104B80000F94F3329B01AC01698D7A8D8B8D9C8DD6
:104B90000F945C396B017C01A5019401C501B4013E
:104BA0000F945D399B01AC01C701B6010F94573AD0
:104BB0000F94FF3AD80195968D909D90AD90BC9042
:104BC0009897750164012D813E814F815885C21AE5
:104BD000D30AE40AF50A0F94D03AC61AD70AE80AAB
:104BE000F90AF7FE8EC02D893E894F89588DCA017A
:104BF000B9010F94F3326B017C0129813A814B8119
:104C00005C81CA01B9010F945D3969877A878B8706
:104C10009C8720E030E0A90169817A818B819C81A9
:104C20000F948D32882309F43BC1C501B4010F9460
:104C3000923229853A854B855C850F94F332A70122
:104C400096010F945C396D837E838F839887A301CF
:104C50009201C301B2010F94F3329B01AC016D814B
:104C60007E818F8198850F945D392B013C0120E076
:104C700030E040E850E469817A818B819C810F9417
:104C8000F3329B01AC01C301B2010F94573A0F9468
:104C90003B3A2B013C0120E030E0A9010F94BD3BE1
:104CA00018161CF0412C512C3201C301B2010F9493
:104CB000D03A6D837E838F83988786169706A806E1
:104CC000B90620F48D829E82AF82B8866D817E8186
:104CD0008F8198850F94923229853A854B855C8522
:104CE0000F94F332A70196010F945D390F940B3C9A
:104CF0000F94D03A69877A878B879C87C12CD12CF7
:104D0000760169857A858B859C8529893A894B89C5
:104D10005C89621B730B840B950B0F949232298173
:104D20003A814B815C810F94573A20E034E244EFA2
:104D300059E40F94F3320F94D03A4B015C0169852A
:104D40007A858B859C852D853E854F855889621B8C
:104D5000730B840B950B0F94923229813A814B810E
:104D60005C810F94573A20E034E244EF59E40F9409
:104D7000F3320F94D03A2B013C013FE683169104A5
:104D8000A104B10408F090C0F401EE0FFF1FEE0F74
:104D9000FF1FE35AF04F85919591A591B4918983B6
:104DA000292E3A2EBD8B4FE644165104610471043E
:104DB00008F083C0F201EE0FFF1FEE0FFF1FE35A52
:104DC000F04F45915591659174919A01CB014D81B8
:104DD0005E816F817885D80199964D935D936D932F
:104DE0007C939C974C0D5D1D6E1D7F1DF80145A7A2
:104DF00056A767A770ABEB5AFF4F49895A896B8951
:104E00007C894083518362837383D5968D929D9272
:104E1000AD92BC92D897F80141AE52AE63AE74AE7B
:104E2000FD9649814083218232825D895383349685
:104E3000208331838283938369857A858B859C85E2
:104E4000D1966D937D938D939C93D49778962D8571
:104E50003E854F85588920833183428353836C96E6
:104E60000FB6F894DEBF0FBECDBFDF91CF911F917B
:104E70000F91FF90EF90DF90CF90BF90AF909F90F9
:104E80008F907F906F905F904F903F902F900895FC
:104E900060E070E0CB0141CE60E070E0CB0188CEF5
:104EA00060E070E0CB01F3CEC501B4010E94BC1BF1
:104EB0006983272E382E9D8B76CFC301B2010E94C5
:104EC000BC1B9B0184CF8091181390911913891BEF
:104ED000877019F490E080E008959091151399235C
:104EE00051F0833030F48FEF890F19F08093151350
:104EF000F1CF109215138091191327E6829FC001FC
:104F00001124835B964FFC01208120FDE3CF20918B
:104F100019132F5F277020931613309119132091C6
:104F20001713321304C020911613209317130895FA
:104F300090916F0081E091FD02C080E00895909112
:104F40006F009D7F90936F000895CF92DF92EF9254
:104F5000FF92FC01C080D180E280F3802091ED0CB3
:104F60003091EE0C4091EF0C5091F00CC701B6015E
:104F70000F94F3320F94CA3B609336137093371338
:104F80008093381390933913C0922613D09227132D
:104F9000E0922813F092291390911813809119131D
:104FA000981731F0FF90EF90DF90CF900C94281E6F
:104FB0000E94D4230E9498274091361350913713B2
:104FC0006091381370913913409342055093430513
:104FD0006093440570934505882331F0FF90EF906E
:104FE000DF90CF900C94C7C2FF90EF90DF90CF90EE
:104FF00008954F925F926F927F928F929F92AF929D
:10500000BF92CF92DF92EF92FF920F931F93CF93B5
:10501000DF93EC018B017A016901F90180819181B3
:10502000A281B381FA014081518162817381F801CB
:1050300080809180A280B380488059806A807B8084
:1050400040921A1350921B1360921C1370921D13FE
:1050500080921E1390921F13A0922013B0922113DE
:1050600040932213509323136093241370932513BA
:105070008093261390932713A0932813B09329139A
:105080002091ED0C3091EE0C4091EF0C5091F00C12
:10509000F60160817181828193810F94F3320F94C4
:1050A000CA3B4B015C012091E90C3091EA0C409124
:1050B000EB0C5091EC0CF70160817181828193813E
:1050C0000F94F3320F94CA3B6B017C012091E50CE5
:1050D0003091E60C4091E70C5091E80CF8016081AA
:1050E0007181828193810F94F3320F94CA3B2B011B
:1050F0003C012091E10C3091E20C4091E30C509185
:10510000E40C688179818A819B810F94F3320F943A
:10511000CA3B60932A1370932B1380932C139093A4
:105120002D1340922E1350922F13609230137092D1
:105130003113C0923213D0923313E0923413F092B1
:1051400035138092361390923713A0923813B09291
:1051500039139091181380911913981791F0DF91DA
:10516000CF911F910F91FF90EF90DF90CF90BF9064
:10517000AF909F908F907F906F905F904F900C9426
:10518000281E0E94D4230E949827409132135091E8
:105190003313609134137091351300912E131091D5
:1051A0002F132091301330913113C0902A13D090D7
:1051B0002B13E0902C13F0902D13C0923605D09253
:1051C0003705E0923805F092390500933A051093BF
:1051D0003B0520933C0530933D0540933E0550939D
:1051E0003F056093400570934105409136135091FF
:1051F00037136091381370913913409342055093DF
:1052000043056093440570934505882391F0DF9131
:10521000CF911F910F91FF90EF90DF90CF90BF90B3
:10522000AF909F908F907F906F905F904F900C9475
:10523000C7C2DF91CF911F910F91FF90EF90DF9048
:10524000CF90BF90AF909F908F907F906F905F9026
:105250004F900895CF92DF92EF92FF92CF93DF931A
:10526000C82F0E94982794E0C99FE0011124FE01F5
:10527000EA5CFA4FC080D180E280F38081110E9405
:10528000C7C2CB50DE4EC701B6010F9494322881BD
:1052900039814A815B810F94F332DF91CF91FF9086
:1052A000EF90DF90CF9008953F924F925F926F9270
:1052B0007F928F929F92AF92BF92CF92DF92EF92A6
:1052C000FF920F931F93CF93DF93CDB7DEB768970D
:1052D0000FB6F894DEBF0FBECDBFD82E2A013B011A
:1052E000480159013E2C20E030E0A901C501B80178
:1052F0000F948D32811110C081E08D1508F0B6C079
:1053000060E070E080E793E420E030E040E752E4C2
:105310000F94573A4B015C018D8A9E8AAF8AB88EF2
:105320000D2D10E0F801E65AF04FE491BB24B39440
:105330001E160CF4B12CCC24C39420E030E0A9015B
:10534000C301B2010F94BD3B18160CF0C12CBC1464
:1053500071F092E0D9120BC0332049F081E00F9434
:10536000C72269E170E080E090E00E94E4C280E042
:105370000E942A2969837A838B839C8381E00E941F
:105380002A296D837E838F83988782E00E942A2951
:1053900069877A878B879C8783E00E942A296D879B
:1053A0007E878F87988B000F111F000F111FE1E080
:1053B000F0E0EC0FFD1F0E0F1F1FF801108211828D
:1053C000128213829E01235F3F4FAE01475F5F4F02
:1053D000BE016B5F7F4FCE0101960E94F927F80155
:1053E0004082518262827382198A1A8A1B8A1C8ABD
:1053F00080914B0990914C09892B91F4CE014196F3
:105400007C018E010B5E1F4F9E01235F3F4FAE015B
:10541000475F5F4FBE016B5F7F4F40970E9470F800
:105420000E94D423BC1451F092E0D91205C033205D
:1054300019F080E00F94C7220E948A1F68960FB669
:10544000F894DEBF0FBECDBFDF91CF911F910F91BA
:10545000FF90EF90DF90CF90BF90AF909F908F9094
:105460007F906F905F904F903F90089560E070E85C
:105470008BE395E449CFCF92DF92EF92FF92CF93E7
:10548000DF93C82F0E94982794E0C99FE001112460
:10549000FE01E65DFA4FC080D180E280F380811189
:1054A0000E94C7C2CB50DE4EC701B6010F949432A2
:1054B000288139814A815B810F94F332DF91CF914A
:1054C000FF90EF90DF90CF9008950E9498279091E1
:1054D000191390931813909317139093161394E63F
:1054E0009093151320ED33E030934C0920934B0932
:1054F00081110E94C7C281E080932905089580FF31
:1055000004C09091C70C90FD8E7F81FF05C09091E3
:10551000C70C969590FD8D7F82FF06C09091C70CB9
:105520009695969590FD8B7F08958F929F92AF925E
:10553000BF92CF92DF92EF92FF92CF93DF932091B1
:105540004D02222309F49EC0EC0180919A04C82EDA
:10555000D12CF12CE12C80FF2CC080904F02909038
:105560005002A0905102B0905202288139814A81A4
:105570005B81C501B4010F94BD3B181624F48882E9
:105580009982AA82BB8280905B0290905C02A0907C
:105590005D02B0905E02288139814A815B81C5013C
:1055A000B4010F948D3287FF04C088829982AA8249
:1055B000BB82D701C601B695A7959795879580FFC1
:1055C0002CC08090530290905402A0905502B0904D
:1055D00056022C813D814E815F81C501B4010F943B
:1055E000BD3B181624F48C829D82AE82BF828090CF
:1055F0005F0290906002A0906102B09062022C81E4
:105600003D814E815F81C501B4010F948D3287FFCA
:1056100004C08C829D82AE82BF8282E0F694E794C1
:10562000D794C7948A95D1F7C0FE2CC0C09057027A
:10563000D0905802E0905902F0905A02288539859E
:105640004A855B85C701B6010F94BD3B181624F44B
:10565000C886D986EA86FB86C0906302D090640231
:10566000E0906502F0906602288539854A855B8561
:10567000C701B6010F948D3287FF04C0C886D98652
:10568000EA86FB86DF91CF91FF90EF90DF90CF907D
:10569000BF90AF909F908F9008952F923F924F921E
:1056A0005F926F927F928F929F92AF92BF92CF92B2
:1056B000DF92EF92FF920F931F93CF93DF93CDB7BB
:1056C000DEB7A6970FB6F894DEBF0FBECDBF87EB4F
:1056D00097E00E94952A8091850C83FD7EC02091E1
:1056E0007502309176024091770250917802609174
:1056F000C3077091C4078091C5079091C6070F94A6
:105700008D32882309F469C010914A09111161C0D2
:105710008091670290916802019720917A123091EE
:105720007B12281739073CF40E9418DC84EE9EE0B7
:105730000E94B4C711E02091750230917602409129
:105740007702509178026091C3077091C4078091ED
:10575000C5079091C6070F945C396B017C0120E06E
:1057600030E0A9010F94BD3B87FF04C0F7FAF09425
:10577000F7F8F0942091790230917A0240917B02FF
:1057800050917C02C701B6010F94F33220E030E85B
:105790004BE354E40F94BD3B1816ECF40E9418DC64
:1057A00085EC9EE00E94B4C78091C3079091C40726
:1057B000A091C507B091C6078093750290937602B9
:1057C000A0937702B093780283EC97E00E94A5271C
:1057D00004C010E0B0CF1111E7CF2AE037ED43E26B
:1057E0005CE36091490270914A0280914B02909172
:1057F0004C020F94F3326B017C0160917F02709137
:105800008002072E000C880B990B0F9494329B0199
:10581000AC01C701B6010F94F332698B7A8B8B8B85
:105820009C8B8091C80C882309F180900F0990907F
:105830001009A0901109B0901209C090BF07D09034
:10584000C007E090C107F090C20720E030E0A90156
:10585000C501B4010F948D328823D1F1A7019601BF
:10586000C501B4010F94BD3B181694F1C12CD12C85
:1058700076018E010F5E1F4F23EC37E04FEB57E0B0
:105880006BEB77E087EB97E00F94E00780E1E7EBC5
:10589000F7E0A9E6B2E001900D928A95E1F7A696AD
:1058A0000FB6F894DEBF0FBECDBFDF91CF911F9131
:1058B0000F91FF90EF90DF90CF90BF90AF909F90AF
:1058C0008F907F906F905F904F903F902F900895B2
:1058D0002091690230916A0240916B0250916C02F2
:1058E0006091B7077091B8078091B9079091BA0796
:1058F0000F945C396D8B7E8B8F8B988F20916D020E
:1059000030916E0240916F02509170026091BB071E
:105910007091BC078091BD079091BE070F945C39D0
:10592000698F7A8F8B8F9C8F2091710230917202D8
:105930004091730250917402C701B6010F945C3913
:105940006D8F7E8F8F8F98A3209175023091760294
:1059500040917702509178026091C3077091C4071B
:105960008091C5079091C6070F945C396B017C014B
:1059700020E030E0A9016D897E898F89988D0F9490
:105980008D3281110CC020E030E0A901698D7A8D43
:105990008B8D9C8D0F948D32882309F467CF2D89D0
:1059A0003E894F89588DCA01B9010F94F3324B01DA
:1059B0005C01298D3A8D4B8D5C8DCA01B9010F9424
:1059C000F3329B01AC01C501B4010F945D394B0169
:1059D0005C012D8D3E8D4F8D58A1CA01B9010F94E8
:1059E000F3329B01AC01C501B4010F945D394B0149
:1059F0005C01A7019601C701B6010F94F3329B0128
:105A0000AC01C501B4010F945D390F940B3C4B01FF
:105A10005C012DEB37E346E855E30F948D3287FFA9
:105A20000FC020E030E0A901C701B6010F94BD3BD3
:105A30004601570187FF04C0B7FAB094B7F8B09495
:105A40002DEB37E346E855E3C501B4010F948D32E1
:105A500087FD1CCF20E030E040EA51E4C501B401ED
:105A60000F94573A0F94D03A1B01672B19F4222454
:105A70002394312CB10190E080E00F9492329B018D
:105A8000AC0160E070E080E89FE30F94573A2B018F
:105A90003C01AC019B01C501B4010F94F3324B01F1
:105AA0005C01A30192016D897E898F89988D0F9485
:105AB000F3326D8B7E8B8F8B988FA3019201698D52
:105AC0007A8D8B8D9C8D0F94F332698F7A8F8B8FAB
:105AD0009C8FA30192016D8D7E8D8F8D98A10F9467
:105AE000F3326D8F7E8F8F8F98A3A3019201C70130
:105AF000B6010F94F33269A37AA38BA39CA380E130
:105B0000E9E6F2E08E010F5F1F4FD80101900D9280
:105B10008A95E1F70E9429742B013C0128EC420E82
:105B2000511C611C711C0DA31EA381E0281A3108B1
:105B300009F460C00E9429748B019C0104191509A5
:105B40002609370937FD59C02B013C0128EC420ECC
:105B5000511C611C711C80E00E94C3DF2D893E89AD
:105B60004F89588D69817A818B819C810F945D3931
:105B700069837A838B839C83298D3A8D4B8D5C8DD1
:105B80006D817E818F8198850F945D396D837E83D1
:105B90008F8398872D8D3E8D4F8D58A169857A858D
:105BA0008B859C850F945D3969877A878B879C8765
:105BB00029A13AA14BA15CA16D857E858F8598892D
:105BC0000F945D396D877E878F87988B750164018F
:105BD0008E010F5E1F4F9E01235F3F4FAE01475F57
:105BE0005F4FBE016B5F7F4F8DA19EA10F94E007B9
:105BF00081119BCF750164013CCE0E94378FAECFDF
:105C00008091C2049091C304A091C404B091C504D2
:105C10008093490290934A02A0934B02B0934C02A6
:105C20008091C0049091C1049093800280937F0280
:105C300008958091490290914A02A0914B02B0913F
:105C40004C028093C2049093C304A093C404B09305
:105C5000C50480917F02909180029093C10480934B
:105C6000C00484E690E09093800280937F020895C0
:105C70008F929F92AF92BF92CF92DF92EF92FF925C
:105C8000CF93DF938090490290904A02A0904B02FC
:105C9000B0904C02FC01C080D180E280F38020E013
:105CA00030E0A901C701B6010F948D32882341F07D
:105CB000C0924902D0924A02E0924B02F0924C020A
:105CC000C0917F02D091800284E690E090938002A0
:105CD00080937F02C0907902D0907A02E0907B029C
:105CE000F0907C0280E090E0A0E8BFE3809379022E
:105CF00090937A02A0937B02B0937C020E944D2B7A
:105D00008092490290924A02A0924B02B0924C02B9
:105D1000D0938002C0937F02C0927902D0927A021F
:105D2000E0927B02F0927C02DF91CF91FF90EF90A6
:105D3000DF90CF90BF90AF909F908F9008950F937A
:105D40001F93CF93DF9300D01F92CDB7DEB79C0196
:105D500007EB17E090E1E9E6F2E0D80101900D923F
:105D60009A95E1F7F9012081318142815381F8014F
:105D700060857185828593850F945D39F801608710
:105D800071878287938780E090E0A0EAB0E48983FE
:105D90009A83AB83BC83CE0101960E94382E0F906C
:105DA0000F900F900F90DF91CF911F910F91089559
:105DB000AF92BF92CF92DF92EF92FF920F931F9319
:105DC000CF93DF93CDB7DEB764970FB6F894DEBFFD
:105DD0000FBECDBF0E94022187FDAFC08AE50E94A1
:105DE00081BE882309F4BAC040E050E0BA018AE5D8
:105DF0000E94EEBE7B018C012091710230917202F3
:105E0000409173025091740260E070E088EC93E47A
:105E10000F945C395B016C019701A8010F94BD3BA5
:105E2000181614F07501860120E030E0A901B701D1
:105E3000C8010F94BD3B181624F4E12CF12C00E0AE
:105E400010E0B701C8010F94C93A072E000C880B67
:105E5000990B0F949432698B7A8B8B8B9C8B20E0FF
:105E600030E0A9010F948D32882321F0CE014196B4
:105E70000E949F2E80E090E0A0EAB1E48D879E878B
:105E8000AF87B88B19861A861B861C868CE40E9405
:105E900033BE882309F467C00E9409BE6B017C01F0
:105EA00020E030E0A901C701B6010F94BD3B87FF98
:105EB00004C0F7FAF094F7F8F094CD82DE82EF8216
:105EC000F88620917C1230917D122430310574F0D7
:105ED00080917A1290917B12821B930B97FF03C0E3
:105EE00091958195910901E004970CF400E080E020
:105EF0000E94CEEC882359F022E0AE01435F5F4F51
:105F0000BE016B5F7F4FCE0109960E94EBEB698962
:105F10007A898B899C898B019C01305809831A836B
:105F20002B833C8320E030E0A9010F948D3288233D
:105F300021F0CE0101960E949F2E64960FB6F89430
:105F4000DEBF0FBECDBFDF91CF911F910F91FF90AC
:105F5000EF90DF90CF90BF90AF900895E12CF12C9F
:105F600000E211E449CFC090EC04D090ED04E09041
:105F7000EE04F090EF0494CFCF92DF92EF92FF9275
:105F80000F931F93C12CD12C76018C0125E732E0B1
:105F900041E752E06DE672E089E692E00F94E00797
:105FA0001F910F91FF90EF90DF90CF9008954F9247
:105FB0005F926F927F928F929F92AF92BF92CF9299
:105FC000DF92EF92FF920F931F93CF93DF93CDB7A2
:105FD000DEB72C970FB6F894DEBF0FBECDBF2B01F6
:105FE0003C0129873A874B875C8747015801F601B6
:105FF000E080F1800281138120E030E0A901B70147
:10600000C8010F948D32882309F488C05E2D4F2D6E
:10601000302F212F852F942FA32FB22F89839A837E
:10602000AB83BC8320E030E0A901B701C8010F9425
:106030008D32811108C0E0904502F0904602009137
:10604000470210914802C701D8018D839E83AF8318
:10605000B887A501940160917102709172028091DC
:106060007302909174020F948D3287FF0CC080925E
:10607000710290927202A0927302B0927402CE01E9
:1060800001960E94BC2F4092690250926A0260926F
:106090006B0270926C0289859A85AB85BC85809372
:1060A0006D0290936E02A0936F02B0937002CE01C6
:1060B00005960E94BC2FA501940160917102709118
:1060C000720280917302909174020F94BD3B181676
:1060D00064F48092710290927202A0927302B09264
:1060E0007402CE0101960E94BC2F0E94D4232C96EC
:1060F0000FB6F894DEBF0FBECDBFDF91CF911F91D9
:106100000F91FF90EF90DF90CF90BF90AF909F9056
:106110008F907F906F905F904F90089550E040E097
:1061200030E820E477CFCF92DF92EF92FF920F9387
:106130001F936A01E0907102F09072020091730265
:1061400010917402FB012081318142815381FC0155
:1061500060817181828193810E94D72F1F910F915D
:10616000FF90EF90DF90CF900895CF92DF92EF9263
:10617000FF920F931F936B01FC01E080F18002817D
:106180001381E9E6F2E024813581468157816081FF
:106190007181828193810E94D72F1F910F91FF906F
:1061A000EF90DF90CF900895AF92BF92CF92DF92A1
:1061B000EF92FF920F931F93CF93DF9300D01F9224
:1061C000CDB7DEB7FC01E080F1800281138161115F
:1061D00012C0A0907102B0907202C0907302D09071
:1061E00074029501A601B701C8010F948D3287FF93
:1061F00002C07501860120E030E048EC53E4B701AD
:10620000C8010F948D3287FD04C0E12CF12C08ECFD
:1062100013E4C701D80189839A83AB83BC836EEEF4
:1062200072E0CE0101960E94B5300F900F900F9052
:106230000F90DF91CF911F910F91FF90EF90DF9022
:10624000CF90BF90AF900895EF92FF920F931F935E
:10625000CF93DF937C018B010E9498C3C9E6D2E003
:106260002091790230917A0240917B0250917C0218
:10627000F70160817181828193810F94573A2C8557
:106280003D854E855F850F945D396C877D878E8750
:106290009F87C8010E94BC2FDF91CF911F910F9162
:1062A000FF90EF900C94D4238F929F92AF92BF9265
:1062B000CF92DF92EF92FF921F93CF93DF93CDB7F0
:1062C000DEB760970FB6F894DEBF0FBECDBF182FB4
:1062D00080E00E942A294B015C018092B4049092D4
:1062E000B504A092B604B092B70481E00E942A29B6
:1062F0006B017C01C092B804D092B904E092BA0458
:10630000F092BB0482E00E942A296093BC0470933F
:10631000BD048093BE049093BF041D861E861F8615
:10632000188A89829A82AB82BC82CD82DE82EF8219
:10633000F88669877A878B879C8783E00E942A2961
:106340006D877E878F87988B8091C80C882321F07A
:10635000CE0101960E9472231E3FD9F480E1FE0116
:106360003196A9E6B2E001900D928A95E1F7609628
:106370000FB6F894DEBF0FBECDBFDF91CF911F9156
:10638000FF90EF90DF90CF90BF90AF909F908F9055
:10639000089584E0189FF0011124DF01A759BD4F33
:1063A00081E090E08C0F9D1FE80FF91F4081518123
:1063B000628173814D935D936D937C931397D7CFD7
:1063C0000D943F1F0F931F93CF93DF93EC018B012D
:1063D00081E00F94C72269E170E080E090E00E94C4
:1063E000E4C2B801CE010E94B530C0911E0680E023
:1063F0000F94C72210921E0682E00E9454310E9420
:10640000E031C2FBCC27C0F981E08C27DF91CF912E
:106410001F910F910895CF93DF93CDB7DEB72C97DF
:106420000FB6F894DEBF0FBECDBF0F941D200E94A3
:1064300098279CE0E6E3F5E0DE01119601900D92CD
:106440009A95E1F781110E94C7C2CE0101960E9480
:10645000A1972C960FB6F894DEBF0FBECDBFDF918B
:10646000CF9108952F923F924F925F926F927F92B9
:106470008F929F92AF92BF92CF92DF92EF92FF9254
:106480000F931F93CF93DF9300D0CDB7DEB78090EB
:10649000690290906A02A0906B02B0906C024090EA
:1064A0006D0250906E0260906F0270907002C0900A
:1064B0007102D0907202E0907302F09074020E9418
:1064C000BA1C0E942D240DE312E18FE492E09B831D
:1064D0008A8381E3282E82E1382E198289810E94E5
:1064E000081DC8010E9496B8EA81FB8161937193EF
:1064F00081939193FB83EA83C1010E9496B8EA815C
:10650000FB816087718782879387F981FF5FF983B9
:106510000C5F1F4F84E0280E311CF330F9F681E147
:1065200095E00F9482200E946AC20E94B023A501C8
:1065300094016091690270916A0280916B0290915E
:106540006C020F948D3281111CC0A30192016091E5
:106550006D0270916E0280916F02909170020F94A3
:106560008D3281110EC020917102309172024091E2
:10657000730250917402C701B6010F948D328823C3
:10658000B9F00F900F900F90DF91CF911F910F9165
:10659000FF90EF90DF90CF90BF90AF909F908F9043
:1065A0007F906F905F904F903F902F900C940B32A4
:1065B0000F900F900F90DF91CF911F910F91FF904F
:1065C000EF90DF90CF90BF90AF909F908F907F9093
:1065D0006F905F904F903F902F9008958091B304FB
:1065E000659B6EC080618093B3049091030180919C
:1065F000B30491FF67C080628093B3048091B304B9
:106600004B9B62C084608093B3048091B3049091EB
:10661000B204981709F45AC092E09093B1048093A1
:10662000B2048091DB05811105C08091C7078823E2
:1066300009F459C08091280580FF10C08091DC05C5
:1066400080FD0CC08091B00484FF08C080911E06BC
:10665000806180931E0680E00E94C197809128058A
:10666000869580FF11C08091DC05869580FD0CC069
:106670008091B00485FF08C080911E0680628093DF
:106680001E0681E00E94C197809128058695869517
:1066900080FF29C08091DC058695869580FF23C008
:1066A0008091C7078823F9F08091B00482FF1BC056
:1066B00080911E06846080931E0682E00C94C19730
:1066C0008F7E91CF8F7D98CF8B7F9DCF8091B104AE
:1066D000882309F4A6CF81508093B1048111A1CF02
:1066E0009093B0049ECF08958091DB05811104C082
:1066F0008091C707882331F062E070E080E090E08D
:106700000C94E4C208953F924F925F926F927F92F1
:106710008F929F92AF92BF92CF92DF92EF92FF92B1
:106720000F931F93CF93DF9300D01F92CDB7DEB7A7
:10673000382E80E090E0A0E2B1E489839A83AB83B5
:10674000BC83C0900F13D0901013E0901113F09001
:10675000121320E030E0A901C701B6010F948D3279
:1067600087FF0CC0A701960160E070E080E291E431
:106770000F945C3969837A838B839C8360E0CE01BC
:1067800001960E94D4304090690250906A02609055
:106790006B0270906C0280906D0290906E02A090DF
:1067A0006F02B0907002332089F10E9439DE1982A5
:1067B0001A821B821C82E0907102F090720200919A
:1067C000730210917402CE0101966C01A50194012F
:1067D000C301B2010E94D72F3092C7070E947433C1
:1067E0000F900F900F900F90DF91CF911F910F910D
:1067F000FF90EF90DF90CF90BF90AF909F908F90E1
:106800007F906F905F904F903F9008950E94F6DDCB
:10681000CECF2F923F924F925F926F927F928F9244
:106820009F92AF92BF92CF92DF92EF92FF920F931F
:106830001F93CF93DF93CDB7DEB766970FB6F8946B
:10684000DEBF0FBECDBFF82E282E312CF101E65A47
:10685000F04FD49022E0821335C08091C707811198
:1068600003C081E00E9483330E9439DE811139C167
:1068700086E59FE00E9496B820E030E0A9010F94E1
:106880008D328823F9F06D2DDD0C770B880B990B79
:106890000F9494322B013C0186E59FE00E9496B84C
:1068A0004B015C0120E030E040EA50E40F948D326F
:1068B00011E087FF1CC0812C912C90EAA92E90E456
:1068C000B92E15C06D2DDD0C770B880B990B0F942D
:1068D00094322B013C01C101880F991F880F991F29
:1068E000825B904F0E9496B84B015C0110E0A301BF
:1068F0009201C501B4010F94F3324B015C016101B7
:10690000CC0CDD1CCC0CDD1CC6018E5B904F0E94B4
:1069100096B8EE24E394E12620E030E040EC5FE31B
:106920000F94F332A30192010F94F332AB01BC0137
:1069300000E010E098018F2D0E94542920E030E003
:10694000A901C501B4010F948D32F601EA5CF04F44
:10695000FA8BE98B882309F44DC0F2E000E010E0E7
:1069600020E431E4FF1619F000E010E09801B501D1
:10697000A4017058E12C8F2D0E945429A501940187
:10698000C501B4010F945D396B8B7C8B8D8B9E8B15
:1069900022E0F216E9F0F101ED5CF04F6491611133
:1069A00007C00E9418DC81E19FE00E94B4C76AE042
:1069B00070E090E080E00F9492329B01AC0160E0C7
:1069C00070E088E492E40F94573A8B019C0104C074
:1069D00000E010E020EC30E4EE24E3944B895C8985
:1069E0006D897E898F2D0E94542932E0F312D0C028
:1069F0000E94F6DD81E090E0A0E0B0E00F2C04C042
:106A0000880F991FAA1FBB1F0A94D2F72091C70CA9
:106A1000282B2093C70C20919A04822B80939A04F0
:106A200089899A890E9496B8F601E759FD4F6083DB
:106A300071838283938382E0F8121AC020910F132E
:106A40003091101340911113509112136091710203
:106A50007091720280917302909174020F945C396C
:106A60006093710270937202809373029093740228
:106A7000F601E35CF74F10821182128213828F2D90
:106A80000E94081D0E94E031F601E759FD4F808108
:106A90009181A281B381F601E954F84F80839183FB
:106AA000A283B38392E0F916A9F18CE0EFE9F2E05A
:106AB000DE01119601900D928A95E1F7E1E0F0E098
:106AC000EC0FFD1FEC0DFD1D80809180A280B38036
:106AD00020E030E0A901C501B4010F948D3281118D
:106AE0001EC066960FB6F894DEBF0FBECDBFDF9115
:106AF000CF911F910F91FF90EF90DF90CF90BF90BB
:106B0000AF909F908F907F906F905F904F903F904D
:106B10002F9008950E949CB88111E3CFC6CF20E04A
:106B200030E0A901C501B4010F94BD3B87FF04C04B
:106B3000B7FAB094B7F8B094F601E759FD4F6F017A
:106B4000A3019201C501B4010F94F3329B01AC0182
:106B5000F60160817181828193810F945C39F60125
:106B60006083718382839383F2E080E090E0A0E40D
:106B7000B1E4FF1621F080E090E0A8E4B2E48D8754
:106B80009E87AF87B88BCE010D960E94BC2FA9CFF0
:106B900081E090E0A0E0B0E00F2C04C0880F991FC6
:106BA000AA1FBB1F0A94D2F72091C70C282B209351
:106BB000C70C20919A04822B80939A0489899A8920
:106BC0000E9496B8F601E759FD4F60837183828376
:106BD00093834ECF0F931F938091B311813019F59A
:106BE0000E9429740091CE041091CF042091D0040A
:106BF0003091D104601B710B820B930B28EE33E0B4
:106C000040E050E00F94D1386091D2047091D304E9
:106C10008091D4049091D504620F731F841F951F37
:106C20001F910F9108956091D6047091D7048091BF
:106C3000D8049091D904D6CF1092B3111092CE04FB
:106C40001092CF041092D0041092D1041092D60466
:106C50001092D7041092D8041092D9041092D20442
:106C60001092D3041092D4041092D50408958F92F8
:106C70009F92AF92BF92CF92DF92EF92FF920F93CB
:106C80001F93CF93DF93CDB7DEB72C970FB6F89451
:106C9000DEBF0FBECDBF8B0140E050E068E472E480
:106CA0004D835E836F83788740E050E060EA70E454
:106CB00049875A876B877C878130B9F1823009F424
:106CC00059C020E030E040E050E4609171027091E2
:106CD000720280917302909174020F945D394B019E
:106CE0007C0120E030E048EC53E40F94BD3B1816E3
:106CF00034F4812C912C88ECE82E93E4F92EF801E1
:106D0000A084B184C284D3849401A701B501C601D3
:106D10000F94BD3B181614F054016701C501D6014C
:106D200089839A83AB83BC8348C0BE01675F7F4F72
:106D3000C80108960E94B530B8016C5F7F4FAE0164
:106D40004B5F5F4FC8010E9493300E940B322C961C
:106D50000FB6F894DEBF0FBECDBFDF91CF911F916C
:106D60000F91FF90EF90DF90CF90BF90AF909F90EA
:106D70008F900895F8012085318542855385609173
:106D800071027091720280917302909174020F945B
:106D90005D396B017C0120E030E048EC53E40F9456
:106DA0008D3287FD06C0C12CD12C28ECE22E23E4C5
:106DB000F22EC982DA82EB82FC82BE01675F7F4FCE
:106DC000CE010196B7CFCF92DF92EF92FF92CF9391
:106DD000DF93C62FFC01C080D180E280F38020E0E9
:106DE00030E0A901C701B6010F948D3220E030E0F8
:106DF000A90187FD14C020E030E048EC52E4C7014F
:106E0000B6010F94BD3B24E630E040E050E0181698
:106E100034F0C701B6010F94C93A9B01AC01C230EE
:106E2000A0F4D0E0C85BD64FAFEFB0E00F941239BA
:106E300024E630E040E050E00F94F3382F3F310576
:106E400019F010F02FEF30E02883DF91CF91FF9001
:106E5000EF90DF90CF900895E8E4F5E01082118282
:106E60001282138214820C9411F1EF92FF920F930D
:106E70001F93CF93DF93CDB7DEB78C01EDB6FEB68F
:106E80000F94DA3101962DB73EB7281B390B0FB698
:106E9000F8943EBF0FBE2DBF8DB79EB70196B801C7
:106EA0000F94D3310F947A230FB6F894FEBE0FBE21
:106EB000EDBEDF91CF911F910F91FF90EF9008955C
:106EC0008091090180FD06C08091D01483FB882742
:106ED00080F9089580E00895CF92DF92EF92FF92BB
:106EE000FC01C080D180E280F380663019F51092F9
:106EF0004D0510924E0510924F05109250051092BC
:106F000051050E94BD8B20E030E0A901C701B60108
:106F10000F948D3287FF1DC0C12CD12C7601C70183
:106F2000B6010F94CA3BCB01FF90EF90DF90CF905A
:106F30000C9485BD0E942C3720E030E0A901C701E8
:106F4000B6010F948D3287FF15C0C12CD12C76016C
:106F500021C020E030E04CE053E4C701B6010F94BB
:106F6000BD3B1816E4F6C12CD12C9CE0E92E93E42D
:106F7000F92ED5CF20E030E046E953E4C701B60151
:106F80000F94BD3B181634F4C12CD12C86E9E82EA1
:106F900083E4F82EC701B6010F94CA3BCB01FF90E2
:106FA000EF90DF90CF900C94A4239091C70C977032
:106FB00081E0973009F080E008952091990420FF46
:106FC00014C020E83EE3629FA001639F500D729FB2
:106FD000500D1124CA01969587959695879500972F
:106FE00031F08A950000E9F708950C94E4C2089501
:106FF000CF93DF931092860C1092190D10921B0DF7
:1070000010921A0D1092AE041092AD04CFEFDFEF84
:107010008091D01485FD07C00E94D677D0934F137E
:10702000C0934E13F5CF8FEF9FEF90934F13809344
:107030004E13DF91CF9108958F929F92AF92BF929E
:10704000CF92DF92EF92FF920F931F93CF93DF9334
:107050007C0121E5E20EF11CD7014C914A3509F083
:10706000A4C06C01B2E5CB0ED11CF6013081353ADB
:1070700009F09BC0EC01C05BDF4F2881233008F48E
:1070800094C08C0100561F4FD8014C93E15BFF4F19
:10709000308331962083EF54F1093081E05BFF4F5C
:1070A00030833038B1F43196AC54B1093C9130831F
:1070B000E854F109AF5ABF4F50E040E02250330B83
:1070C00042175307CCF4808132968D934F5F5F4F08
:1070D000F7CF233031F5313809F074C0FC01EC559D
:1070E000FF4FDC01AC5ABF4F2C9120833196885A58
:1070F0009F4FDC018C9180834801B12CA12C8881A9
:1071000090E002968A159B050CF43FC0F401819132
:107110004F010E941DC60E943EF1FFEFAF1ABF0A49
:10712000EECF323821F5FC01EC5AFF4F308141811E
:10713000E05BFF4F408331963083DC01AA55BF4F9F
:1071400050E040E02350330B42175307ACF6FA01EE
:10715000EE7FE45AFF4FE80FF91F608171817C9345
:1071600011966C9311974E5F5F4F1296EDCF2430BE
:1071700019F6333809F6FC01EC5AFF4F20813181B2
:10718000E05BFF4F30833196B0CF80E5DE011D928A
:107190008A95E9F78AE1F80111928A95E9F78AE57B
:1071A000D7018C9385EAF6018083DF91CF911F91FF
:1071B0000F91FF90EF90DF90CF90BF90AF909F9096
:1071C0008F900895323809F097CFADCFCF93DF93EA
:1071D000D091B31189E192E10E94B4C78AE00E9484
:1071E0008CC78091320D873009F449C083E08093C9
:1071F000300D81E08093860280E190E090936714E7
:107200008093661485E080935A14C2E8C0935D149D
:1072100084E190E1A0E0B0E080935E1490935F146D
:10722000A0936014B09361148AE094E10E941C382A
:1072300061E070E080E090E00E94DD3781E09AE557
:10724000909367148093661485E390E0909369149B
:107250008093681487E080935A14C0935D1484E887
:1072600090E0A0E0B0E080935E1490935F14A09350
:107270006014B09361148AE094E10E941C388091FC
:10728000B311813089F1823061F50E94EA35609353
:10729000D2047093D3048093D4049093D50481E0F6
:1072A0008093B3110E9429746093CE047093CF042D
:1072B0008093D0049093D104D23089F08091CA0594
:1072C0009091CB0501969093CB058093CA051092BF
:1072D0009B0410929C0410929D0410929E0481E0E5
:1072E00004C00E941C36DBCF80E0DF91CF9108956F
:1072F0000E944FF51092C60C10922D020E94E3C31B
:10730000882351F08091D01482FD06C084E49EE071
:107310009093160D8093150D61E08DE39EE00E9421
:10732000C3C80C94E6388091B3118130C1F589E56A
:107330009EE00E94B4C78AE00E948CC781E09AE573
:10734000909367148093661487E590E09093691496
:107350008093681487E080935A1482E880935D14C8
:1073600084E890E0A0E0B0E080935E1490935F1416
:10737000A0936014B09361148AE094E10E941C38D9
:1073800082E08093B3110E9429746093D6047093B5
:10739000D7048093D8049093D90481E0089580E0C5
:1073A00008950F931F930E9429740091C5051091B1
:1073B000C6052091C7053091C805011511052105A5
:1073C000310509F067C020913C13222309F45FC006
:1073D000E0913A13215020933C1321E02E0F20938B
:1073E0003A1330913D13231302C010923A1324E054
:1073F000E29FF0011124E25CFC4E008111812281A8
:1074000033810093C1051093C2052093C3053093C7
:10741000C405600F711F811D911D6093C505709398
:10742000C6058093C7059093C8058091C3059091C8
:10743000C405892B61F11FB7F89488E49EE00E948F
:10744000B4C78AE00E948CC784E096E090936714EA
:107450008093661480EA90E890936914809368148E
:1074600087E080935A1482E880935D1480EA90E06C
:10747000A0E0B0E080935E1490935F14A09360143A
:10748000B09361148AE094E10E941C381FBF1F91E1
:107490000F910895601B710B820B930B97FDF7CF33
:1074A00040981092C5051092C6051092C70510921B
:1074B000C805EDCF0F931F93CF93DF938C01EB01A2
:1074C00090913C1320913D13921305C00E94D13935
:1074D0000E94378FF5CF80913B1334E0839FF001FA
:1074E0001124E25CFC4E11830083D383C2839F5F2F
:1074F00090933C138F5F281739F080933B13DF91F3
:10750000CF911F910F91089510923B13F8CF2F92B6
:107510003F924F925F926F927F928F929F92AF9223
:10752000BF92CF92DF92EF92FF920F931F93CF9370
:10753000DF93009709F0AAC110921B0D10921A0D4B
:107540009093AE048093AD04BAE0CB2EB0E2DB2E74
:10755000E12CF12C15E002E846015701C4E1D0E02E
:107560001092AD131092AC131093A0130093A313B9
:107570008092A4139092A513A092A613B092A71381
:1075800080E593E10E941C3821972FEF821A920A1E
:10759000A20AB20A209721F744E1C40ED11CE11CD3
:1075A000F11C8AE5C81680E2D806E104F104A1F6D0
:1075B000C12CA0E2DA2EE12CF12CD5E0C2E8109229
:1075C000AD131092AC13D093A013C093A313C09229
:1075D000A413D092A513E092A613F092A71380E50E
:1075E00093E10E941C381092AD131092AC13D0930B
:1075F000A013C093A313D701C6018C529F4FAF4F66
:10760000BF4F8093A4139093A513A093A613B09398
:10761000A71380E593E10E941C38EFEFCE1ADE0A33
:10762000EE0AFE0AFAE0CF16F0E2DF06E104F1040A
:1076300031F6FEEDCF2EF0E2DF2EE12CF12CD5E07D
:10764000C2E81092AD131092AC13D093A013C09364
:10765000A313C092A413D092A513E092A613F092A4
:10766000A71380E593E10E941C382FEFC21AD20ABB
:10767000E20AF20A46EEC41640E2D406E104F1043E
:1076800001F7CC24C394E2E1DE2EE12CF12C0AE0D8
:1076900010E0D5E0C2E81093AD130093AC13D09383
:1076A000A013C093A313C092A413D092A513E09289
:1076B000A613F092A71380E593E10E941C38109363
:1076C000AD130093AC13D093A013C093A313D701B1
:1076D000C6018096A11DB11D8093A4139093A5139C
:1076E000A093A613B093A71380E593E10E941C38E2
:1076F0008FEFC81AD80AE80AF80AE5E0CE16E2E1E8
:10770000DE06E104F10439F600911A0D10911B0D0B
:107710000115110509F0D6C08091190D882309F4CF
:10772000E1C02AE030E240E050E069EB73E080E540
:1077300093E10E9443F1C1E0D0E003E010E0E0906B
:107740001A0DF0901B0D35E0332E42E8242E442410
:107750004A94542C64E0662E712C7FE1C72E74E0AD
:10776000D72E80911A0D90911B0D800F911FE81656
:10777000F90608F0D5C0C7010E945AF2882309F41F
:1077800081C080912E1261E272E1882311F06EE2D5
:1077900072E1FB0101900020E9F7CF010197861B00
:1077A000970BF4E1FC9F9001FD9F300D1124265FA3
:1077B0003F4D50E040E0459710F0FB01128A80E514
:1077C00093E10E9443F1CE018F5F9D4EB0E0A0E0B7
:1077D00021964E0124E0880C991C2A95E1F7FDEFD3
:1077E0008F1AFFE99F0AB12CA12C2091D01424FFFD
:1077F0007EC07092AD136092AC133092A0132092B1
:10780000A3138093A4139093A513A093A613B093EE
:10781000A71380E593E10E941C38D092AD13C0926B
:10782000AC133092A0132092A3138092A4139092D1
:10783000A513A092A613B092A71380E593E10E942E
:107840001C38B70185E09EE00E94D3C980912E12BA
:107850006EE272E1811102C061E272E182E09EE0BB
:107860000E940ADC66E87CE08EEF9DE00E940ADC64
:1078700061E272E18DEF9DE00E940ADC89EF9DE0FC
:107880000E94B4C72FEFE21AF20A6BCF20911A0DB3
:1078900030911B0DA901415051096091AD047091C7
:1078A000AE046817790738F42C5F3F4F30931B0DF7
:1078B00020931A0D45CE4430510508F43DCE245096
:1078C0003109F4CF0430110569F48091190D882332
:1078D00031F083E090E090931B0D80931A0DD0E07F
:1078E000C0E02DCFD0E0C0E004E010E028CF10923F
:1078F000AD131092AC133092A0132092A313809377
:10790000A4139093A513A093A613B093A71380E597
:1079100093E10E941C385092AD134092AC1381CF7A
:10792000DF91CF911F910F91FF90EF90DF90CF905B
:10793000BF90AF909F908F907F906F905F904F908F
:107940003F902F900895AF92BF92CF92DF92EF9227
:10795000FF920F931F93CF93DF93EC0184E6C82E21
:1079600080E2D82EE12CF12C02E8A12C90E2B92E75
:1079700015E000935D14C0925E14D0925F14E09203
:107980006014F0926114B0926714A0926614109380
:107990005A148AE094E10E941C388FEFC81AD80A62
:1079A000E80AF80A88E7C81680E2D806E104F1047C
:1079B00001F724E630E240E050E0BE018AE094E1C5
:1079C000DF91CF911F910F91FF90EF90DF90CF90BB
:1079D000BF90AF900C9443F10F931F93CF93DF931D
:1079E0008C016F3F19F41092F41160E02091F411B2
:1079F000862F062E000C990B2817190609F08CF516
:107A00006093F41160E087E09EE00E94C3C8C80163
:107A10000E94B4C78AE00E948CC7C8010F94DA3173
:107A2000800F911FEC01C01BD10BC034D1053CF07D
:107A30000197FC012491207C2038D1F3F3CFDD277E
:107A4000AE01B80184EB91E10F94FB31CC54DE4ED2
:107A5000188284EB91E1DF91CF911F910F910C94EB
:107A6000A33CDF91CF911F910F910895DF92EF9288
:107A7000FF920F931F93CF93DF93CDB7DEB7CA5A10
:107A8000D1090FB6F894DEBF0FBECDBFCF55DF4F83
:107A9000188219821A821B82C15AD0408091C60373
:107AA0009091C703A091C803B091C903CB55DF4F94
:107AB00088839983AA83BB83C55AD04084E690E02B
:107AC0009093E7048093E604109217051092160530
:107AD0001092180526E135E044E050E0BE016B55F8
:107AE0007F4F86EE94E00E9482DE8091E6049091C2
:107AF000E70402969093E7048093E604109217053A
:107B00001092160581E0C655DF4F8883CA5AD040CF
:107B1000CE0186559F4F0E9422A526E135E048E41C
:107B200050E06DEC7CE086EE94E00E9482DE26E17F
:107B300035E040E150E064E379E086EE94E00E94B5
:107B400082DE8AE097EDA3EABCE3CF55DF4F88835E
:107B50009983AA83BB83C15AD040CE018F559F4FD2
:107B60000E9419A589E498E00E9434A58FE092E074
:107B70000E942BA58BE092E00E9419A580910F092D
:107B800090911009A0911109B091120989839A83EB
:107B9000AB83BC838E010F5F1F4FC8010E9419A5E4
:107BA000CF55DF4F188219821A821B82C15AD040EA
:107BB0007E018DE6E80EF11C83E0D7018C9389836A
:107BC000CE018F559F4F0E9419A5C7010E9422A583
:107BD000C8010E9422A54AE0D42EDA94DD2031F0BB
:107BE000CE018F559F4F0E9419A5F7CF87E093E1F3
:107BF0000E9434A5CF55DF4F188219821A821B824A
:107C0000C15AD0403AE0D32EDA94DD2031F0CE01D3
:107C10008F559F4F0E9419A5F7CF85E0D82ED982A6
:107C2000F701D082C8010E9422A5C7010E9422A5A7
:107C300026E135E048E050E069E075E086EE94E04A
:107C40000E9482DE26E135E048E050E061E075E028
:107C500086EE94E00E9482DE26E135E044E650E0C4
:107C600063ED77E086EE94E00E9482DE19828FEF6A
:107C7000D7018C93C8010E942BA5C7010E9422A5A1
:107C800026E135E044E050E062EF72E086EE94E0F9
:107C90000E9482DE8091DD058983C8010E942BA5A8
:107CA00026E135E040E150E061EF74E086EE94E0DB
:107CB0000E9482DE198A1A8A1B8A1C8A80E090E060
:107CC000A0E8BFE38D879E87AF87B88B80917F1236
:107CD00090918012A0918112B091821289839A832F
:107CE000AB83BC832CEA35EC47E25EE36091831200
:107CF0007091841280918512909186120F94573A58
:107D00006D837E838F8398872CEA35EC47E25EE3B0
:107D100060918712709188128091891290918A12D5
:107D20000F94F33269877A878B879C8726E135E049
:107D300044E150E0B80186EE94E00E9482DE84E1E6
:107D400090E09A838983C8010E9407A5809114124C
:107D500090911512A0911612B091171289839A83EF
:107D6000AB83BC832CEA35EC47E25EE360911812EA
:107D70007091191280911A1290911B120F94573A18
:107D80006D837E838F8398872CEA35EC47E25EE330
:107D900060911C1270911D1280911E1290911F1201
:107DA0000F94F33269877A878B879C87C8010E947A
:107DB00010A58CE0EBEAF2E0D80101900D928A95D3
:107DC000E1F7C8010E9410A51982C8010E9422A5EE
:107DD0008FE790E09A838983C8010E9407A5E7EBAB
:107DE000F2E0D80101900D92DA94E1F726E135E056
:107DF00045E050E0B80186EE94E00E9482DE80917A
:107E0000F0048983C8010E942BA580E2ECEBF2E02C
:107E1000D80101900D928A95E1F726E135E040E224
:107E200050E0B80186EE94E00E9482DEF7011082F5
:107E3000C7010E942BA58CE398E00E942BA588E344
:107E400098E00E9419A5CF55DF4F188219821A8237
:107E50001B82C15AD040CE018F559F4F0E9419A559
:107E600080E2D8011D928A95E9F726E135E040E2EB
:107E700050E0B80186EE94E00E9482DEFE01F996A1
:107E800088E0DF011D928A95E9F744E650E060E062
:107E900070E049835A836B837C834D835E836F8359
:107EA000788783E090E0A0E0B0E089879A87AB878D
:107EB000BC874D875E876F87788B498B5A8B6B8B1E
:107EC0007C8B8D8B9E8BAF8BB88F898F9A8FAB8F6E
:107ED000BC8F8D8F9E8FAF8FB8A38EE190E0A0E016
:107EE000B0E089A39AA3ABA3BCA38DA39EA3AFA329
:107EF000B8A789A79AA7ABA7BCA78DA79EA7AFA72E
:107F0000B8AB89AB9AABABABBCAB8DAB9EABAFABFD
:107F1000B8AF26E135E040E450E0B80186EE94E0E9
:107F20000E9482DE90E1D92EF8018D2D11928A9562
:107F3000E9F726E135E040E150E0B80186EE94E053
:107F40000E9482DED8011D92DA94E9F726E135E03D
:107F500040E150E0B80186EE94E00E9482DE84E4C5
:107F600099E00E9419A52CE0D22EF8018D2D1192D6
:107F70008A95E9F726E135E04CE050E0B80186EE5D
:107F800094E00E9482DE8CE6D8011D928A95E9F782
:107F900026E135E04CE650E0B80186EE94E00E9420
:107FA00082DE8AED94E00E9410A526E135E048E0EB
:107FB00050E068EE74E086EE94E00E9482DEF70105
:107FC0001192DA94E9F7C755DF4F1882C95AD040A9
:107FD00080E090E0A0E4B0E4C356DF4F888399834B
:107FE000AA83BB83CD59D040C7010E9434A5CE01DE
:107FF00087559F4F0E9422A5CE0183569F4F0E9416
:1080000019A580E3D7011D928A95E9F789E492E1E9
:108010000E94B4C78AE00E948CC726E135E040E3A5
:1080200050E0B70186EE94E00E9482DE8091180550
:10803000811128C00091E6041091E7048091160593
:1080400090911705F7019183808384E690E09093E7
:10805000E7048093E60426E135E044E050E062E086
:1080600073E086EE94E00E9482DEC7010E9407A5BD
:1080700091E00537134009F490E080911805892BB1
:108080008093180580911805811105C060E08DE787
:1080900092E10E94EC3C8DE592E10E94B4C78AE037
:1080A0000E948CC79091180581E08927C655DF4F43
:1080B0000FB6F894DEBF0FBECDBFDF91CF911F91F9
:1080C0000F91FF90EF90DF9008951092C60C1092E0
:1080D0002D028091D01480648093D01461E085E1FA
:1080E0009EE00E94C3C84AE25EE062E37EE085E073
:1080F0000E945DF360E08CE19EE00C94EC3CCF923A
:10810000DF92EF92FF920F931F93CF93DF93CDB740
:10811000DEB77C01CDB6DEB60F94DA3101962DB70D
:108120003EB7281B390B0FB6F8943EBF0FBE2DBFCC
:108130000DB71EB70F5F1F4FB701C8010F94D331A2
:10814000F80101900020E9F73197E01BF10B7597DA
:1081500020F08CED92E0F801848BC8010E94A33CD2
:108160000FB6F894DEBE0FBECDBEDF91CF911F914A
:108170000F91FF90EF90DF90CF900895CF93DF9312
:1081800000D01F92CDB7DEB78EEC9DE00E94B4C741
:108190008AE00E948CC78091320D8330D9F1198218
:1081A0001A821B821C8260E0CE0101960E94E33697
:1081B00019821A821B821C8261E0CE0101960E9404
:1081C000E33681E08093850210922F0D8093860222
:1081D00081E09AE5909367148093661483E390E0BE
:1081E000909369148093681487E080935A1482E80E
:1081F00080935D1484E890E0A0E0B0E080935E148A
:1082000090935F14A0936014B09361148AE094E19A
:108210000E941C380F900F900F900F90DF91CF911C
:108220000895CF92DF92EF92FF92CF93C82F809163
:10823000B3118150823008F069C00E94BE40109294
:10824000B3110E9429746093D6047093D70480936D
:10825000D8049093D904C0909B04D0909C04E090E3
:108260009D04F0909E040E94EA35AB01BC0140934E
:108270009B0450939C0460939D0470939E04809192
:10828000CE059091CF05A091D005B091D1058C1964
:108290009D09AE09BF09840F951FA61FB71F8093C4
:1082A000CE059093CF05A093D005B093D105C11111
:1082B0000AC0C1E00E941A238C2FCF91FF90EF904B
:1082C000DF90CF9008958091CC059091CD050196D7
:1082D0009093CD058093CC050E94EA35C090D205DD
:1082E000D090D305E090D405F090D505C616D706FA
:1082F000E806F906F0F60E94EA356093D20570931D
:10830000D3058093D4059093D505D3CFC0E0D2CFC9
:108310008F929F92AF92BF92CF92DF92EF92FF9295
:108320000F931F93CF93DF930E94F8373AE0C32E49
:1083300030E2D32EE12CF12C15E002E84601570182
:10834000CAE0D0E0109267141092661410935A1489
:1083500000935D1480925E1490925F14A09260145A
:10836000B09261148AE094E10E941C3821978FEF4B
:10837000881A980AA80AB80A209721F78AE0C80E36
:10838000D11CE11CF11C82EDC81680E2D806E10484
:10839000F104A1F6C12C20E2D22EE12CF12CD5E083
:1083A000C2E81092671410926614D0935A14C093C6
:1083B0005D14C0925E14D0925F14E0926014F0924B
:1083C00061148AE094E10E941C38109267141092A4
:1083D0006614D0935A14C0935D14D701C6018C5211
:1083E0009F4FAF4FBF4F80935E1490935F14A09345
:1083F0006014B09361148AE094E10E941C388FEFFE
:10840000C81AD80AE80AF80A8AE0C81680E2D8062C
:10841000E104F10431F69EEDC92E90E2D92EE12C53
:10842000F12CD5E0C2E81092671410926614D09334
:108430005A14C0935D14C0925E14D0925F14E092FF
:108440006014F09261148AE094E10E941C388FEF6E
:10845000C81AD80AE80AF80A86EEC81680E2D806D2
:10846000E104F10401F7CC24C39482E1D82EE12C7D
:10847000F12C0AE010E0D5E0C2E8109367140093F5
:108480006614D0935A14C0935D14C0925E14D092B7
:108490005F14E0926014F09261148AE094E10E940B
:1084A0001C381093671400936614D0935A14C09329
:1084B0005D14D701C6018096A11DB11D80935E1485
:1084C00090935F14A0936014B09361148AE094E1D8
:1084D0000E941C388FEFC81AD80AE80AF80A85E10A
:1084E000C81682E1D806E104F10439F682E190E091
:1084F0009093671480936614D0935A14C0935D14BC
:1085000084E190E1A0E0B0E080935E1490935F146A
:10851000A0936014B09361148AE094E1DF91CF914D
:108520001F910F91FF90EF90DF90CF90BF90AF9091
:108530009F908F900C941C384F925F926F927F9215
:108540008F929F92AF92BF92CF92DF92EF92FF9263
:108550000F931F93CF93DF9300D000D01F921F92F1
:10856000CDB7DEB78091AB0481110AC48091A90414
:108570009091AA049C012F5F3F4F3093AA0420934F
:10858000A9048E3E924008F4FBC380917A12909128
:108590007B12909367148093661405E000935A143D
:1085A00012E810935D1486E390E1A0E0B0E08093C0
:1085B0005E1490935F14A0936014B09361148AE0EA
:1085C00094E10E941C3880910F12909110129093A8
:1085D00067148093661400935A1410935D148CE30F
:1085E00090E1A0E0B0E080935E1490935F14A093BC
:1085F0006014B09361148AE094E10E941C38809169
:108600007C1290917D12909367148093661400936E
:108610005A1410935D1484E390E1A0E0B0E08093DD
:108620005E1490935F14A0936014B09361148AE079
:1086300094E10E941C388091111290911212909333
:1086400067148093661400935A1410935D148AE3A0
:1086500090E1A0E0B0E080935E1490935F14A0934B
:108660006014B09361148AE094E10E941C3881E0A8
:108670008093AB041092AA041092A9048091320D49
:10868000882339F10E94281D811123C08091A804FC
:108690008F5F8093A8048091A804853620F0109203
:1086A000A8041092320DE091320DE150E73008F04D
:1086B0006AC00E2E000CFF0B8827EE59FC4B8F4F23
:1086C0000D9454396C43BB438745B345F4452C4660
:1086D000BF431092A804DFCF0E94D537882309F446
:1086E00052C081E08093860280EC9DE00E94B4C776
:1086F0008AE00E948CC780E190E090936714809399
:10870000661485E080935A1412E810935D1484E196
:1087100090E1A0E0B0E080935E1490935F14A0938A
:108720006014B09361148AE094E10E941C3881E0E7
:108730009AE5909367148093661486E390E0909393
:1087400069148093681487E080935A1410935D1421
:1087500084E890E0A0E0B0E080935E1490935F1412
:10876000A0936014B09361148AE094E10E941C38D5
:108770001092320D08C00E94D537882321F00E9444
:10878000281D8823A9F380918602882309F433C722
:108790008091AC048111C0C284E096E0909367148C
:1087A0008093661480EA90E890936914809368142B
:1087B00017E010935A1402E800935D1480EA90E0E9
:1087C000A0E0B0E080935E1490935F14A0936014D7
:1087D000B09361148AE094E10E941C388091810278
:1087E00090918202A0918302B09184020097A1052A
:1087F000B10509F03FC2109267141092661415E09B
:1088000010935A1400935D148AE890E1A0E0B0E060
:1088100080935E1490935F14A0936014B0936114DE
:108820008AE094E10E941C3889E090E090936714FC
:108830008093661410935A1400935D148CE890E1B1
:10884000A0E0B0E080935E1490935F14A093601456
:10885000B09361148AE094E10E941C3880918102F7
:1088600090918202A0918302B09184020097F1E07E
:10887000AF07B10508F441C2B0936714A093661422
:10888000909369148093681487E080935A1482E867
:1088900080935D1488E890E1A0E0B0E080935E14DE
:1088A00090935F14A0936014B09361148AE094E1F4
:1088B0000E941C388091810290918202A0918302D3
:1088C000B0918402BA2FA92F982F8827009721E012
:1088D000A207B10508F417C2B0936714A0936614F9
:1088E000909369148093681487E080935A1412E877
:1088F00010935D1481EA90E0A0E0B0E080935E14F4
:1089000090935F14A0936014B09361148AE094E193
:108910000E941C388091C80C882309F4FAC183E0B6
:1089200090E0909367148093661485E080935A14C6
:1089300010935D1485E490E1A0E0B0E080935E14B4
:1089400090935F14A0936014B09361148AE094E153
:108950000E941C388091AC04875E8093AC04209107
:10896000AC04822F90E0253608F021C29093671462
:108970008093661485E080935A1482E880935D1496
:1089800080E090E1A0E0B0E080935E1490935F14EB
:10899000A0936014B09361148AE094E10E941C38A3
:1089A0000E94281D811114C20E94E3C3811105C0D9
:1089B0009091990491FD0E94281D9091990480FB4B
:1089C00091F99093990491FD03C28091D01482FD96
:1089D000FFC18091B3118150823008F4F9C16091D8
:1089E000111270911212072E000C880B990B0F9424
:1089F00094326B017C0120E030E0A9010F948D32AC
:108A0000882309F4BBC660910F1270911012072ED3
:108A1000000C880B990B0F9494322B013C0120E041
:108A200030E040E050E4C701B6010F945C39A30187
:108A300092010F94BD3B18160CF4C2C660917A12D5
:108A400070917B12072E000C880B990B0F949432B7
:108A50006D837E838F83988760917C1270917D12E5
:108A6000072E000C880B990B0F9494324B015C017C
:108A700020E030E040E251E40F945C392D813E81EA
:108A80004F8158850F94BD3B18160CF499C620E011
:108A900030E040E050E4C701B6010F945D39A30116
:108AA00092010F948D3287FD10C020E030E040E24B
:108AB00051E4C501B4010F945D392D813E814F8190
:108AC00058850F948D3287FF6AC684E190E09093B9
:108AD00067148093661485E080935A1482E880932B
:108AE0005D1484E190E1A0E0B0E080935E14909387
:108AF0005F14A0936014B09361148AE094E10E9423
:108B00001C388091300D81117CC682E07AC682EBE0
:108B10009DE00E94B4C78AE00E948CC781E09AE57C
:108B2000909367148093661480E490E090936914A6
:108B30008093681417E010935A1482E880935D14B0
:108B400084E890E0A0E0B0E080935E1490935F141E
:108B5000A0936014B09361148AE094E10E941C38E1
:108B60001093320D10CE80911F0D882309F40BCE87
:108B70000E94D537882309F406CE0E94281D811152
:108B800002CE84EA9DE00E94B4C78AE00E948CC7AE
:108B90008091200D90E0B0E0A0E0895B9F4FAE4F48
:108BA000B54A21E03AE53093671420936614909318
:108BB00069148093681487E080935A1482E8809344
:108BC0005D1484E890E0A0E0B0E080935E149093A0
:108BD0005F14A0936014B09361148AE094E10E9442
:108BE0001C3810921F0DC4CD0E94D537882309F47C
:108BF000CACD0E94281D8111C6CD81E080938602D6
:108C00001092320D86E99DE00E94B4C78AE00E946E
:108C10008CC781E09AE590936714809366148EE484
:108C200090E0909369148093681487E080935A14BD
:108C300082E880935D1484E890E0A0E0B0E0809347
:108C40005E1490935F14A0936014B09361148AE053
:108C500094E10E941C3897CD0E94281D811193CD6C
:108C600019821A821B821C8262E0CE0101960F9447
:108C700042087ECD0196A11DB11D35E0B695A795A0
:108C8000979587953A95D1F70197A109B109009772
:108C9000E1E0AE07B10548F1B0936714A093661404
:108CA000909369148093681410935A1412E81093E7
:108CB0005D148AE890E1A0E0B0E080935E149093A8
:108CC0005F14A0936014B09361148AE094E10E9451
:108CD0001C3888E090E0909367148093661485E0D8
:108CE00080935A1410935D14A9CD909367148093C8
:108CF000661485E080935A14D9CF909367148093BB
:108D0000661485E0C2CD909367148093661485E065
:108D1000ECCD82E090E005CE8A3F08F020CE8EEFC9
:108D20008093AC0485E89DE00E94B4C78AE00E946D
:108D30008CC781E08093860281E09AE59093671466
:108D4000809366148DE290E0909369148093681488
:108D500087E080935A1482E880935D1484E890E061
:108D6000A0E0B0E080935E1490935F14A093601431
:108D7000B09361148AE094E10E941C381092AB0415
:108D800028960FB6F894DEBF0FBECDBFDF91CF910E
:108D90001F910F91FF90EF90DF90CF90BF90AF9019
:108DA0009F908F907F906F905F904F900895845622
:108DB0009109909367148093661485E080935A1408
:108DC00082E880935D1481E090E1A0E0B0E0DCCD2A
:108DD0008CE090E0909367148093661415E01093F4
:108DE0005A1482E880935D1484E190E1A0E0B0E041
:108DF00080935E1490935F14A0936014B0936114F9
:108E00008AE094E10E941C380E94EA3520E13EE0AD
:108E100040E050E00F94D1382115310581E048073A
:108E2000510508F470C05093671440936614309352
:108E300069142093681487E080935A1412E8109301
:108E40005D1480E190E1A0E0B0E080935E14909327
:108E50005F14A0936014B09361148AE094E10E94BF
:108E60001C380E94EA3520E13EE040E050E00F94DB
:108E7000D1382CE330E040E050E00F94D13830930B
:108E800067142093661405E000935A1410935D1440
:108E900082E190E1A0E0B0E080935E1490935F14D3
:108EA000A0936014B09361148AE094E10E941C388E
:108EB0000E94981F882309F45CC48F5F8093A704E5
:108EC000E82EF12C833330F5EE0CFF1CF092671482
:108ED000E092661400935A1410935D148EE090E1B2
:108EE000A0E0B0E080935E1490935F14A0936014B0
:108EF000B09361148AE094E10E941C3810926714C8
:108F0000109266142BC0309367142093661410934C
:108F10005A1494CF84E690E090936714809366147B
:108F200000935A1410935D148EE090E1A0E0B0E03D
:108F300080935E1490935F14A0936014B0936114B7
:108F40008AE094E10E941C38A2E3EA1AA0E8FA0A37
:108F5000EE0CFF1CF0926714E092661400935A1412
:108F600010935D148FE090E1A0E0B0E080935E1478
:108F700090935F14A0936014B09361148AE094E11D
:108F80000E941C380E94981F90E090936714809371
:108F9000661485E080935A1482E880935D1486E11C
:108FA00090E1A0E0B0E080935E1490935F14A093F2
:108FB0006014B09361148AE094E10E941C3820E0B0
:108FC00030E0A90160910F1370911013809111137B
:108FD000909112130F945D3920E030E048EC52E498
:108FE0000F94F3320F94C93A709367146093661428
:108FF00005E000935A1412E810935D1486E290E1A4
:10900000A0E0B0E080935E1490935F14A09360148E
:10901000B09361148AE094E10E941C3880917D0233
:1090200090917E02909367148093661400935A1473
:1090300010935D1480E093E1A0E0B0E080935E14B3
:1090400090935F14A0936014B09361148AE094E14C
:109050000E941C3820E030E040E251E46091E10CD5
:109060007091E20C8091E30C9091E40C0F94F33238
:109070000F94D03A709367146093661400935A1457
:1090800010935D1482E492E1A0E0B0E080935E145E
:1090900090935F14A0936014B09361148AE094E1FC
:1090A0000E941C3820E030E040E251E46091E50C81
:1090B0007091E60C8091E70C9091E80C0F94F332DC
:1090C0000F94D03A709367146093661400935A1407
:1090D00010935D1486E492E1A0E0B0E080935E140A
:1090E00090935F14A0936014B09361148AE094E1AC
:1090F0000E941C3820E030E040E251E46091E90C2D
:109100007091EA0C8091EB0C9091EC0C0F94F3327F
:109110000F94D03A709367146093661400935A14B6
:1091200010935D148AE492E1A0E0B0E080935E14B5
:1091300090935F14A0936014B09361148AE094E15B
:109140000E941C3820E030E040E251E46091ED0CD8
:109150007091EE0C8091EF0C9091F00C0F94F33223
:109160000F94D03A709367146093661400935A1466
:1091700010935D148EE492E1A0E0B0E080935E1461
:1091800090935F14A0936014B09361148AE094E10B
:109190000E941C3820E030E048EC52E46091071354
:1091A000709108138091091390910A130F94F33270
:1091B0000F94C93A709367146093661400935A141D
:1091C00010935D1486E392E1A0E0B0E080935E141A
:1091D00090935F14A0936014B09361148AE094E1BB
:1091E0000E941C3820E030E048EC52E460910B1300
:1091F00070910C1380910D1390910E130F94F33214
:109200000F94C93A709367146093661400935A14CC
:1092100010935D148AE392E1A0E0B0E080935E14C5
:1092200090935F14A0936014B09361148AE094E16A
:109230000E941C3880918D0290918E029093671449
:109240008093661400935A1410935D1482E592E1A2
:10925000A0E0B0E080935E1490935F14A09360143C
:10926000B09361148AE094E10E941C3880918B02D3
:1092700090918C02909367148093661400935A1413
:1092800010935D1484E592E1A0E0B0E080935E1459
:1092900090935F14A0936014B09361148AE094E1FA
:1092A0000E941C3820E030E040E251E460917F12DF
:1092B0007091801280918112909182120F94F332FA
:1092C0000F94D03A709367146093661400935A1405
:1092D00010935D1486E592E1A0E0B0E080935E1407
:1092E00090935F14A0936014B09361148AE094E1AA
:1092F0000E941C382CEA35EC47E25EE36091831251
:109300007091841280918512909186120F94573A31
:1093100020E030E040E251E40F94F3320F94D03A71
:10932000709367146093661400935A1410935D143D
:109330008AE592E1A0E0B0E080935E1490935F1420
:10934000A0936014B09361148AE094E10E941C38E9
:109350002CEA35EC47E25EE3609187127091881247
:109360008091891290918A120F94F33220E030E0BC
:1093700040E251E40F94F3320F94D03A70936714A3
:109380006093661400935A1410935D148EE592E175
:10939000A0E0B0E080935E1490935F14A0936014FB
:1093A000B09361148AE094E10E941C3820E030E020
:1093B00040E251E4609114127091151280911612DE
:1093C000909117120F94F3320F94D03A7093671460
:1093D0006093661400935A1410935D1482E692E130
:1093E000A0E0B0E080935E1490935F14A0936014AB
:1093F000B09361148AE094E10E941C382CEA35ECA9
:1094000047E25EE3609118127091191280911A126E
:1094100090911B120F94573A20E030E040E251E463
:109420000F94F3320F94D03A7093671460936614DC
:1094300000935A1410935D1486E692E1A0E0B0E028
:1094400080935E1490935F14A0936014B0936114A2
:109450008AE094E10E941C382CEA35EC47E25EE396
:1094600060911C1270911D1280911E1290911F121A
:109470000F94F33220E030E040E251E40F94F332F5
:109480000F94D03A709367146093661400935A1443
:1094900010935D148AE692E1A0E0B0E080935E1440
:1094A00090935F14A0936014B09361148AE094E1E8
:1094B0000E941C388091290D811105C080912B0DCF
:1094C000882309F46DC060917A1270917B12072E87
:1094D000000C880B990B0F94943220E030E048EC9C
:1094E00052E40F94F3326B017C0160917C12709115
:1094F0007D12072E000C880B990B0F9494329B0160
:10950000AC01C701B6010F94573A0F94D03A6536B3
:10951000710510F064E670E0709367146093661450
:1095200005E000935A1412E810935D1484E290E170
:10953000A0E0B0E080935E1490935F14A093601459
:10954000B09361148AE094E10E941C3860917A1211
:1095500070917B12072E000C880B990B0F9494329C
:109560006B017C0120E030E04AE253E40F94BD3B04
:10957000181624F48091290D811146C160917C1246
:1095800070917D12072E000C880B990B0F9494326A
:109590009B01AC01C701B6010F94BD3B87FFAFC172
:1095A00080911F0D882339F180911E0D91E0980F55
:1095B00090931E0D90E0909367148093661485E05D
:1095C00080935A1482E880935D1482E490E1A0E0D5
:1095D000B0E080935E1490935F14A0936014B093F6
:1095E00061148AE094E10E941C3880911E0D8A303B
:1095F00010F010921E0D0E946037882309F4B5C147
:109600006091170D7091180DEE24E394F12C611503
:109610007105A9F090E080E00F94923220E030E0F4
:1096200040E85EE30F94F3320F943B3A20E030E0E1
:1096300040E85FE30F945D390F94D03A7B0101E07D
:1096400010E08091190D811102C010E000E08091BE
:109650004E1390914F138F3F980711F40E94CC80C6
:1096600090934F1380934E13080F191FB80190E089
:1096700080E00F94923220E030E040E85EE30F9407
:10968000F3320F943B3A4B015C01F0926714E09285
:10969000661405E000935A1412E810935D1480E1FB
:1096A00093E1A0E0B0E080935E1490935F14A093E8
:1096B0006014B09361148AE094E10E941C38C501E3
:1096C000B4010F94D03A70936714609366140093BA
:1096D0005A1410935D1482E193E1A0E0B0E080930E
:1096E0005E1490935F14A0936014B09361148AE0A9
:1096F00094E10E941C380AEA14E1AAE1FA2E809152
:109700005704909158042091A5043091A604891B18
:109710008F7309F449C12A3131050CF0DBC19091F6
:109720005704809158044FEF5FEF981749F0E82FE6
:10973000F0E0E95AFB4F42818F5F8F7380935804AA
:10974000F901E655FB4E40838091AA148A3509F051
:10975000B3C162E070E080E090E00E94DD3780916C
:10976000A5049091A60401969093A6048093A50465
:10977000C6CF1092671410926614ACCB60917C1225
:1097800070917D12072E000C880B990B0F94943268
:1097900020E030E0A9010F948D32811134C98CE0B2
:1097A00090E0909367148093661485E080935A1438
:1097B00082E880935D1484E190E1A0E0B0E0F3CB17
:1097C0008DE090E0909367148093661485E0809319
:1097D0005A1482E880935D1484E190E1A0E0B0E047
:1097E00080935E1490935F14A0936014B0936114FF
:1097F0008AE094E10E941C388091300D811101C0F3
:1098000081E08093300DDBCB1092290D20E030E019
:1098100040E251E46091210D7091220D8091230D61
:109820009091240D0F94F3320F94C93A70936714FA
:109830006093661400935A1410935D1484E590E1CC
:10984000A0E0B0E080935E1490935F14A093601446
:10985000B09361148AE094E10E941C3820E030E06B
:1098600040E251E46091250D7091260D8091270D05
:109870009091280D0F94F3320F94C93A70936714A6
:109880006093661400935A1410935D1488E590E178
:10989000A0E0B0E080935E1490935F14A0936014F6
:1098A000B09361148AE094E10E941C3884E69DE044
:1098B0000E94B4C78AE00E948CC781E09AE5909329
:1098C00067148093661481E490E090936914809308
:1098D000681487E080935A1410935D1484E890E034
:1098E000A0E0B0E080935E1490935F14A0936014A6
:1098F000B09361148AE094E10E941C3851CE6091CB
:109900002B0D662309F44CCE062E000C770B8BE44E
:109910009DE00E947BCA8AE00E948CC710922B0DAA
:1099200084E090E0909367148093661485E08093C0
:109930005A1412E810935D148EE890E1A0E0B0E0B4
:1099400080935E1490935F14A0936014B09361149D
:109950008AE094E10E941C3881E09AE590936714B4
:109960008093661483E590E0B0CF10926714109254
:10997000661405E000935A1412E810935D1480E118
:1099800093E1A0E0B0E080935E1490935F14A09305
:109990006014B09361148AE094E10E941C38109224
:1099A00067141092661493CE121613060CF492C02C
:1099B00080910E1490910F14A0911014B091111475
:1099C0008C34E0E19E07A105B10509F4D7C98A34BA
:1099D0009041A105B10509F4D1C920E030E040E291
:1099E00051E46091690270916A0280916B029091DA
:1099F0006C020F94F3320F94C93A7093671460931A
:109A0000661405E000935A1412E810935D1488E47C
:109A100090E1A0E0B0E080935E1490935F14A09377
:109A20006014B09361148AE094E10E941C3820E035
:109A300030E040E251E460916D0270916E028091DD
:109A40006F02909170020F94F3320F94C93A7093A1
:109A500067146093661400935A1410935D148AE49B
:109A600090E1A0E0B0E080935E1490935F14A09327
:109A70006014B09361148AE094E10E941C3820E0E5
:109A800030E040E251E46091710270917202809185
:109A90007302909174020F94F3320F94C93A709349
:109AA00067146093661400935A1410935D148CE449
:109AB00090E1A0E0B0E056C9121613060CF01FCEDC
:109AC000F8012F2D11922A95E9F71092A604109211
:109AD000A50415CE90910B148091AA14981321C05F
:109AE00090910C148091AB1498131BC02330310556
:109AF000C4F09091AC1490930A148091AD148093AB
:109B00000D149330D1F4982F9D7F9038B1F490913B
:109B1000AE149F3409F059C09091AF149B3409F0F2
:109B200054C0EAEAF4E18AE1DF011D928A95E9F77F
:109B30001092A6041092A5043BCF833809F045C0CB
:109B40008091AE149091AF14982789279827B0E0A0
:109B5000A0E080930E1490930F14A0931014B09370
:109B60001114C090B014D12CF12CE12CC09212141D
:109B7000D0921314E0921414F092151421EB34E1F6
:109B800040E050E0BA014C155D056E057F0508F018
:109B90004AC0DB01CA01B695A795979587950696A9
:109BA000880F991FFC01E65FFB4ED9018C9111963D
:109BB0009C91892798278927918380834E5F5F4FE7
:109BC0006F4F7F4F2E5F3F4FDECF813861F5809121
:109BD000AE1490E0B0E0A0E080930E1490930F14C8
:109BE000A0931014B09311148091AF14482F50E03B
:109BF00070E060E0409312145093131460931414B7
:109C000070931514A0EBB4E1E6E1F4E190E030E0EC
:109C100020E08217930739F04D9150E04193519322
:109C20002F5F3F4FF6CFEAEAF4E18AE1DF011D92B0
:109C30008A95E9F71092A6041092A5040F94E408FF
:109C4000B7CE6F927F928F929F92AF92BF92CF9238
:109C5000DF92EF92FF920F931F93CF93DF93CDB7D5
:109C6000DEB764970FB6F894DEBF0FBECDBF10927B
:109C7000D0008091D00082608093D0001092D500F7
:109C800080E18093D4008091D10080618093D100E5
:109C90008091D10088608093D1008091D10080684C
:109CA0008093D1008091D1008F7D8093D1008AE58F
:109CB00080935B1480930B1485EA80935C148093EB
:109CC0000C14EAEAF4E18AE1DF011D928A95E9F7D2
:109CD00080912E0D882309F473C283E090E0909365
:109CE00067148093661485E080935A1482E8809309
:109CF0005D148FE190E1A0E0B0E080935E1490935A
:109D00005F14A0936014B09361148AE094E10E9400
:109D10001C3884E690E0909367148093661405E005
:109D200000935A1412E810935D1486E090E1A0E0CD
:109D3000B0E080935E1490935F14A0936014B0938E
:109D400061148AE094E10E941C388BE090E09093CB
:109D500067148093661400935A1410935D1480E086
:109D600092E1A0E0B0E080935E1490935F14A09322
:109D70006014B09361148AE094E10E941C38109240
:109D800067141092661400935A1410935D1484E3C0
:109D900090E1A0E0B0E080935E1490935F14A093F4
:109DA0006014B09361148AE094E10E941C38109210
:109DB00067141092661400935A1410935D148AE38A
:109DC00090E1A0E0B0E080935E1490935F14A093C4
:109DD0006014B09361148AE094E10E941C38809171
:109DE0007A1290917B12909367148093661400937B
:109DF0005A1410935D1486E390E1A0E0B0E08093E4
:109E00005E1490935F14A0936014B09361148AE081
:109E100094E10E941C3880910F129091101290933F
:109E200067148093661400935A1410935D148CE3A6
:109E300090E1A0E0B0E080935E1490935F14A09353
:109E40006014B09361148AE094E10E941C3882E0AF
:109E500090E0909367148093661400935A141093C3
:109E60005D148EE190E1A0E0B0E080935E149093E9
:109E70005F14A0936014B09361148AE094E10E948F
:109E80001C3881E08093850270E6C72E70E1D72EE2
:109E9000E12CF12C109267141092661400935A145E
:109EA00010935D14C0925E14D0925F14E09260141F
:109EB000F09261148AE094E10E941C38BFEFCB1A43
:109EC000DB0AEB0AFB0AE4E7CE16E0E1DE06E1047A
:109ED000F10401F7CE0101967C0184E1D7011D92C6
:109EE0008A95E9F781E08F9390E99F938F9398E6A5
:109EF0009F938F939F938AEC93E09F938F93FF920E
:109F0000EF920F94E53C20E630E140E050E067ED51
:109F100073E08AE094E10E9443F12AE630E140E0F8
:109F200050E064EE73E08AE094E10E9443F124E79C
:109F300030E140E050E0B7018AE094E10E9443F153
:109F40002EE730E140E050E060EF73E08AE094E11A
:109F50000E9443F1109267141092661400935A14F1
:109F600010935D148EE090E1A0E0B0E080935E1469
:109F700090935F14A0936014B09361148AE094E10D
:109F80000E941C38109267141092661400935A14A1
:109F900010935D148FE090E1A0E0B0E080935E1438
:109FA00090935F14A0936014B09361148AE094E1DD
:109FB0000E941C380FB6F894DEBF0FBECDBF4AE03A
:109FC000C42E40E2D42EE12CF12C55E0752E62E82F
:109FD000662E460157010AE010E0109267141092B5
:109FE000661470925A1460925D1480925E1490927E
:109FF0005F14A0926014B09261148AE094E10E9410
:10A000001C3801501109FFEF8F1A9F0AAF0ABF0ACF
:10A010000115110511F78AE0C80ED11CE11CF11CD5
:10A0200092EDC91690E2D906E104F10491F6C12C33
:10A0300030E2D32EE12CF12C05E012E810926714E7
:10A040001092661400935A1410935D14C0925E141B
:10A05000D0925F14E0926014F09261148AE094E16F
:10A060000E941C38109267141092661400935A14C0
:10A0700010935D14D701C6018C529F4FAF4FBF4F55
:10A0800080935E1490935F14A0936014B093611456
:10A090008AE094E10E941C38AFEFCA1ADA0AEA0A91
:10A0A000FA0ABAE0CB16B0E2DB06E104F10431F6BD
:10A0B0002EEDC22E20E2D22EE12CF12C05E012E88A
:10A0C000109267141092661400935A1410935D1442
:10A0D000C0925E14D0925F14E0926014F09261140A
:10A0E0008AE094E10E941C38EFEFCE1ADE0AEE0AF5
:10A0F000FE0AF6EECF16F0E2DF06E104F10401F706
:10A10000CC24C39482E1D82EE12CF12C9AE0A92E24
:10A11000B12C05E012E8B0926714A0926614009387
:10A120005A1410935D14C0925E14D0925F14E092A2
:10A130006014F09261148AE094E10E941C38B0929D
:10A140006714A092661400935A1410935D14D701FB
:10A15000C6018096A11DB11D80935E1490935F147B
:10A16000A0936014B09361148AE094E10E941C38BB
:10A170008FEFC81AD80AE80AF80A95E1C91692E1E1
:10A18000D906E104F10439F684E39DE00E94B4C7E6
:10A190008AE00E948CC764960FB6F894DEBF0FBEAB
:10A1A000CDBFDF91CF911F910F91FF90EF90DF9086
:10A1B000CF90BF90AF909F908F907F906F900895B9
:10A1C00082E090E08CCD0E94214E1092AC0481E0A0
:10A1D0008093860286EE9DE00E94B4C78AE00C94CC
:10A1E0008CC7AB01BC014093CC145093CD14609349
:10A1F000CE147093CF1484E396E10C94757CCF93C6
:10A20000DF93DB01F9019C919130C1F0943080F033
:10A2100094509C938830D1F480819181009771F0A3
:10A22000019791838083480F591FEA01188206C065
:10A230008C3539F49C5F9C93943041F4DF91CF913D
:10A2400008958B3339F781E08C93F8CF20813181E9
:10A25000B9016F5F7F4F71836083420F531FEA0123
:10A260008883808191818F3591056CF7E7CF0F93BB
:10A270001F9381E00091CC141091CD142091CE1445
:10A280003091CF144091C8145091C9146091CA14F0
:10A290007091CB14041715072607370708F480E0E0
:10A2A0001F910F9108954F925F926F927F928F92BC
:10A2B0009F92AF92BF92CF92DF92EF92FF920F9355
:10A2C0001F93CF931092A4041092A3042FE3209322
:10A2D000A2041092A1041092A00410929F04109264
:10A2E00052041092530410925404109255049C018D
:10A2F000F90190812F5F3F4F9032D1F39E34C9F422
:10A30000818190ED980F9A3020F08D3211F08B32D0
:10A3100081F432969F012F5F3F4F808180538A30B6
:10A3200008F47EC09F012F5F3F4F8081803209F487
:10A3300079C0F093CA07E093C9078F010F5F1F4FE1
:10A34000C0816AE270E0C8010F94AB3C009731F025
:10A35000FC01319780818032E1F31182CD3429F004
:10A36000C43519F0C73409F04BC0F80180810F5F84
:10A370001F4F8032D1F380538A3008F041C0C09320
:10A38000A20490E080E04AE0DF011196489F90012E
:10A39000499F300D1124C901C0972081820F911D62
:10A3A00027FD9A95218130ED320F3A30E8F19093F4
:10A3B000A1048093A0042E3261F4329630E04AE08A
:10A3C000DF0131962C9150ED520F5A3078F13093D5
:10A3D0009F049D01D9012F5F3F4F4C914032D1F333
:10A3E000CD34A1F58E31910539F030F587319105E5
:10A3F00019F08C31910551F5B093A404A093A304F6
:10A40000CF911F910F91FF90EF90DF90CF90BF9071
:10A41000AF909F908F907F906F905F904F90089536
:10A42000F90178CFF9017ECFFD01AECF349F200D29
:10A43000112430ED320FC4CF8537910538F08737BE
:10A440009105D0F2803A23E09207B1F25091C9070A
:10A4500070E060E0C12CD12C7601C394FD013196EF
:10A460004C91442309F492C04132A1F4CD3491F4CB
:10A470008032910579F4F093A404E093A30463E29D
:10A4800070E0CF010F94AB3C009709F4B9CFFC0109
:10A490001082B6CF41544A3108F073C0DF012D91CC
:10A4A000203209F459C030ED320F3A3008F465C05B
:10A4B0002E3209F053C0218120532A3008F45DC0A8
:10A4C00030E020E06115710519F4BF016150710998
:10A4D000A42FB0E02601370104C0440C551C661CB3
:10A4E000771C4A95D2F78090520490905304A09024
:10A4F0005404B090550484289528A628B728809243
:10A50000520490925304A0925404B0925504211521
:10A510003105A9F1251BA85CBB4F2C932081215448
:10A52000DF012A3108F49ACFDF012191222309F4B7
:10A5300095CF30ED320F3A30B8F333ED320F323081
:10A5400098F32B3289F39D012F5F3F4F4C9140329E
:10A5500009F084CFD901F7CFFD01A0CF2D3219F03A
:10A560002B3209F0ADCF218130ED320F3A3028F097
:10A570002E3209F0A5CF22819FCF9F01A9CF20E0E5
:10A58000CACF6115710551F6BD01C8CF7093A404FF
:10A590006093A30435CFCF93DF93EC018991882397
:10A5A00019F00E948CC7FACF8DE00E948CC78AE018
:10A5B000DF91CF910C948CC7EF92FF920F931F9372
:10A5C000CF93DF93CDB7DEB762970FB6F894DEBFB7
:10A5D0000FBECDBF0E947F2A882309F43FC04EE002
:10A5E00054E082FF02C043E054E02EE034E081FFFB
:10A5F00002C025E034E080FD2EC08EE094E05F9341
:10A600004F933F932F939F938F938FEF9EE09F9352
:10A610008F938E010F5F1F4F1F930F930F94243260
:10A620000E9418DCC8010E94CB52C8010E9417F595
:10A630000FB6F894DEBF0FBECDBF81E062960FB6B5
:10A64000F894DEBF0FBECDBFDF91CF911F910F9168
:10A65000FF90EF90089587E094E0D1CF80E0EECFB7
:10A66000AF92BF92CF92DF92EF92FF920F931F9320
:10A67000CF93DF93CDB7DEB7E6970FB6F894DEBF82
:10A680000FBECDBF0091A3041091A404F801019066
:10A690000020E9F731976F01C01AD10AF801CF0104
:10A6A000801B910B8C159D053CF481918F32B9F77D
:10A6B000DF0111971C92F3CF8BE1E0EFF4E1DE01B3
:10A6C0005C9601900D928A95E1F7F12CE12CEC1447
:10A6D000FD040CF05DC0F801EE0DFF1D80818111BD
:10A6E00003C08FEFE81AF80A5801AE0CBF1CF50141
:10A6F0008081882309F44CC0FFEFEF1AFF0AF801AC
:10A70000EE0DFF1D7F01E01AF10A81918111FACF50
:10A71000CE014C960E94C7808BE1FE017C96DE0143
:10A72000119601900D928A95E1F7B501CE0101963F
:10A730000E94D578CE0101960E94D4BF8FE20E947C
:10A740008CC780912E1281113BC089E094E00E9459
:10A75000347C8091D01484FF1BC019821C8221E0BC
:10A76000A501BE01645E7F4FCE0101960E94098360
:10A77000811129C08AE00E948CC70E9418DCB501B3
:10A7800084EE9CE00E940ADCCE0101960E94D4BFB8
:10A790008AE00E948CC7CE014C960E94D4BFE696F8
:10A7A0000FB6F894DEBF0FBECDBFDF91CF911F91E2
:10A7B0000F91FF90EF90DF90CF90BF90AF900895F2
:10A7C0008EE292E1C4CFCE014C960E9436808BE19E
:10A7D000FE013196DE015C9601900D928A95E1F7BB
:10A7E000CE0101960E94D4BF72CF3F924F925F92EA
:10A7F0006F927F928F929F92AF92BF92CF92DF9291
:10A80000EF92FF920F931F93CF93DF9380915404A5
:10A8100087FD38C0809155048370A1F5C091131352
:10A82000D0911413488159816A817B8185ED9CE028
:10A830000E94E5C94C815D816E817F818AE691E34A
:10A840000E94E5C940910F135091101360911113AC
:10A850007091121387E691E30E94E5C98AE0DF91C7
:10A86000CF911F910F91FF90EF90DF90CF90BF900D
:10A87000AF909F908F907F906F905F904F903F90A0
:10A880000C948CC760900713709008138090091384
:10A8900090900A13A0900B13B0900C1300910D131D
:10A8A00010910E13C0900F13D0901013E09011135D
:10A8B000F090121388E50E9481BEC82F882309F406
:10A8C0009AC00E9409BE362E472E582ED92F20E05E
:10A8D00030E044EB53EC0F94BD3B87FD0DC020E00E
:10A8E00030E044EB53E4632D742D852D9D2F0F94A0
:10A8F0008D3218160CF081C068E671E082EC9CE0A5
:10A900000E947BCA68E671E08DEB9CE00E947BCAE6
:10A910008AEB9CE00E94B4C7C0E089E50E9481BE3A
:10A92000882361F10E9409BE362E472E582ED92F5A
:10A9300020E030E044EB53EC0F94BD3B87FD0DC0AD
:10A9400020E030E044EB53E4632D742D852D9D2FE2
:10A950000F948D3218160CF055C068E671E087EA46
:10A960009CE00E947BCA68E671E082EA9CE00E945B
:10A970007BCA8FE99CE00E94B4C7C0E08AE50E94D0
:10A9800081BE882309F443C00E9409BE6B017C018B
:10A9900020E030E040E151EC0F94BD3B87FD0AC060
:10A9A00020E030E040E151E4C701B6010F948D3260
:10A9B00018166CF567EF7FEF8DE89CE00E947BCA6C
:10A9C00069E070E088E89CE00E947BCA85E89CE032
:10A9D000DF91CF911F910F91FF90EF90DF90CF907B
:10A9E000BF90AF909F908F907F906F905F904F90AF
:10A9F0003F900C94B4C7C1E090CF632C742C852C8D
:10AA00009D2E8BCFA32CB42C052D1D2FB7CFCC237F
:10AA1000E1F0C301D4018093071390930813A0932E
:10AA20000913B0930A13C501D80180930B139093B7
:10AA30000C13A0930D13B0930E13C0920F13D0926A
:10AA40001013E0921113F0921213DF91CF911F9126
:10AA50000F91FF90EF90DF90CF90BF90AF909F90BD
:10AA60008F907F906F905F904F903F900895CF921E
:10AA7000DF92EF92FF928AE50E9481BE882309F45B
:10AA80005AC00E9409BE20E030E040E050EC0F9434
:10AA90008D32C12CD12CE12C90ECF92E87FD0FC00A
:10AAA0000E9409BE20E030E040E050E40F94BD3B3E
:10AAB00018160CF462C00E9409BE6B017C01209143
:10AAC000E90C3091EA0C4091EB0C5091EC0CC70171
:10AAD000B6010F94F3320F94C93ACB010E94A0F44F
:10AAE00080E50E9433BE81114EC0A701960160919E
:10AAF0000F137091101380911113909112130F94F2
:10AB00005D3960930F13709310138093111390931A
:10AB100012130E9418DC40910F1350911013609192
:10AB200011137091121386E79CE00E94E5C98AE038
:10AB30000E948CC705C083E50E9481BE8111A1CF10
:10AB40008091540487FD24C080915504837001F5E1
:10AB50000E9418DC40910F13509110136091111353
:10AB60007091121387E69CE00E94E5C98AE0FF908D
:10AB7000EF90DF90CF900C948CC7C12CD12CE12C9E
:10AB800080E4F82E9CCF0E94F5BD8111AECFD8CFC6
:10AB900082E50E9433BE8111DBCFFF90EF90DF9002
:10ABA000CF9008954F925F926F927F928F929F9273
:10ABB000AF92BF92CF92DF92EF92FF92CF93DF934B
:10ABC000CDB7DEB72C970FB6F894DEBF0FBECDBF62
:10ABD000409013095090140960901509709016095F
:10ABE00020914F02309150024091510250915202F7
:10ABF000C301B2010F945D3969837A838B839C838F
:10AC00008090170990901809A0901909B0901A091E
:10AC100020915302309154024091550250915602B6
:10AC2000C501B4010F945D396D837E838F8398874E
:10AC3000C0901B09D0901C09E0901D09F0901E09DE
:10AC400020915702309158024091590250915A0276
:10AC5000C701B6010F945D3969877A878B879C8716
:10AC600020915B0230915C0240915D0250915E0246
:10AC7000C301B2010F945D392B013C0120915F02A9
:10AC8000309160024091610250916202C501B401AD
:10AC90000F945D394B015C01209163023091640295
:10ACA0004091650250916602C701B6010F945D396B
:10ACB0006B017C010E9418DC88E894E00E94B4C714
:10ACC00083E50E9433BE882321F00E94F5BD809366
:10ACD0004D0280914D02811151C08FE694E00E9497
:10ACE000B4C780E894E00E94B4C749815A816B815F
:10ACF0007C8186EE93E10E94E5C94D815E816F8182
:10AD000078858AE691E30E94E5C949855A856B8575
:10AD10007C8587E691E30E94E5C98EE794E00E9476
:10AD2000B4C786E794E00E94B4C7B301A20186EEDF
:10AD300093E10E94E5C9B501A4018AE691E30E946E
:10AD4000E5C9B701A60187E691E30E94E5C98AE05B
:10AD50002C960FB6F894DEBF0FBECDBFDF91CF911A
:10AD6000FF90EF90DF90CF90BF90AF909F908F902B
:10AD70007F906F905F904F900C948CC783E794E026
:10AD8000AECF2F923F924F925F926F927F928F92AF
:10AD90009F92AF92BF92CF92DF92EF92FF920F936A
:10ADA0001F93CF93DF93CDB7DEB7E5970FB6F89437
:10ADB000DEBF0FBECDBF8DAB209137042CAB81E041
:10ADC000809337048091A2048D3409F40EC6843533
:10ADD00011F40C942D6C873409F091C18091A0047A
:10ADE0009091A1048B31910509F430C208F079C12A
:10ADF0008430910508F030C120911F068230910502
:10AE000008F4E1C1213009F0E4C111E0029709F032
:10AE100010E00E94D51F19821A821B821C821D829B
:10AE20001E821F82188682E50E9481BE882309F453
:10AE3000E3C10E9409BE6B017C0120E030E0A90162
:10AE40000F948D32882309F4EAC040906902509033
:10AE50006A0260906B0270906C0280916D0290911A
:10AE60006E02A0916F02B09170028CA79DA7AEA751
:10AE7000BFA78090B7079090B807A090B907B0908F
:10AE8000BA078091BB079091BC07A091BD07B09114
:10AE9000BE0788AB99ABAAABBBABA5019401C301BC
:10AEA000B2010F948D3281110DC028A939A94AA988
:10AEB0005BA96CA57DA58EA59FA50F948D328823D7
:10AEC00009F4ADC0A3019201C501B4010F945C392E
:10AED00020E030E040E05FE30F94F33268A779A709
:10AEE0008AA79BA72CA53DA54EA55FA568A979A912
:10AEF0008AA99BA90F945C3920E030E040E05FE331
:10AF00000F94F3322B013C0120E030E0A901C7018E
:10AF1000B6010F948D32881F8827881F181709F4EF
:10AF200062C180E090E0A0E8BFEB8CA79DA7AEA730
:10AF3000BFA728A539A54AA55BA5CA01B9010F94E9
:10AF4000F3324B015C01A3019201C301B2010F94E2
:10AF5000F3329B01AC01C501B4010F945D390F942C
:10AF60000B3C4B015C01AC019B01C701B6010F9486
:10AF70005C3968AB79AB8AAB9BABA5019401C70187
:10AF8000B6010F945D399B01AC0168A979A98AA922
:10AF90009BA90F94F3326B017C0120E030E0A90102
:10AFA0000F94BD3B87FD24C1C701B6010F940B3C34
:10AFB0006B017C01C301B2019058A50194010F946B
:10AFC000573A2CA53DA54EA55FA50F94F332A701D6
:10AFD00096010F94F33228A539A54AA55BA50F94D5
:10AFE0005D3969837A838B839C83A501940168A56D
:10AFF00079A58AA59BA50F94573A2CA53DA54EA5EA
:10B000005FA50F94F332A70196010F94F332A301C9
:10B0100092010F945D396D837E838F83988720E042
:10B0200030E0A90169817A818B819C810F948D32F6
:10B030008111F6C020E030E0A9016D817E818F8111
:10B0400098850F948D328111EBC00E9414DC80E64C
:10B0500095E00E94B4C7BDC08531910509F4B9C01F
:10B060008A31910509F4EFC0049709F048C080E5E2
:10B070000E9481BEC12CD12C7601882321F00E9430
:10B0800086B86B017C0183E50E9481BE882361F054
:10B090000E9409BE20E030E04AE754E40F94F33206
:10B0A0000F94D03A6B017C010E94D4238091B4119B
:10B0B000811105C060E086E795E00E94EC3C0E94AB
:10B0C0002974C60ED71EE81EF91E0E9429746C1939
:10B0D0007D098E099F0997FF7CC080E00E94C3DF35
:10B0E000F4CF8232910509F444C360F48D319105A7
:10B0F00009F46CC208F4C3C04E9709F4BFC20F94A0
:10B100006C2367C08A35910509F4F8C308F58A975E
:10B11000B1F780911F06813009F05BC089E40E947D
:10B1200081BE082FF12C882319F00E9405BEF82E4D
:10B130008AE40E9481BEE82E882309F41DC30E9480
:10B1400005BE182F01111BC3153008F422C31AC302
:10B150008B35910509F4D5C38C35910581F6809125
:10B160009F04882309F4D1C3893099F56AEEA62E8D
:10B1700062E0B62E79E6C72E72E0D72EE12C00E011
:10B1800010E0D5018D915D010E9481BEF82E8823CB
:10B1900061F0133011F4082FFE2C0E9409BEF60155
:10B1A0006083718382839383EF2C1F5FF4E0CF0E63
:10B1B000D11C143031F7EE2009F4F9C30E94E031BC
:10B1C0000E940B3206C0213021F40E94D51F0E943C
:10B1D0004D2B3DA9311102C00F9419238CA98093E6
:10B1E00037040C948E6480E090E0A0E8BFE39DCE2D
:10B1F000C12CD12C7601DECE89E40E9481BE882349
:10B2000031F00E9409BE69837A838B839C838AE430
:10B210000E9481BE882309F402CF0E9409BEFBCEA2
:10B22000412FBE016F5F7F4F87EB97E00E947793BE
:10B230000E9429746093051270930612809307127E
:10B2400090930812C6CF0E94DBD3C3CF87E00E9441
:10B25000DC528111BECF8CE0EEEDF2E0DE01119602
:10B2600001900D928A95E1F770E060E080E50E9420
:10B27000C71FBE016F5F7F4F0E943736AACF87E09E
:10B280000E947F2A811106C060E08FE40E9420BFE7
:10B2900081119FCF0E94D42310924E026091C80C5E
:10B2A0008CE40E9420BFE82E80E00E94C7C10E946B
:10B2B000297460930512709306128093071290937D
:10B2C00008120E94192E81E08093DB050E947433DE
:10B2D0008AE50E9433BEF82E882369F081E00E943F
:10B2E0007F2A182F82E00E947F2A11110C94506C43
:10B2F00011E0811101C010E088E50E9433BE811188
:10B300000C94426C111149C189E50E9433BE082F8B
:10B31000811307C0012FF11204C011E001E0FF24E6
:10B32000F39482E50E9481BE882309F439C10E940A
:10B3300009BE6CA37DA38EA39FA320E030E0A901EA
:10B340000F948D32882381F0111105C0011103C0C3
:10B35000FF2009F414C160E0CE0184960E94D4302D
:10B360000E94A6C50E9470C5112309F47DC0002368
:10B3700009F477C01092690210926A0210926B026F
:10B3800010926C0210926D0210926E0210926F0277
:10B39000109270020E94E03182E49FE00E9496B811
:10B3A0004B015C0186E49FE00E9496B82B013C01B2
:10B3B000AC019B01C501B4010F94BD3B18160CF004
:10B3C000F4C0A5019401C301B2010F94573A9B0147
:10B3D000AC010F94F33220E030E040E85FE30F94DB
:10B3E0005D390F940B3C20E030E048E452E40F94C8
:10B3F000F33268A379A38AA39BA320E030E040EC5A
:10B400005FE3C301B2010F94F33269837A838B83C4
:10B410009C8320E030E040EC5FE3C501B4010F9471
:10B42000F3326C8F7D8F8E8F9F8FAE01405E5F4FAA
:10B43000BE016F5F7F4FCE014C960E9493300E94F9
:10B440008A1F1092690210926A0210926B02109287
:10B450006C0210926D0210926E0210926F021092A6
:10B46000700280E00E940934002319F081E00E94FC
:10B470000934FF2009F483C010921E0510921D05A7
:10B4800010921F0583E00E94DC52811178C00E9457
:10B49000E0312091490830914A0840914B08509181
:10B4A0004C0860E070E084E393E40F945C392B0176
:10B4B0003C0120914D0830914E0840914F08509129
:10B4C000500860E070E084E393E40F945C394B0132
:10B4D0005C018091710290917202A0917302B0910F
:10B4E00074028093BF079093C007A093C107B093E5
:10B4F000C2070091131310911413D8012D913D919F
:10B500004D915C91C301B2010F945C396093B70710
:10B510007093B8078093B9079093BA07F801248114
:10B52000358146815781C501B4010F945C39609320
:10B53000BB077093BC078093BD079093BE0787EB52
:10B5400097E00E9490BD8823A9F11C8E1D8E1E8E4F
:10B550001F8E88E0E7EBF7E0DE01119601900D9277
:10B560008A95E1F7AE01445E5F4FBE016B5F7F4F8E
:10B57000CE0101960E94933082E00E9409340E941D
:10B58000E0318091DA058093DB058E2D0E94C7C1E2
:10B590000E94002E0E940B321CCE012F10E0C1CE63
:10B5A00060E070E080E890E4C4CEA3019201C501A0
:10B5B000B4010BCF60E081E995E00E94EC3C0E9471
:10B5C00018DC8FE795E00E94B4C7D9CF14E00E9441
:10B5D000297460930512709306128093071290935A
:10B5E00008128091C80C811127C08EE40E9433BEDE
:10B5F000882321F082EA95E00E94826C87E00E9415
:10B60000DC5281111FC00E94EFE68823D9F011504F
:10B6100001F130E020E04AE25EE06DEC75E085E0AB
:10B620000E941CC961E080EC95E00E94C3C888EAD2
:10B6300095E00E94826CCBCF60E08FE40E9420BF37
:10B64000882399F20E94F4C88BE696E00E94826CEF
:10B65000C0CD61E08EE596E00E94C3C889EE95E01A
:10B660000E94826C61E085E19EE00E94C3C840E0D8
:10B6700070E060E08AED95E00E94F2DE0091131325
:10B6800010911413D8012D913D914D915C916091D1
:10B69000690270916A0280916B0290916C020F9422
:10B6A0005D39AB01BC0188E50E94EEBE69837A83F7
:10B6B0008B839C83F8012481358146815781609179
:10B6C0006D0270916E0280916F02909170020F94E2
:10B6D0005D39AB01BC0189E50E94EEBE6D837E83BE
:10B6E0008F839887BE016B5F7F4FCE0101960E94CA
:10B6F000BFB8882309F46DCD80E00E94C7C10E94C5
:10B70000192E61E085E40E9420BF182F01E021E09E
:10B71000482FBE016B5F7F4FCE0101960F94A92386
:10B720006B017C01AC019B010F944F3C811119C04E
:10B7300049815A816B817C818DE896E00E94E5C940
:10B740004D815E816F81788588E896E00E94E5C929
:10B75000B701A60183E896E00E94E5C98AE00E944D
:10B760008CC70E94002E11110E94A5B80E940B32B6
:10B7700030CD0E9442CF2DCD10E0002351F0F4E0F7
:10B78000FF1528F485E996E00E94B4C722CDE110A8
:10B79000DBCC80E1E9E6F2E0A7EBB7E001900D92A7
:10B7A0008A95E1F7002319F16F2DFF0C770B880BB9
:10B7B000990B0F9494322091090530910A0540911C
:10B7C0000B0550910C050F94F33220910105309137
:10B7D000020540910305509104050F945D39609373
:10B7E000B7077093B8078093B9079093BA07EE2014
:10B7F00019F1612F110F770B880B990B0F9494326D
:10B8000020910D0530910E0540910F0550911005C6
:10B810000F94F332209105053091060540910705FC
:10B82000509108050F945D396093BB077093BC0776
:10B830008093BD079093BE0760E080E50E9420BF23
:10B840008823C1F10023D1F0E0911313F091141378
:10B8500020813181428153816091B7077091B8078F
:10B860008091B9079091BA070F945C396093B7073C
:10B870007093B8078093B9079093BA07EE20D1F080
:10B88000E0911313F091141324813581468157817F
:10B890006091BB077091BC078091BD079091BE0776
:10B8A0000F945C396093BB077093BC078093BD070E
:10B8B0009093BE0740E050E0BA0186E40E94EEBEDD
:10B8C0006B017C0120E030E0A9010F94BD3B18160C
:10B8D0008CF420E030E040E752E4C701B6010F9459
:10B8E000573A69837A838B839C83CE0101960E94A9
:10B8F000382E6FCC60E070E0CB01F3CF10923708A8
:10B9000068CC8FE08093370864CC5AEEC52E52E0A5
:10B91000D52EF12CE12C00E010E0D6018D916D01C7
:10B920000E9481BE382E8823D9F10E9409BE4B01A6
:10B930005C01133059F0F701ED5EF64F2081318143
:10B94000428153810F945C394B015C01F701E75947
:10B95000FD4F2081318142815381C501B4010F9493
:10B960005C392B013C012DEB37E346E855EB0F9496
:10B97000BD3B87FD0AC02DEB37E346E855E3C30125
:10B98000B2010F948D3218165CF41330C1F480921A
:10B99000750290927602A0927702B0927802032DFF
:10B9A0001F5FB4E0EB0EF11C143009F0B6CF00239A
:10B9B00009F406CC85E792E00E94A52701CCF701A7
:10B9C000E35CF74F5F01A301920160817181828185
:10B9D00093810F945D39D5016D937D938D939C93E5
:10B9E0001397812F0E94081DDBCF8091A0049091B6
:10B9F000A1048937910511F40C94A16608F0B2C135
:10BA00008D34910509F497C608F0CEC08A319105AE
:10BA100009F4CCC508F071C08431910509F412C550
:10BA200008F04EC08131910509F4D1C408F042C03C
:10BA3000029708F064CB80E50E9481BEC12CD12C16
:10BA40007601882321F00E9486B86B017C0183E592
:10BA50000E9481BE882361F00E9409BE20E030E090
:10BA60004AE754E40F94F3320F94D03A6B017C010F
:10BA70000E94D4238091A3049091A404892B09F4FB
:10BA8000A1C40F947A238091A0049091A10466EB45
:10BA900076E0892B11F46EEA76E030E020E04EEBA0
:10BAA00056E082E00E941CC940E0C701B6010E9436
:10BAB00008EF8FCB429709F022CB0E948EBE89CB34
:10BAC0008731910509F4F3C470F48531910509F4C7
:10BAD000EAC4469709F013CB8091D01482FD79CB4C
:10BAE0000E94508076CB8831910509F4F5C44997BE
:10BAF00009F005CB0E9432226CCB8032910509F40B
:10BB0000D9C5C0F58D31910509F4BDC570F48B31EF
:10BB1000910509F45EC54C9709F0F1CA8091A30420
:10BB20009091A4040E94428554CB8E31910509F472
:10BB3000B1C54F9709F0E3CA0E94EA356C8F7D8F3B
:10BB40008E8F9F8FBE016F5F7F4FCE014C960E94FC
:10BB5000601ECE0101960E9417F50E9418DCBE01FE
:10BB60006F5F7F4F82E397E00E940ADC8AE00E94C9
:10BB70008CC72FCB8934910509F4C9C550F48132A3
:10BB8000910509F4C0C5C09709F0B9CA0E9485CAD9
:10BB900020CB8B34910509F4CAC58C34910509F08A
:10BBA000AECA0E94933915CB8C36910509F411CB9E
:10BBB00008F071C08535910509F4B0C790F582355C
:10BBC000910509F49BC720F58E34910509F4B7C59A
:10BBD0008135910509F093CA0E94EA8B0E94E52302
:10BBE0000E94F1C30E94F4C31092D2071092D107B1
:10BBF0001092D00768EE73E080E090E00E94E4C20B
:10BC00000E94F9C360E08DEF97E00E94EC3CE1CA2E
:10BC10008335910509F47AC78435910509F44DCF30
:10BC20006ECA8936910509F467C600F58C35910511
:10BC300009F499C78836910509F061CA8091850C8D
:10BC400083FDC7CA0E94022187FDC3CA83E50E9403
:10BC500081BE882341F00E9405BE0E94A42361E0BA
:10BC600080E00F948D260F94EC25B3CA8A36910597
:10BC700009F46DC68B36910509F041CA60E080E594
:10BC80000E9414BF823008F0A4CAE82FF0E0E85BFD
:10BC9000F64F10829ECA8237910511F40C945466B7
:10BCA000A0F58F36910509F47BC6C8F48D36910551
:10BCB00009F4D7C58E36910509F021CA8EE40E9499
:10BCC00081BE882309F485CA0E94D1BD6093B50D59
:10BCD0007093B60D8093B70D9093B80D7ACA8037E4
:10BCE000910509F476CA8137910509F008CA83E500
:10BCF0000E9481BE882309F49AC60E94E1BD8D335B
:10BD000008F090C68093000264CA8637910509F452
:10BD1000DBC7B8F48337910509F4CEC785379105A1
:10BD200009F0EDC98091A3049091A404009709F44F
:10BD3000C7C7DC012C91222309F4C2C70E9417F562
:10BD400048CA8737910511F40C949D668837910590
:10BD500009F0D5C981E08093DB058093DA050E9464
:10BD6000743337CA8A39E1E09E0709F432CA08F011
:10BD7000D0C18C3D910511F40C944C6708F076C04D
:10BD8000893C910509F4E7C708F055C08B39910546
:10BD900009F48DC6D8F48D37910509F4ABCE8C38F3
:10BDA000910509F0ACC98091850C83FD12CA83E529
:10BDB0000E9481BE882309F40CCA0E9405BE0E941D
:10BDC00085BD61E080E00F948D2603CA8E3B91050E
:10BDD00009F43AC6883C910509F091C90E940221F4
:10BDE000182F87FDF6C900913C0884E40E9481BEAB
:10BDF000F82E8823B9F00E9409BE4B015C0120E0B7
:10BE000030E0A9010F948D32882309F4A2C724E001
:10BE10001202F0011124E85CF74F80829182A28225
:10BE2000B3820F2D602F83E50E9420BF80933C08D2
:10BE30000E942D24CEC98D3C910509F4D9C758F430
:10BE40008B3C910509F4B1C78C3C910509F057C9A9
:10BE50000E94F6C9BEC98E3C910509F4CDC7833D49
:10BE6000910509F04CC90E94D255B3C98E3221E028
:10BE7000920711F40C94876808F0B4C08232A1E0F4
:10BE80009A0711F40C94656848F58D3D910511F4FD
:10BE90000C948F678831914009F031C980E50E9488
:10BEA00033BE882309F495C90E9405BE8C01892BF5
:10BEB00011F00C94586883E50E9433BE882311F476
:10BEC0000C94ED670E9405BE8F3F980711F00C940B
:10BED000E66784E093E10E94FEC37BC98C32F1E007
:10BEE0009F0711F40C9469688D32914009F007C9DD
:10BEF00060E085E40E9414BF81110C947F6880E5A6
:10BF00000E9433BE882351F00E9409BE60937F12C5
:10BF100070938012809381129093821289E40E9420
:10BF200033BE882381F00E9409BE2CEA35EC47E23B
:10BF30005EE30F94F33260938312709384128093C4
:10BF400085129093861284E40E9433BE882381F088
:10BF50000E9409BE2CEA35EC47E25EE30F94573AA3
:10BF600060938712709388128093891290938A123B
:10BF70000E9418DC40917F125091801260918112D2
:10BF8000709182128EE498E00E94E5C92CEA35ECAB
:10BF900047E25EE360918312709184128091851272
:10BFA000909186120F94573AAB01BC018AE498E055
:10BFB0000E94E5C92CEA35EC47E25EE36091871206
:10BFC000709188128091891290918A120F94F332A5
:10BFD000AB01BC0186E498E00E94E5C98AE00E94BA
:10BFE0008CC7F7C8803931E0930711F40C941269BB
:10BFF00008F07DC08F32B1E09B0711F40C94CD683E
:10C000008033914009F07BC880E50E9433BE8823CD
:10C0100051F00E9409BE6093141270931512809320
:10C0200016129093171289E40E9433BE882381F080
:10C030000E9409BE2CEA35EC47E25EE30F94F3322E
:10C04000609318127093191280931A1290931B1216
:10C0500084E40E9433BE882381F00E9409BE2CEA4A
:10C0600035EC47E25EE30F94573A60931C127093ED
:10C070001D1280931E1290931F120E9418DC409193
:10C0800014125091151260911612709117128CE6CD
:10C0900098E00E94E5C92CEA35EC47E25EE3609146
:10C0A00018127091191280911A1290911B120F940C
:10C0B000573AAB01BC0188E698E00E94E5C92CEA3A
:10C0C00035EC47E25EE360911C1270911D12809185
:10C0D0001E1290911F120F94F332AB01BC0184E643
:10C0E00098E00E94E5C98AE00E948CC772C8813935
:10C0F000F1E09F0711F40C9416698239914011F018
:10C100000C947F580E949CB80E94A5B80E940B32E4
:10C1100060C88C3032E0930711F40C94B16A08F0D7
:10C1200068C08C3AB1E09B0711F40C94F06970F58B
:10C13000843AF1E09F0711F40C947369C8F48C39C8
:10C1400031E0930711F40C9420698D39914011F07E
:10C150000C947F5883E50E9433BE882311F40C941D
:10C16000166C0E94F5BD8093F0040E94B4BF31C8E4
:10C17000853AB1E09B0711F40C947769863A9140B7
:10C1800011F00C947F580E945DCE23C8863FF1E0E9
:10C190009F0711F40C94A36A70F4843F31E0930775
:10C1A00011F40C949F6A853F914011F00C947F58D4
:10C1B0000E9420B30EC8873FB1E09B0711F40C9496
:10C1C000A76A883F914011F00C947F5881E08093DA
:10C1D00015050E94FF2210921505882311F40C9476
:10C1E000E9580E9418DC86E799E00E94B4C70C94D5
:10C1F000E9588C36F3E09F0711F40C94E95808F0E5
:10C2000091C08D3B32E0930711F40C94DC6A08F086
:10C210007AC08835B2E09B0711F40C94C26A8B3562
:10C22000924011F00C947F580E940221082F87FF42
:10C2300002C00C94E95885E50E9433BE882369F159
:10C240000E9409BE4B015C01E02E002E000CFF088D
:10C2500020E030E0A9010F94BD3B87FF04C0B7FA8E
:10C26000B094B7F8B09420E030E84BE354E4C50153
:10C27000B4010F94BD3B970153E0220F331F5A9531
:10C28000E1F728513B4F181614F40C94C66AD901F3
:10C290008D929D92AD92BC9213978CE40E9433BE16
:10C2A000882311F40C94E9580E9409BE6B017C01AB
:10C2B000002E000C110B20E030E0A9010F94BD3BD3
:10C2C00087FF04C0F7FAF094F7F8F09420E030E824
:10C2D0004BE354E4C701B6010F94BD3B980143E022
:10C2E000220F331F4A95E1F728513B4F181614F4DB
:10C2F0000C94D16AD9011496CD92DD92ED92FC9204
:10C3000017970C94E9588E3BF2E09F0711F40C94B8
:10C31000E06A8335934011F00C947F580E94F553E6
:10C320000C94E958873E33E0930711F40C94066CA3
:10C33000C8F48438B3E09B0711F40C949B6B803AEB
:10C34000934011F00C947F582091A3043091A404E1
:10C350009091D01492609093D014C9010E944285AC
:10C360000C94E958883EF3E09F0711F40C94226C7A
:10C37000893E934011F00C947F588091C61481112E
:10C380000C94266C0E94ACBF0E9437850E94EA354F
:10C390006D3371058105910520F08CED99E00E94C7
:10C3A000826C88ED99E00E94826C84EE8093AF04E9
:10C3B00084EC99E00E94B4C780EC99E00E94826C02
:10C3C0000C94E95887EC96E00E9435375CCB80915D
:10C3D000520484FD18C08091540487FD14C08091DC
:10C3E0005504837081F460E08AED96E00E94EC3C95
:10C3F0005F988A9880910801817080930601479820
:10C4000012980C94E95888E50E9433BE81115F9818
:10C4100089E50E9433BE81118A988AE50E9433BE65
:10C42000882331F08091080181708093060147983C
:10C4300085E40E9433BE882311F40C94E9581298C5
:10C440000C94E9588091D01483FF25C082EF96E0C8
:10C450000E94B4C78091D01483FF17C080EF94E18D
:10C460000E94C7808BE1E0EFF4E1DE0111960190BC
:10C470000D928A95E1F770E060E0CE0101960E948E
:10C480007E86CE0101960E94D4BF83EE96E00E9484
:10C49000B4C70C94E9580E9418DC83E097E00E942E
:10C4A000B4C70C94E9580E9461800C94E9588091BB
:10C4B000A3049091A404FC012191222331F02032A5
:10C4C000D9F7DF0111971C92F7CF60E00E948B85AE
:10C4D0001092AF040C94E95883E50E9481BE882332
:10C4E00021F00E94D1BD0E94F15084E50E9481BEDE
:10C4F0008823A9F00E94D1BD6B017C010E941C36EB
:10C50000C092D204D092D304E092D404F092D50425
:10C51000CD28CE28CF2819F081E08093B3118091E7
:10C52000B2118823F9F080E090E0A0EAB1E48983B9
:10C530009A83AB83BC831C8E1D8E1E8E1F8E18A209
:10C5400019A21AA21BA210E000E020E0AE014F5F8A
:10C550005F4FBE01645E7F4FCE0180960E942FED3B
:10C560000C94E9580E94E3C3882381F00E943E782E
:10C570000E94E63883E998E00E94EF7F10921C0E3B
:10C5800010921D0E10921E0E10921F0E61E08DE390
:10C590009EE00E94C3C84AE25EE06DE077E085E07D
:10C5A0000E945DF30E944FF50C94E9588091D014DD
:10C5B00083FD02C00C94E95883E50E9481BE882364
:10C5C00011F40C94E9580E94D1BD0E94F1500C94D2
:10C5D000E95883E40E9433BE882361F183E297E047
:10C5E0000E94B4C7809137168823F9F0BE016F5FAF
:10C5F0007F4F84E396E10E94827FCE0101960E94E4
:10C60000347CCE0101960E940D8180912E128823E8
:10C6100039F080E20E948CC78EE292E10E94347C65
:10C620008AE00E948CC70C94E95889E197E00E9447
:10C63000B4C7F6CF83E50E9481BE882301F10E9432
:10C64000E1BD182F8C3308F08CE380932C040E94FA
:10C6500029746B017C01212F30E0A8EEB3E00F9428
:10C660002539C60ED71EE81EF91EC0922804D092A6
:10C670002904E0922A04F0922B040C94E9580E94B9
:10C68000FC770C94E9588091D0148E7F8093D0145D
:10C690000C94E9588091D01483FD02C00C94E958A1
:10C6A0000F94FF228091A3049091A4040E94CF8450
:10C6B0000C94E9588091D01482FD0E94D42380917B
:10C6C000D01483FD02C00C94E95860E080E50E941C
:10C6D00020BF182F682F8091A3049091A4040E947A
:10C6E0008B8583E50E9481BE882321F00E94D1BD05
:10C6F0000E94F1500E943E7811110C94E9580E945A
:10C70000E6380C94E9580E9430530C94E95880E5BF
:10C710000E9433BE882311F40C94E9580E94E1BDB5
:10C72000853608F084E68093AF040C94E9580E94A3
:10C73000E6380C94E9580E94F1C30C94E95870E073
:10C7400060E083E50E9405BF8E34910531F40E94BC
:10C7500043230E944FF50C94E9588DE997E00E941D
:10C76000B4C76091CA057091CB0584E997E00E9437
:10C77000D3C96091CC057091CD0587E897E00E9400
:10C78000D3C96091CA057091CB058091CC05909179
:10C79000CD05681B790B8091B311815021E030E009
:10C7A000823010F030E020E0621B730B8CE797E0E2
:10C7B0000E94D3C98AE00E948CC784E797E00E9458
:10C7C000B4C78091CE059091CF05A091D005B091CE
:10C7D000D1058C8F9D8FAE8FBF8FBE016F5F7F4F56
:10C7E000CE014C960E94601EBE016F5F7F4F87E6B0
:10C7F00097E00E940ADC8091D2059091D305A09128
:10C80000D405B091D5058C8F9D8FAE8FBF8FBE01A3
:10C810006F5F7F4FCE014C960E94601EBE016F5F1E
:10C820007F4F87E597E00E940ADC20E030E04AE78E
:10C8300054E46091D6057091D7058091D805909108
:10C84000D9050F94573AAB01BC018FE397E00E94E2
:10C85000E5C98DE60E948CC78AE00E948CC70C94C3
:10C86000E9588091850C83FF02C00C94E9580E941E
:10C870000221082F87FF02C00C94E95883E50E942B
:10C8800081BE182F882359F10E9405BE0E94A4235F
:10C8900061E081E00F948D2620917C1230917D1211
:10C8A00080917A1290917B1282179307F4F480EBB7
:10C8B00097E09F938F938BEB97E09F938F931F92BB
:10C8C0000F94E5220F94EC250F900F900F900F908E
:10C8D0000F90612F802F0E94058A0C94E95882E501
:10C8E0000E9481BE8111D0CFBEC985EA97E0112395
:10C8F00001F30F94EC25EDCF0E940221182F87FD44
:10C900000AC080EC97E00E94B4C7812F0E941B8868
:10C910008AE00E948CC73CA930933704E5960FB695
:10C92000F894DEBF0FBECDBFDF91CF911F910F9165
:10C93000FF90EF90DF90CF90BF90AF909F908F903F
:10C940007F906F905F904F903F902F90089560E0A0
:10C9500080E50E9414BFF82E81E08F1510F40C942E
:10C96000E95881E40E9433BE60914809062F811185
:10C9700002C00FEF10E083E50E9481BE882349F0DA
:10C980000E94D1BD8B016F3F710519F010F00FEFC0
:10C9900010E0EF2DF0E0E85BF64F00830C94E958CF
:10C9A00083E50E9433BE882331F060E083E50E9476
:10C9B00014BF8093850C0E9418DC81ED97E00E94E3
:10C9C000B4C78091850C882351F110E000E020E08D
:10C9D0008091850C90E0B0E0A0E0002E04C0B695F8
:10C9E000A795979587950A94D2F780FF12C0FF24E8
:10C9F000F394F20E222319F08CE20E948CC7F80106
:10CA0000EE0FFF1FE953F84F859194910E94B4C730
:10CA10002F2D0F5F1F4F05301105D1F601CE83EC8E
:10CA200097E005CE8CE3809300020C94E9580E94B5
:10CA300018DC6091000288ED97E00E94DDC98AE071
:10CA40000E948CC70C94E9588091850C83FF02C02A
:10CA50000C94E95883E50E9481BE182F8823E9F0E1
:10CA60000E9405BE0E9485BD60E081E00F948D2686
:10CA7000209111123091121280910F129091101288
:10CA8000821793078CF08FED97E060E00E94EC3CFA
:10CA9000812F0E948E880C94E95882E50E9481BE05
:10CAA0008111DECF0C94E9588EEE97E0EECF83E54E
:10CAB0000E9481BE882311F40C94E9580E94E1BDC4
:10CAC000182F8C3308F08CE3809331040E94297472
:10CAD0006B017C01212F30E0A8EEB3E00F942539E3
:10CAE000C60ED71EE81EF91EC0922D04D0922E0449
:10CAF000E0922F04F09230040C94E95880913708AA
:10CB00008F7D8061809337080C94E95880913708B5
:10CB10008F7E8062809337080C94E95883E50E94E9
:10CB200033BE882311F40C94E9580E942974609351
:10CB300005127093061280930712909308120E94B8
:10CB400009BE20E030E04AE754E40F94F3320F943A
:10CB5000D03A6093320470933304809334049093FA
:10CB600035040C94E9580E94022187FF02C00C94FE
:10CB7000E9588091520484FD09C08091540487FDD6
:10CB800005C080915504837009F489C02AEEC22E35
:10CB900022E0D22E3DECE32E3CE0F32E10E0D60155
:10CBA0008D916D010E9481BE882309F465C0133008
:10CBB00009F06DC00E9409BE4B015C0120E030E02D
:10CBC00040EA51E40F948D3287FF4EC0A5019401D5
:10CBD0006091ED0C7091EE0C8091EF0C9091F00C47
:10CBE0000F94573A2B013C01AC019B016091400925
:10CBF0007091410980914209909143090F94F33259
:10CC000060934009709341098093420990934309CE
:10CC1000A30192016091FD0C7091FE0C8091FF0CBC
:10CC20009091000D0F94F3326093FD0C7093FE0C05
:10CC30008093FF0C9093000D60912C0970912D0949
:10CC400080912E0990912F090F949232A3019201A5
:10CC50000F94F3320F94D03A60932C0970932D09FE
:10CC600080932E0990932F098092ED0C9092EE0CF8
:10CC7000A092EF0CB092F00C1F5FF4E0EF0EF11CED
:10CC8000143009F08CCF0E94B0230C94E9580E9414
:10CC900009BEF701648B758B868B978BEDCF81E096
:10CCA0000F948C220C94E9580F941D208AE293E192
:10CCB0000E94A1970C94E9580E948D1D0C94E9588C
:10CCC0000E944FF50C94E9580091A3041091A4041C
:10CCD00094E0F12C40E09150F9F0F8018081282F88
:10CCE0002B7F213499F421812133B1F4813411F166
:10CCF000853409F441E098012E5F3F4F89012F5F91
:10CD00003F4FF80180818032C9F3E5CF803521F4AF
:10CD1000818180538A3078F341110E9418DCFF2012
:10CD200021F08FE098E00E94B4C7C8010E94CB5266
:10CD30000C94E958FF24F394DECF0E943F1F0C941B
:10CD4000E9581092DB051092DA050E9474330C94B6
:10CD5000E95880E06BC80E94022187FF02C00C9452
:10CD6000E9580AEE12E08DECE82E8CE0F82E9EEEEB
:10CD7000C92E92E0D92ED8018D918D010E9433BE2B
:10CD8000882359F00E9409BE0F94D03AF7016083BE
:10CD90007183828393830E94BA1CF4E0EF0EF11C2E
:10CDA000C016D10641F70C94E9580E94022187FF72
:10CDB00002C00C94E9581AEEE12E12E0F12E10E0B8
:10CDC00000E0D7018D917D010E9433BE882349F098
:10CDD0000E9409BEF801E353F34F64A375A386A331
:10CDE00097A30C5F1F4F0031110559F70C94E958B8
:10CDF0000E94C2C70C94E958B9E4EB2EB8E0FB2EB0
:10CE000010E088E5810F0E9433BE882351F00E9414
:10CE100009BEF7016083718382839383812F0E940F
:10CE2000081D1F5FF4E0EF0EF11C133051F78091E5
:10CE3000540487FF02C00C94E0588091550483701D
:10CE400011F00C94E0584091490850914A086091C3
:10CE50004B0870914C0882E198E00E94E5C940912E
:10CE60004D0850914E0860914F08709150088AE625
:10CE700091E30E94E5C94091510850915208609198
:10CE800053087091540887E691E30E94E5C98AE04F
:10CE90000E948CC70C94E95882E40E9433BE882318
:10CEA00041F080917F0290918002909302028093E2
:10CEB000010282E50E9433BE882341F08091010285
:10CEC000909102029093800280937F0283E50E94FA
:10CED00081BE882331F00E9405BE9093800280932A
:10CEE0007F028091520490915304A0915404B09118
:10CEF0005504892B8A2B8B2B11F00C94E9586091E7
:10CF00007F027091800289E198E00E947BCA85E2ED
:10CF10000E948CC78AE00E948CC70C94E9580E943A
:10CF20000221082F87FF02C00C94E95883E50E9474
:10CF300081BE002E000C110B7801EE0CFF1C882323
:10CF400059F10E9405BEF701E358FD4F918380839C
:10CF5000000F111F000F111F980127583D4F790135
:10CF6000BC01990F880B990B0F9494322AE037ED8E
:10CF700043E25CE30F94F3320753134FD8012D9132
:10CF80003D914D915C910F94F332F7016083718371
:10CF9000828393830C94E9580E9418DC85E40E94F4
:10CFA0008CC780E3800F0E948CC7F701E358FD4FC8
:10CFB000608171818DE198E00E947BCA85E20E94C8
:10CFC0008CC78AE00E948CC70C94E958BC0184E0AD
:10CFD00093E10E946CC40C94E9580E9418DC70E044
:10CFE00060E088E298E00E947BCA8091061358E5D1
:10CFF000C52E52E0D52EC81AD10887FDD394CC0C8B
:10D00000DD1CCC0CDD1C0D2C000CEE08FF08809103
:10D01000051378E8872E912C881A910887FD939440
:10D02000880C991C880C991C092C000CAA08BB08B8
:10D030008091041390E08F3FC9F1FC01EE0FFF1FB8
:10D04000E80FF91FE554FD4E8181928133E0880F8E
:10D05000991F3A95E1F7B0E0A0E044E0B595A795B7
:10D06000979587954A95D1F702969C012F5F3F4F80
:10D07000032E000C440B550B281939094A095B098A
:10D08000A4EBB0E00F941239A701960128193909D1
:10D090004A095B090F94F338B90185E298E00E94D0
:10D0A0007BCA8AE00E948CC70C94E95880E0DDCFEF
:10D0B0000E9414DCB8018FE398E00E947BCA80E3F1
:10D0C00098E00E94B4C70C94E9580E9437550C941C
:10D0D000E95864E071E083E50E94C71F8C0168EEA7
:10D0E00073E080E50E94C71F893823E1920710F0A2
:10D0F00088E893E1B8010E945A3A0C94E9580E94DA
:10D1000014DC82E598E00E94B4C70C94E95883E5EA
:10D110000E9433BE182F882369F00E9405BE9C012F
:10D12000909368028093670291E0232B09F090E0CE
:10D1300090934A0980E50E9433BE882361F02091D4
:10D14000670230916802232B11F00E94F5BD809395
:10D150004A090C94E95811110C94E9580E9418DC02
:10D160008CE898E00E94B4C780914A09882391F026
:10D1700084E798E00E94B4C76091670270916802EA
:10D180008BE798E00E947BCA87E798E00E94B4C7CB
:10D190000C94E95880E798E0EDCF70E060E085E41A
:10D1A0000E9405BFF82E3FEF8317C9F1882341F095
:10D1B0008CEA98E00E94B4C70E9466F30C94E95888
:10D1C00004EB10E083E50E9481BE882319F00E94E1
:10D1D00005BE8C0165E070E083E40E9405BFE82E87
:10D1E00060E085E50E9420BFD82E60E08FE998E0DE
:10D1F0000E94EC3CB801110F880B990B0F949432EC
:10D2000069837A838B839C832D2D4E2D6F2DCE01C8
:10D2100001960E94D6A60E944FF50C94E95806E4A8
:10D2200010E0D0CF0E94D4230C94E9588091C70716
:10D2300081110C94E05881E00E9483330C94E058F3
:10D24000809152048878F9F4809154048670D9F45E
:10D250000E9418DC80EF98E00E94B4C780910F0212
:10D260000E94C7C940910B0250910C0260910D02BF
:10D2700070910E0280ED98E00E94E5C98AE00E945C
:10D280008CC70C94E95888E40E9433BE882321F0AF
:10D290000E94F5BD8093360482E50E9433BE082FBC
:10D2A00083E50E9433BE182F011102C0882341F08C
:10D2B0000E9498C3112321F00E94F5BD80930F02B4
:10D2C00084E40E9433BE882311F40C94E9580E9430
:10D2D00009BE60930B0270930C0280930D02909331
:10D2E0000E020C94E9580E941CDC0C94E9586FEF74
:10D2F0007FEF89E40E9405BF082F6FEF7FEF8AE47C
:10D300000E9405BF182F8AE50E9481BED12C811191
:10D3100007C081E50E9481BED82E882309F4B8C2D7
:10D32000C02E81E0800F863008F052C0912E81E03F
:10D33000810F863008F04CC00E9409BE2B013C01D1
:10D34000F02E07FDF12C07FF02C004E0C02E812E55
:10D3500017FD812C17FF02C014E0912EB5E03B2E83
:10D36000CF1410F40C94E958E82C3F9C5001112480
:10D370009E1460F10E2D10E020E030E0A901DD20C8
:10D3800069F0F501E00FF11FEE0FFF1FEE0FFF1F19
:10D39000ED52F84F20813181428153810A0D1B1DCE
:10D3A000000F111F000F111F0D52184FC301B201C2
:10D3B0000F945D39D8016D937D938D939C93139752
:10D3C0006E2D8F2D0F94BA21E394D2CFF394C8CF52
:10D3D0000E9414DC81E299E00E94B4C70C94E958E1
:10D3E00087E00E94DC5281110C94E95876E3C72E45
:10D3F0007FE0D72EE9E6F2E0F9A7E8A79E012F5FCC
:10D400003F4F1901790110E000E0C6010E9496B873
:10D41000A8A5B9A58D909D90AD90BD90B9A7A8A7DE
:10D42000A50194010F945C392B013C01F701408266
:10D4300051826282738220E030E040EA51EC0F9426
:10D44000BD3B87FD0AC020E030E040EA51E4C30163
:10D45000B2010F948D32181684F4F801E65AF04F99
:10D46000E4911E1654F4B7FAB094B7F8B094D7010B
:10D470008D929D92AD92BC921397F70181909190FD
:10D48000A190B1907F0120E030E040EA51ECC5016D
:10D49000B4010F94BD3B87FD3FC020E030E040EA7F
:10D4A00051E4C501B4010F948D321816ACF10F5F31
:10D4B0001F4FF4E0CF0ED11C0330110509F0A5CFAA
:10D4C00069E4E62E68E0F62E10E0F1018191919179
:10D4D000A191B1911F01F70181939193A193B19310
:10D4E0007F01812F0E94081D1F5F133071F70E947A
:10D4F0000B3260E08AE399E00E94EC3C63E972E061
:10D5000084E690E00E945A3A6AEB72E084E690E08A
:10D510000E945A3A0C94E9580E9414DC88E599E07C
:10D520000E94B4C761E08AE499E00E94EC3C68E2A2
:10D5300070E088EC90E00E945A3A0C94E9580E94FE
:10D54000363D0C94E9580E943DA50C94E95861E0E1
:10D5500083E50E9420BF91E089270E94EAAB0C94EA
:10D56000E9588091D01482FF05C080648093D01464
:10D570000C94E95883FD02C00C94E9580F94FF22E3
:10D580000C94E9580E9427210C94E95880E090E817
:10D59000ABE3B4E4F90180839183A283B3830C9459
:10D5A0004D6180E090E8ABE3B4E4F90184839583B6
:10D5B000A683B7830C94E9580E94D82E0C94E9589E
:10D5C0000E940221182F87FF02C00C94E9588AE5B7
:10D5D0000E9481BE812C912C90E2A92E91E4B92E5B
:10D5E000882379F040E050E0BA018AE50E94EEBE5F
:10D5F0004B015C0120E030E0A9010F94BD3B1816FF
:10D600007CF580E090E0A0EAB0E489839A83AB8364
:10D61000BC8320917102309172024091730250914B
:10D620007402C501B4010F945D396B017C0120E0E7
:10D6300030E048EC53E40F948D3287FD06C0C12CD6
:10D64000D12C88ECE82E83E4F82ECC8EDD8EEE8E85
:10D65000FF8EBE016F5F7F4FCE014C960E94B530AA
:10D6600085E50E9433BE882309F45AC00E9409BE92
:10D670006B017C0120E030E0A901C701B6010F94E5
:10D68000BD3B87FF04C0F7FAF094F7F8F094F7FA7F
:10D69000F094F7F8F094C982DA82EB82FC8280E0A1
:10D6A0000E94CEEC882321F0CE0101960E9408C38F
:10D6B00020E030E0A901C501B4010F94BD3B18166C
:10D6C00014F00C94E95880E090E0A0EAB0E489837B
:10D6D0009A83AB83BC83A501940160917102709120
:10D6E000720280917302909174020F945C396B0105
:10D6F0007C0120E030E0A9010F94BD3B18161CF01E
:10D70000C12CD12C7601CC8EDD8EEE8EFF8EBE012B
:10D710006F5F7F4FCE014C960E94B5300C94E95854
:10D7200028E01202F0011124E851FB4FC080D180A3
:10D73000E280F3809FCFA0904409B0904509C0904B
:10D740004609D09047098BE40E9481BE882339F1B5
:10D750000E9409BE7B018C0120E030E0A9010F94FA
:10D76000BD3B87FD0AC020E030E040E251E4B70154
:10D77000C8010F948D321816A4F48FE30E948CC751
:10D780008BE40E948CC78CE899E00E94B4C784E8BF
:10D7900099E00E94B4C781E899E00E94B4C775017E
:10D7A00086019701A801B501C6010F948D32882327
:10D7B00061F00E94D423C701D8018093440990935B
:10D7C0004509A0934609B09347098091520490916E
:10D7D0005304A0915404B0915504892B8A2B8B2BB0
:10D7E00011F00C94E9580E9418DC409144095091C2
:10D7F0004509609146097091470980EA99E00E94C5
:10D80000E5C98AE00E948CC70C94E95881E08093B6
:10D810001F061092F41160E083E50E9420BF811181
:10D820000C94E9580E942FF80C94E9580E9418DCD7
:10D830008BEA99E00E94B4C78091F0040E94C7C9A6
:10D840000C94E9580E94F46C0C94E9580E943884B6
:10D8500081110C94E9580C94C2611091A0040E94AB
:10D8600029746093051270930612809307129093A7
:10D870000812112311F40C94E958812F0E94658736
:10D880000C94E95811110C948A5911E00C948459A4
:10D890000E9414DC81E099E00E94B4C70C94E9581E
:10D8A000882399F30C948D59DF92EF92FF920F9396
:10D8B0001F93CF93DF93EC01E090C907F090CA0764
:10D8C0008AE0D82E6AE070E0CE010F94AB3C8C0168
:10D8D000009711F0FC011082CE010E94535181E0AB
:10D8E0000E94C1560115110519F0E801D992EACF3D
:10D8F000C701DF91CF911F910F91FF90EF90DF90C3
:10D900000C9453514F925F926F927F928F929F929D
:10D91000AF92BF92CF92DF92EF92FF920F931F933D
:10D92000CF93DF93CDB7DEB77C014DB65EB6609086
:10D93000C9077090CA078DB69EB66AE070E0C7014D
:10D940000F94C8316C018C010E191F09892B21F429
:10D95000C7010F94DA318C01C80101962DB73EB78B
:10D96000281B390B0FB6F8943EBF0FBE2DBF8DB7E5
:10D970009EB701965C01A801B7010F94FB31F50138
:10D98000E00FF11F1082C5010E94535181E00E94F7
:10D99000C156C114D10451F076019FEFE91AF90A7A
:10D9A0000FB6F8949EBE0FBE8DBEC5CF0FB6F894CD
:10D9B0009EBE0FBE8DBEC3010E9453510FB6F89498
:10D9C0005EBE0FBE4DBEDF91CF911F910F91FF90B4
:10D9D000EF90DF90CF90BF90AF909F908F907F900F
:10D9E0006F905F904F9008954F925F926F927F92E9
:10D9F0008F929F92AF92BF92CF92DF92EF92FF925F
:10DA00000F931F93CF93DF93CDB7DEB7C059D109E2
:10DA10000FB6F894DEBF0FBECDBF0E94C2BF8823F1
:10DA2000B9F183E50E9433BE882309F449C088E92F
:10DA300094E00E94B4C78AE00E948CC78EEF809366
:10DA4000AC0481E0809386021092AB0481E09AE5F9
:10DA500090936714809366148CE490E0909369141B
:10DA60008093681487E080935A1482E880935D1451
:10DA700084E890E0A0E0B0E080935E1490935F149F
:10DA8000A0936014B09361148AE094E10E941C3862
:10DA9000C057DF4F0FB6F894DEBF0FBECDBFDF918A
:10DAA000CF911F910F91FF90EF90DF90CF90BF909B
:10DAB000AF909F908F907F906F905F904F90089560
:10DAC00083E40E9433BE882349F00E94ACBF0E94C9
:10DAD00037850E948C840E94BE40DACF8090FC087B
:10DAE0009090FD08A090FE08B090FF088091050975
:10DAF00080FF05C09091850C98609093850C869569
:10DB0000817080934A0982E495E00E94826C809142
:10DB10008B0890918C089E012F5F3F4F79010097F1
:10DB200099F09F938F9389E395E09F938F933F9311
:10DB30002F930F942432C7010E94546C0F900F90C2
:10DB40000F900F900F900F908091890890918A0804
:10DB5000009799F09F938F9380E395E09F938F9325
:10DB6000FF92EF920F942432C7010E94546C0F90E1
:10DB70000F900F900F900F900F906E0131E8C30E31
:10DB8000D11C609168087091690880916A08909131
:10DB90006B08860123E041E00F945A2D9F938F93E9
:10DBA0008EE195E09F938F93FF92EF920F94243232
:10DBB000C7010E94546C86E195E00E94826C87E068
:10DBC0008093C70C80939A040F900F900F900F9042
:10DBD0000F900F90809184088823F9F06091850858
:10DBE00070918608809187089091880823E041E031
:10DBF0000F945A2D9F938F938DE095E09F938F9371
:10DC0000FF92EF920F942432C7010E94546C0F9040
:10DC10000F900F900F900F900F9080918D08882398
:10DC2000A1F01F928F931F921F9280E095E09F9327
:10DC30008F93FF92EF920F942432C7010E94546C8D
:10DC40000FB6F894DEBF0FBECDBF80918E0888233B
:10DC5000A9F01F928F931F9281E08F9380E095E04F
:10DC60009F938F93FF92EF920F942432C7010E94EB
:10DC7000546C0FB6F894DEBF0FBECDBF40908F0836
:10DC800050909008609091087090920820E030E0E9
:10DC9000A901C301B2010F948D32811104C080919A
:10DCA000050982FF20C0860121E041E0C301B201E5
:10DCB0000F945A2D9F938F938091050982FB88279B
:10DCC00080F91F928F9383EF94E09F938F93FF923D
:10DCD000EF920F942432C7010E94546C0FB6F8944F
:10DCE000DEBF0FBECDBF60915A0870915B08809176
:10DCF0005C0890915D088E010F581F4F23E041E0B2
:10DD00000F945A2D782E692E6091560870915708FD
:10DD10008091580890915908860123E041E00F94C2
:10DD20005A2D6F927F929F938F9382EE94E09F93F0
:10DD30008F93FF92EF920F942432C7010E94546C8C
:10DD400060915E0870915F08809160089091610811
:10DD500023E041E00F945A2D87ED94E00E94826CFD
:10DD6000DF92CF928DEC94E09F938F93FF92EF928E
:10DD70000F942432C7010E94546C809167088F93DE
:10DD8000809166088F9386EC94E09F938F93FF9227
:10DD9000EF920F942432C7010E94546C6091620884
:10DDA00070916308809164089091650823E041E0D8
:10DDB0000F945A2D9F938F938CEB94E09F938F93A6
:10DDC000FF92EF920F942432C7010E94546C8CE0B2
:10DDD000ECE6F8E0A9E4B8E001900D928A95E1F74D
:10DDE0008CE0E8E7F8E0ADE3B8E001900D928A95A9
:10DDF000E1F780E00E94081D81E00E94081D82E09A
:10DE00000E94081D809104098093370881E0809367
:10DE1000F0040E94B4BF83E998E09F938F938BE056
:10DE200091E29F938F93FF92EF920F9424320FB65B
:10DE3000F894DEBF0FBECDBFC7010E94546C809125
:10DE400003098F93809102098F93809101098F9329
:10DE5000809100098F93BF92AF929F928F928EEA2A
:10DE600094E09F938F93FF92EF920F942432C70117
:10DE70000E94546C0FB6F894DEBF0FBECDBF08CE23
:10DE8000CF93DF93C091210EC0931F0981E6C89FF5
:10DE9000E0011124CD5DD14F8091850C80FF05C03C
:10DEA0000E9418DCCE010E94CB52CE010E94535139
:10DEB00080E0DF91CF910C94C1563FB7F8948091E8
:10DEC000AE069091AF06A091B006B091B10626B50E
:10DED000A89B05C02F3F19F00196A11DB11D3FBFA2
:10DEE000BA2FA92F982F8827BC01CD01620F711D71
:10DEF000811D911D42E0660F771F881F991F4A956B
:10DF0000D1F708958BE1E0EFF4E1ABE0B5E10190EA
:10DF10000D928A95E1F78091D01480628093D0149D
:10DF20000895CF938091AF11C1E08823C9F080910B
:10DF3000B0119091B1114091A7115091A811609129
:10DF4000A9117091AA11DC01ED91FC910288F3896D
:10DF5000E02D27EA3FE01995C82F811104C0C0E0E9
:10DF60008C2FCF9108954091AB115091AC116091DD
:10DF7000AD117091AE114115510561057105B9F0F2
:10DF80008091B0119091B111DC01ED91FC9102886A
:10DF9000F389E02D27EA3FE01995882301F31092D9
:10DFA000AB111092AC111092AD111092AE111092F3
:10DFB000AF11D6CF0F931F93CF93DF93CDB7DEB7BB
:10DFC00060970FB6F894DEBF0FBECDBF8C01DC01A9
:10DFD000ED91FC910280F381E02DBE016F5F7F4FD8
:10DFE0001995882309F464C08981807CC9F56F8103
:10DFF000637070E0762F6627770F770F8885B4E01F
:10E000008B9FC0011124682B792B89858295869579
:10E0100086958370682B6F5F7F4F90E080E02A8544
:10E020002370220F3B8537FB332730F9232B3E81AA
:10E030003F70230F3327331F2750310904C0660F69
:10E04000771F881F991F2A95D2F760960FB6F8940C
:10E05000DEBF0FBECDBFDF91CF911F910F9108950D
:10E06000803419F568856695669570E090E080E0EB
:10E07000CB01772766272A85622B098510E0102FB0
:10E080000027012E000C220B330B602B712B822BEF
:10E09000932B6F5F7F4F8F4F9F4F4AE0660F771F25
:10E0A000881F991F4A95D1F7D0CF8BE0F801848360
:10E0B00060E070E0CB01C9CF0895FC018281089532
:10E0C0004F925F926F927F928F929F92AF92BF9288
:10E0D000EF92FF920F931F93CF93DF93B0E2A0E0F4
:10E0E0006A2F70E0AB014B0F511D559547954111BB
:10E0F00017C0E6E9FFE185919491282F822FDF91E7
:10E10000CF911F910F91FF90EF90BF90AF909F9094
:10E110008F907F906F905F904F900895B42FE2CFD3
:10E12000A41711F0B41303C0E2E1F0E2E4CF9A01C6
:10E1300021503109220F331F220F331FF901EC56F2
:10E14000F04EE590F490F901E856F04E05911491E7
:10E150008E159F051CF3A42F081719070CF4C0CFC8
:10E16000BC01F901EA56F04EC591D491F901E65689
:10E17000F04EA590B4906E197F09072E000C880B05
:10E18000990B0F9494322B013C01B5016C1B7D0B54
:10E19000072E000C880B990B0F9494329B01AC0155
:10E1A000C301B2010F94F3324B015C01B8016E1947
:10E1B0007F09072E000C880B990B0F9494329B015A
:10E1C000AC01C501B4010F94573A4B015C01BE018B
:10E1D000DD0F880B990B0F9494329B01AC01C501A4
:10E1E000B4010F945D390F94C93A262F972F86CF2B
:10E1F000EF92FF920F931F93E0921905F0921A0588
:10E2000000931B0510931C0560932405709325054E
:10E21000809326059FEFFF27621B730B840B30F45E
:10E22000809570956195790B890B99279093BE061F
:10E23000A6E06A9F0092B206512DEE277A9F500DFC
:10E24000E11D8A9FE00D5093B306E093B406AFE062
:10E250006A9F0092B606512DEE277A9F500DE11D60
:10E260008A9FE00D5093B706E093B806AAE06A9F34
:10E270000092BA06512DEE277A9F500DE11D8A9F1C
:10E28000E00D5093BB06E093BC061F910F91FF90E9
:10E29000EF90089500000000000000008091DC0570
:10E2A00080FF21C089988FEF809320068091DC0544
:10E2B000869580FF1BC08F988FEF809321068091F9
:10E2C000DC058695869580FF14C080910B018270D5
:10E2D0008093090143988FEF80932206000000008D
:10E2E000000000000895899A81E0DECF8F9A81E0D6
:10E2F000E4CF80910B018095827080930901439A4D
:10E3000081E0EACF0F931F93CF93811113C0C42FE5
:10E310008B010E9418DC87ED92E10E94B4C7C8010E
:10E320000E94B4C7CC2331F08AE0CF911F910F91A6
:10E330000C948CC7CF911F910F9108950F9300916A
:10E34000150521E0022726E135E04CE050E0BC0154
:10E3500086EE94E00E940DC40F9108950F930091F2
:10E36000150521E0022726E135E044E050E0BC013C
:10E3700086EE94E00E940DC40F9108950F930091D2
:10E38000150521E0022726E135E041E050E0BC011F
:10E3900086EE94E00E940DC40F9108950F930091B2
:10E3A000150521E0022726E135E042E050E0BC01FE
:10E3B00086EE94E00E940DC40F9108950F93009192
:10E3C000150521E0022726E135E041E050E0BC01DF
:10E3D00086EE94E00E940DC40F9108950F93009172
:10E3E000150521E0022726E135E048E050E0BC01B8
:10E3F00086EE94E00E940DC40F9108950F93009152
:10E40000150521E0022726E135E04CE050E0BC0193
:10E4100086EE94E00E940DC40F9108950F9301E0E1
:10E4200026E135E041E050E0BC0186EE94E00E9438
:10E430000DC40F910895CF93DF93C6E7D2E18A818F
:10E440009B810F94851F9D838C83CBE0D2E18A81D1
:10E450009B810E9460709D838C83A8951092A0067A
:10E46000DF91CF9108951F93CF93DF93182FEB0186
:10E470000E9418DC8AE292E20E94B4C786E192E22E
:10E48000113011F48CE192E20E94B4C7BE0182E225
:10E4900092E20E940ADC8AE0DF91CF911F910C94F6
:10E4A0008CC7282F30E0F901E058FC4D9491F90118
:10E4B000E658F94C44912C5C394CF9012491222303
:10E4C00009F435C0992311F191509231F8F4E92FF4
:10E4D000F0E08827E159FD488F4F0D945439A07220
:10E4E000A472817298729C728672A772AD72B172B8
:10E4F000B772BB72BF72C572C9728672CD72D372A7
:10E50000D772809180008F7780938000E22FF0E0B7
:10E51000EE0FFF1FE050FA4CA591B4918FB7F8941D
:10E52000EC91611148C040954E234C938FBF0895E4
:10E53000809180008F7DE8CF80918000877FE4CF3D
:10E5400084B58F7784BDE2CF84B58F7DFBCF80917A
:10E55000B0008F778093B000D9CF8091B0008F7DCD
:10E56000F9CF809190008F7780939000CFCF8091EA
:10E5700090008F7DF9CF80919000877FF5CF8091BB
:10E58000A0008F778093A000C1CF8091A0008F7DE5
:10E59000F9CF8091A000877FF5CF809120018F7700
:10E5A00080932001B3CF809120018F7DF9CF80919E
:10E5B0002001877FF5CF4E2BB8CFCF93DF93EC01AF
:10E5C0008D810E94EAF060E08B81DF91CF910C9405
:10E5D000517261E0FC0183810E9451728FEF0C94B3
:10E5E000DEF0CF93DF93EC016EBDFA01CA019E5FAE
:10E5F0000DB407FEFDCF20812EBD0DB407FEFDCF6B
:10E6000021812EBD3296E817F90791F70DB407FE68
:10E61000FDCF8FEF0E94DEF08FEF0E94DEF00E94B0
:10E62000E3F08E838F71853049F083E18C83CE01D6
:10E630000E94E97280E0DF91CF91089581E0FBCFE5
:10E640001F93CF93DF93182FEB010E94E7F72097DA
:10E6500039F460E0812FDF91CF911F910C945172BA
:10E66000CF3FD10511F461E0F5CFE12FF0E0E058A4
:10E67000FC4DE491E150E23108F0B3C0F0E08827AE
:10E68000EB5BFC488F4F0D94543957735F73647381
:10E690006E737873F17382738A7392739C73A6732B
:10E6A000B073BF73C973F173D373DD73E77384B54C
:10E6B000806884BDC7BDDF91CF911F91089584B557
:10E6C000806284BDC8BDF7CF809180008068809350
:10E6D0008000D0938900C0938800EDCF80918000A6
:10E6E000806280938000D0938B00C0938A00E3CF38
:10E6F00080918000886080938000D0938D00C093CB
:10E700008C00D9CF8091B00080688093B000C09316
:10E71000B300D1CF8091B00080628093B000C093ED
:10E72000B400C9CF80919000806880939000D0930E
:10E730009900C0939800BFCF809190008062809331
:10E740009000D0939B00C0939A00B5CF8091900029
:10E75000886080939000D0939D00C0939C00ABCFC5
:10E760008091A00080688093A0008091A0008F7BA2
:10E770008093A000D093A900C093A8009CCF809163
:10E78000A00080628093A000D093AB00C093AA0049
:10E7900092CF8091A00088608093A000D093AD00BC
:10E7A000C093AC0088CF80912001806880932001C5
:10E7B000D0932901C09328017ECF809120018062EF
:10E7C00080932001D0932B01C0932A0174CF8091B4
:10E7D0002001886080932001D0932D01C0932C01EB
:10E7E0006ACFC038D1050CF03ECF33CF8F929F92C5
:10E7F000AF92BF92CF92DF92EF92FF926B017C01BA
:10E800000E945D6F4B015C01C114D104E104F1046D
:10E81000B9F00E945D6F681979098A099B09683E01
:10E8200073408105910580F321E0C21AD108E10807
:10E83000F10888EE880E83E0981EA11CB11CE4CF7D
:10E84000FF90EF90DF90CF90BF90AF909F908F9010
:10E8500008952FB7F8946091AA067091AB06809145
:10E86000AC069091AD062FBF0895CF92DF92EF9244
:10E87000FF920E9429746B017C0128E5C20E22E000
:10E88000D21EE11CF11C0E94E3F08F3F71F00E9448
:10E8900029746C197D098E099F0997FDF4CF80E0DA
:10E8A000FF90EF90DF90CF90089581E0F9CF0F9324
:10E8B0001F93CF938C010E94DD720E943574C82F84
:10E8C000882371F08DEF0E94DEF00E943574C82F0E
:10E8D000C8010E94E9728C2FCF911F910F9108956A
:10E8E00082E1F8018483F4CF0F931F93CF93DF93DA
:10E8F000EC018B010E94DD720E94357481110CC005
:10E9000085E18C8310E0CE010E94E972812FDF91B6
:10E91000CF911F910F910895A8016CEFCE010E9435
:10E92000F172182F882361F3EECFDF92EF92FF92FE
:10E930000F931F93CF93DF938C01C62FD22FF32E0B
:10E94000E42ED52E0E94DD720E9435748C2F8064D7
:10E950000E94DEF08D2D0E94DEF08E2D0E94DEF0F2
:10E960008F2D0E94DEF08D2F0E94DEF087E8C1110E
:10E9700001C085E90E94DEF0CC3011F40E94E3F082
:10E98000C0E00E94E3F0F801868387FF04C0CF3F18
:10E9900011F0CF5FF6CFDF91CF911F910F91FF90D4
:10E9A000EF90DF9008958F929F92AF92BF92CF9297
:10E9B000DF92EF92FF920F931F93CF93DF93EC01BF
:10E9C0006A017B01590120E030E0A90167E30E9460
:10E9D0009574A501980167E1CE010E94957481119B
:10E9E00027C08F81833039F089E0CC0CDD1CEE1C10
:10E9F000FF1C8A95D1F7A701960169E1CE010E941B
:10EA0000957411E0882319F010E087E08C83CE0123
:10EA10000E94E972812FDF91CF911F910F91FF909A
:10EA2000EF90DF90CF90BF90AF909F908F90089520
:10EA300089E08C8310E0EBCF0F931F93CF93DF938C
:10EA4000EC0189018F81833039F089E0440F551F33
:10EA5000661F771F8A95D1F79A01AB0168E1CE0155
:10EA60000E94957481112AC0A8016EEFCE010E9408
:10EA7000F172182F8823B1F00E943574182F882363
:10EA8000D1F020E030E0A9016DE0CE010E94957444
:10EA9000882321F086E18C8310E004C00E94E3F01B
:10EAA0008111F8CFCE010E94E972812FDF91CF91C1
:10EAB0001F910F91089587E18C83F4CF86E0EBCF0F
:10EAC0001F93CF93DF93EC010E94DD7220E030E0D2
:10EAD000A9016CE0CE010E94957411E0882319F021
:10EAE00010E083E08C83CE010E94E972812FDF91D8
:10EAF000CF911F9108951F93CF93DF93EC018F81E6
:10EB0000833039F089E0440F551F661F771F8A95BF
:10EB1000D1F79A01AB0162E1CE010E94957411E038
:10EB2000882319F010E085E08C83CE010E94E97201
:10EB3000812FDF91CF911F9108958F929F92AF9275
:10EB4000BF92EF92FF920F931F93CF93DF938C01AD
:10EB5000EB017A010E9429744B015C012CE2820EC8
:10EB600021E0921EA11CB11C0E94E3F0F8018683F3
:10EB70008F3F69F40E942974681979098A099B09F1
:10EB800097FDF2CF81E1F8018483C0E021C08E3F80
:10EB900071F5F1E0EF1AF1088FEF8EBDFE012FEF56
:10EBA0000DB407FEFDCF8EB581932EBDCF018C1B1A
:10EBB0009D0B8E159F05A0F30DB407FEFDCF8EB5FE
:10EBC000CE0DDF1D88830E94E3F00E94E3F0C1E0D8
:10EBD000C8010E94E9728C2FDF91CF911F910F9194
:10EBE000FF90EF90BF90AF909F908F9008958FE02F
:10EBF000CACF0F931F93CF93DF93EC018B010E9439
:10EC0000DD7240E052E0B801CE01DF91CF911F915B
:10EC10000F910C949D750F931F93CF93DF93EC018D
:10EC200089018F81833039F089E0440F551F661FB9
:10EC3000771F8A95D1F79A01AB0161E1CE010E945D
:10EC4000957481110AC040E052E0B801CE01DF9115
:10EC5000CF911F910F910C949D7584E08C83CE0110
:10EC60000E94E97280E0DF91CF911F910F9108958A
:10EC70000F931F93CF93DF93EC018B0120E030E0E3
:10EC8000A90169E00E94957481110AC040E150E039
:10EC9000B801CE01DF91CF911F910F910C949D751A
:10ECA00080E18C83CE010E94E97280E0DF91CF91F8
:10ECB0001F910F9108958F929F92AF92BF92CF9222
:10ECC000DF92EF92FF920F931F93CF93DF93EC01AC
:10ECD000162F1F821C824B830E9429746B017C01BA
:10ECE00020EDC20E27E0D21EE11CF11CA89561E0C8
:10ECF0008B810E9451728B810E94E7F7209A289A9B
:10ED0000219A2398229A81E00E94EAF085E08D837F
:10ED10000E94EAF00AE08FEF0E94DEF00150D9F77E
:10ED2000A89520E030E0A90160E0CE010E94957432
:10ED30008E83813081F00E9429746C197D098E09BF
:10ED40009F0997FDEECF81E08C83CE010E94E9728E
:10ED50001A8280E06AC0A8952AEA31E040E050E0DB
:10ED600068E0CE010E949574853041F581E08F8383
:10ED7000A8958F81812C912C5401823029F4812C0B
:10ED8000912CA12C80E4B82E20E030E0A90167E3AB
:10ED9000CE010E949574A501940169E2CE010E9402
:10EDA00095748E838823F1F00E9429746C197D0973
:10EDB0008E099F0997FDE8CF8AE0C6CF04E00E9444
:10EDC000E3F08E830150D9F78A3A11F482E0CFCF75
:10EDD0000E9429746C197D098E099F0997FDBCCF8B
:10EDE00082E0B2CF8F818230C1F420E030E0A9010F
:10EDF0006AE3CE010E949574882311F088E0A4CFC5
:10EE00000E94E3F0807C803C11F483E08F830E94B9
:10EE1000E3F00E94E3F00E94E3F0CE010E94E97269
:10EE200081E08A83173070F41D83DF91CF911F91A9
:10EE30000F91FF90EF90DF90CF90BF90AF909F9099
:10EE40008F90089588E18C8384CF1F920F920FB624
:10EE50000F9211242F933F938F939F93AF93BF9360
:10EE60008091AA069091AB06A091AC06B091AD0638
:10EE70003091A90623E0230F2D3758F50196A11DE7
:10EE8000B11D2093A9068093AA069093AB06A09388
:10EE9000AC06B093AD068091AE069091AF06A091FE
:10EEA000B006B091B1060196A11DB11D8093AE06CA
:10EEB0009093AF06A093B006B093B106BF91AF9107
:10EEC0009F918F913F912F910F900FBE0F901F90A8
:10EED000189526E8230F0296A11DB11DD2CFCF921F
:10EEE000DF92EF92FF920F931F93CF93DF93CDB7F3
:10EEF000DEB7A0970FB6F894DEBF0FBECDBF442398
:10EF000009F445C0611571058105910579F100E0AD
:10EF1000C42ED12CF12CE12CA70196010F94D138ED
:10EF200011E0100FE1E0F0E0EC0FFD1FE00FF11D2C
:10EF300007FDFA956083B901CA01012F61157105BA
:10EF40008105910549F7115010F1E1E0F0E0EC0F77
:10EF5000FD1FE10FF11D17FDFA95908187E39A30AF
:10EF600008F480E3890F0E948CC7EDCF80E3A09660
:10EF70000FB6F894DEBF0FBECDBFDF91CF911F91CA
:10EF80000F91FF90EF90DF90CF900C948CC7A096DC
:10EF90000FB6F894DEBF0FBECDBFDF91CF911F91AA
:10EFA0000F91FF90EF90DF90CF9008958091C5145E
:10EFB0008823C1F081508093C514E0EFF4E18823E9
:10EFC00051F08150990B2BE1289FF001299FF00D02
:10EFD0001124EA5DFA4E8BE1ABE0B5E101900D92B0
:10EFE0008A95E1F78091C514811105C09091D014E4
:10EFF00090629093D0140895CF92DF92EF92FF9297
:10F000008091D01482FF29C0C090CC14D090CD1430
:10F01000E090CE14F090CF1481EE91E20E94B4C73C
:10F020004AE0C701B6010E946F778FE20E948CC749
:10F030006091C8147091C9148091CA149091CB1436
:10F040004AE00E946F778DE00E948CC78AE0FF90B3
:10F05000EF90DF90CF900C948CC783EF91E2FF90FC
:10F06000EF90DF90CF900C94B4C7BC0185E191E2A2
:10F070000E940ADC82E191E20C94B4C78091D01422
:10F0800083FF03C084608093D0140895CF92DF92F1
:10F09000EF92FF920F931F93CF93DF93CDB7DEB71D
:10F0A000EDB6FEB6DC010D900020E9F79D01281BAE
:10F0B000390B285F3F4FEDB7FEB7E21BF30B0FB6DE
:10F0C000F894FEBF0FBEEDBF0DB71EB70F5F1F4F09
:10F0D0009F938F938BE091E29F938F931F930F9356
:10F0E0000F9424326801F4E0CF0ED11C0F900F90E2
:10F0F0000F900F900F900F90D6018D916D01882386
:10F1000049F0082E000C990B0F946F3CF6013197D3
:10F110008083F2CF66E071E2C8010F94BD314FE306
:10F1200050E0B8018EED95E00F94CB3C0FB6F8940B
:10F13000FEBE0FBEEDBEDF91CF911F910F91FF90EC
:10F14000EF90DF90CF900895FC01938591FD13C05F
:10F15000987121E0903109F020E08091D01420FBDB
:10F1600084F98093D014903141F08085873419F46C
:10F1700081858E3711F480E0089581E00895FC01C7
:10F1800020E03EE2DB014D91BD01403249F02830E4
:10F1900011F430833196DB0111974C914083319605
:10F1A0002F5F2B3079F710820895EF92FF920F9323
:10F1B0001F93CF93DF93CDB7DEB7A0970FB6F89428
:10F1C000DEBF0FBECDBF7C018B01BE016F5F7F4FE5
:10F1D000C7010E94A4F11816A4F4CE0101960E9462
:10F1E000A478882391F3BE016F5F7F4F81E292E1A3
:10F1F0000E94BF7861E272E1C8010F948D3C892BB7
:10F2000021F7A0960FB6F894DEBF0FBECDBFDF91F9
:10F21000CF911F910F91FF90EF900895CF92DF92C1
:10F22000EF92FF92CF936B017C01C42F8091A711C5
:10F230009091A811A091A911B091AA118C159D05CA
:10F24000AE05BF0529F10E94916F811108C0C0E091
:10F250008C2FCF91FF90EF90DF90CF900895809109
:10F26000B0119091B111DC01ED91FC910088F18910
:10F27000E02D27EA3FE0B701A6011995882339F36D
:10F28000C092A711D092A811E092A911F092AA11F0
:10F29000CC2321F081E08093AF11DACFC1E0D8CF49
:10F2A0004F925F926F927F928F929F92AF92BF9296
:10F2B000CF92DF92EF92FF920F931F93CF93DF9342
:10F2C000EC01423051056105710590F480E0DF9159
:10F2D000CF911F910F91FF90EF90DF90CF90BF9053
:10F2E000AF909F908F907F906F905F904F90089518
:10F2F00089859A85AB85BC850196A11DB11D8417B2
:10F300009507A607B70710F38F898031C9F5852EB9
:10F31000962EA72EBB248B899C89AD89BE89880E29
:10F32000991EAA1EBB1E280139016A017B0141E01A
:10F33000C501B4010E940E79882341F29F89903162
:10F3400081F5DD24EE24FF24F601EE0FFF1FE955C1
:10F35000F04F118300839A89923008F4B8CF4D8121
:10F360005E816F817885840E951EA61EB71E8092E1
:10F37000AB119092AC11A092AD11B092AE11A7CF8B
:10F38000803209F0A3CF8B899C89AD89BE894A015F
:10F390005B01E7E0B694A79497948794EA95D1F738
:10F3A000BECFE894C7F8DD24EE24FF24F601EE0F6B
:10F3B000FF1FEE0FFF1FE955F04F4082518262821E
:10F3C0007382C9CFCF92DF92EF92FF920F931F9378
:10F3D000CF93DF93FC0181859285A385B485019647
:10F3E000A11DB11D84179507A607B70750F480E04B
:10F3F000DF91CF911F910F91FF90EF90DF90CF9011
:10F40000089587898031A9F5BB27A72F962F852FCF
:10F41000C388D488E588F6888C0D9D1DAE1DBF1D60
:10F42000E9016A017B018F014091A7115091A81158
:10F430006091A9117091AA1184179507A607B707C3
:10F4400049F5F8018789803169F5B701A60155278B
:10F4500066277727440F551F4955504FFA01808181
:10F460009181B0E0A0E088839983AA83BB8381E087
:10F47000BFCF803209F0BBCFC388D488E588F68837
:10F48000DB01CA01C7E0B695A79597958795CA9500
:10F49000D1F7C2CF40E0BC01CD010E940E798111AD
:10F4A000D0CFA5CFB701A6014F775527662777277D
:10F4B000440F551F440F551F4955504FFA01808185
:10F4C0009181A281B381BF70CECF4F925F926F9234
:10F4D0007F92AF92BF92CF92DF92EF92FF920F9303
:10F4E0001F93CF93DF9300D01F92CDB7DEB78C016F
:10F4F00049835A836B837C835901C12CD12C7601BB
:10F50000412C82E0582E612C712C49815A816B81EB
:10F510007C819E012F5F3F4FC8010E94E2798823C2
:10F5200019F1F8018585A301920104C0220F331F50
:10F53000441F551F8A95D2F7DA01C901C80ED91E9A
:10F54000EA1EFB1E49815A816B817C81878980314B
:10F55000F1F481E0483F5F4F61057105B0F2F501BC
:10F56000C082D182E282F3820F900F900F900F90B1
:10F57000DF91CF911F910F91FF90EF90DF90CF908F
:10F58000BF90AF907F906F905F904F90089581E013
:10F59000483F5F4F6F4F7F4008F4B7CFE0CF0F93E6
:10F5A0001F93CF93DF93FC012381222331F080E06E
:10F5B000DF91CF911F910F9108958B01EC01FB0119
:10F5C0008789803139F582E08B831D8A1E8A1F8AE4
:10F5D000188E808D918DB0E0A0E025E0880F991FF6
:10F5E000AA1FBB1F2A95D1F7898B9A8BAB8BBC8B3B
:10F5F0001A8F098F81E08983188619861A861B86DF
:10F600001C821D821E821F82188A1C861D861E86F1
:10F610001F86CECF803259F683E08B83428D538D87
:10F62000648D758D4D8B5E8B6F8B788F9E012F5EF9
:10F630003F4FC8010E94657A8111DACFB8CF3F925F
:10F640004F925F926F927F928F929F92AF92BF92F2
:10F65000CF92DF92EF92FF920F931F93CF93DF939E
:10F66000CDB7DEB72C970FB6F894DEBF0FBECDBF77
:10F670005C01DC0159968D909C90F4018185928506
:10F68000A385B4859C01AD012F5F3F4F4F4F5F4F66
:10F6900029873A874B875C87D50114964D905D90FA
:10F6A0006D907C901797411451046104710409F422
:10F6B00059C0BFEF4B1A5B0A6B0A7B0A312C7301EE
:10F6C00062011D821E821F821886F4018185928547
:10F6D000A385B4852D813E814F8158852817390730
:10F6E0004A075B0708F056C089859A85AB85BC85BB
:10F6F0008C159D05AE05BF0550F482E0C82ED12CB7
:10F70000E12CF12C92E0492E512C612C712C9E01A0
:10F710002F5F3F4FB701A601C4010E94E279882301
:10F72000C9F189819A81AB81BC81892B8A2B8B2B72
:10F7300001F1260137019FEF491A590A690A790A2E
:10F740002D813E814F8158852F5F3F4F4F4F5F4F37
:10F750002D833E834F8358873FEFC31AD30AE30AB2
:10F76000F30AB3CF40805180628073803324339496
:10F77000A6CFC414D504E604F70411F70FEF1FEF6A
:10F780002FEF3FE0B701A601C4010E945079782E07
:10F7900081111AC0712C872D2C960FB6F894DEBFFC
:10F7A0000FBECDBFDF91CF911F910F91FF90EF90D2
:10F7B000DF90CF90BF90AF909F908F907F906F9091
:10F7C0005F904F903F900895F50144815581668187
:10F7D0007781411551056105710539F09701860161
:10F7E000C4010E9450798823A9F2D5011496CD92C4
:10F7F000DD92ED92FC921797332051F0D701C601AC
:10F800000196A11DB11DF40180839183A283B3836E
:10F81000F50185899689A789B08D892B8A2B8B2B39
:10F8200009F0B9CFC58AD68AE78AF08E81818068CF
:10F830008183B1CFCF93DF93EC01462F41706C856C
:10F840007D858E859F850E940E79882351F0888959
:10F8500020E2829FC00111248955904FDF91CF9102
:10F86000089590E080E0FACFCF93DF93EC01899187
:10F87000882319F00E948CC7FACFDF91CF910895A9
:10F88000CF93DF93EC018B81882349F1898187FF36
:10F8900022C061E0CE010E941A7CFC01892BF9F0A4
:10F8A0008081853EE1F08B81823040F489899A899C
:10F8B000AB89BC89848F958FA68FB78F8D899E89E0
:10F8C000938F828F8D899E89AF89B88DB58BA48BDC
:10F8D00089818F778983DF91CF910C94916F81E03B
:10F8E000888380E0DF91CF9108958F929F92AF92AD
:10F8F000BF92CF92DF92EF92FF920F931F93CF931D
:10F90000DF93EC018B8181110EC080E0DF91CF91FC
:10F910001F910F91FF90EF90DF90CF90BF90AF902D
:10F920009F908F90089509891A892B893C89041723
:10F9300015072607370748F34A015B01823031F487
:10F9400088869986AA86BB8681E0E0CF81149104DF
:10F95000A104B10449F4188619861A861B861C82F4
:10F960001D821E821F82F0CF088519852A853B855E
:10F97000E98DFA8D858590E00996B901A80141507D
:10F98000510961097109082E04C07695679557954C
:10F9900047950A94D2F775016401E1E0CE1AD108C7
:10F9A000E108F10804C0F694E794D794C7948A95C7
:10F9B000D2F7C416D506E606F70620F0012B022B77
:10F9C000032B11F58D899E89AF89B88D8C839D831A
:10F9D000AE83BF838E010C5F1F4FC114D104E104BD
:10F9E000F10409F4ADCF4C815D816E817F81980176
:10F9F000898D9A8D0E94E27991E0C91AD108E108B7
:10FA0000F1088111EACF81CFC41AD50AE60AF70AB4
:10FA1000E1CF2F923F924F925F926F927F928F929F
:10FA20009F92AF92BF92CF92DF92EF92FF920F938D
:10FA30001F93CF93DF9300D01F92CDB7DEB78C0119
:10FA40004B011A01DC0113968C911397813009F058
:10FA5000CFC011968C9181FFCBC082FDB5C06101F2
:10FA6000D80118964D915D916D917C911B97C114B1
:10FA7000D10409F41BC159968D919C915A97FC01B0
:10FA800074802FEF270D2A013B0139E076946794AB
:10FA9000579447943A95D1F7722E74207A01F1E089
:10FAA000FF22711020C0E114F104E9F414964D9185
:10FAB0005D916D917C911797411551056105710517
:10FAC00009F09CC055968D919D910D90BC91A02DF3
:10FAD0000097A105B10509F0AAC0C8010E941F7BCB
:10FAE000882309F485C0A12C82E0B82EAE18BF0887
:10FAF000CA14DB0408F45601D80159964D915C9163
:10FB00005A9714968D919D910D90BC91A02D0297BE
:10FB1000A109B109FA01258504C0880F991FAA1F00
:10FB2000BB1F2A95D2F74685578560897189840F56
:10FB3000951FA61FB71F9C01AD01270D311D411D4B
:10FB4000511D29013A01A11432E0B30609F07DC02C
:10FB50008091A7119091A811A091A911B091AA111B
:10FB6000481659066A067B0669F41092AF118FEFAA
:10FB70009FEFDC018093A7119093A811A093A91186
:10FB8000B093AA118091B0119091B111DC01ED9167
:10FB9000FC910288F389E02D9401B301A20119952B
:10FBA000882331F1F80180859185A285B3858A0D7E
:10FBB0009B1DA11DB11D80879187A287B3878A0CE9
:10FBC0009B1CCA18DB084CCFF80141895289638914
:10FBD000748980859185A285B385481759076A077E
:10FBE0007B0709F43CCFC8010E94757C811137CF97
:10FBF00081E0D8018C938FEF9FEF6EC09E012F5F45
:10FC00003F4F0E94E279882399F389819A81AB81E1
:10FC1000BC81F801218D328DF9012789203169F4E9
:10FC2000883FFFEF9F07A105B10508F056CFF80107
:10FC300084839583A683B78356CF883F2FEF92079F
:10FC4000A2072FE0B20798F348CFE114F10431F591
:10FC5000F801408551856285738581899289A389E0
:10FC6000B489481759076A077B07C0F00E94916F53
:10FC7000882309F4BDCF81E08093AF114092A71192
:10FC80005092A8116092A9117092AA11A501B40115
:10FC9000C7018955904F0F94843C84CF41E0C30144
:10FCA000B2010E940E798111F1CFA2CFF8018189B2
:10FCB0009289A389B48984179507A607B70738F4F2
:10FCC0008181418B528B638B748B80688183F801B7
:10FCD000818183FD18C0C1010F900F900F900F908C
:10FCE000DF91CF911F910F91FF90EF90DF90CF9018
:10FCF000BF90AF909F908F907F906F905F904F904C
:10FD00003F902F900895C8010E94407C8111E3CF5D
:10FD10006FCF2F923F924F925F926F927F928F920E
:10FD20009F92AF92BF92CF92DF92EF92FF920F938A
:10FD30001F93CF93DF93EC014B017A018B818111EB
:10FD400015C08FEF9FEFDF91CF911F910F91FF9023
:10FD5000EF90DF90CF90BF90AF909F908F907F906B
:10FD60006F905F904F903F902F900895898180FF12
:10FD7000E8CF89899A89AB89BC89488559856A8584
:10FD80007B85841B950BA60BB70BA70170E060E089
:10FD900084179507A607B70708F47C0167011E01C1
:10FDA00024E0220E311CC114D10409F4A9C04885F5
:10FDB00059856A857B855A0181E0B822898D9A8DA3
:10FDC0002A013B0129E076946794579447942A9539
:10FDD000D1F72B81FC01223081F5628D738D848DEA
:10FDE000958D640D751D861D971D00E012E00A19A2
:10FDF0001B09C016D10608F486010115E2E01E07B2
:10FE000071F44090A7115090A8116090A9117090C2
:10FE1000AA11641575058605970509F04EC040E0E6
:10FE20000E940E79882309F48CCFB5016955704F73
:10FE3000A801C4010F94843C52C0148111501421B4
:10FE4000A114B10471F411110CC0452B462B472BA2
:10FE500051F58D899E89AF89B88D8C839D83AE8342
:10FE6000BF83E98DFA8D4C805D806E807F8022E0BB
:10FE7000421A510861087108858504C0440C551C5C
:10FE8000661C771C8A95D2F786859785A089B189EB
:10FE9000480E591E6A1E7B1EC301B201610F711DFF
:10FEA000811D911DA2CF4C815D816E817F81910169
:10FEB0000E94E2798111D5CF44CFA091B011B091C9
:10FEC000B111ED91FC9111970088F189E02D940119
:10FED000AB01BC01CD011995882309F432CF800E06
:10FEE000911E88859985AA85BB85800F911FA11DCC
:10FEF000B11D88879987AA87BB87C01AD10A53CFBB
:10FF0000C70121CFCF93DF93EB01FC0123812111A6
:10FF100004C080E0DF91CF9108952250223028F470
:10FF20008FE28883198281E0F5CF60E00E941A7C1D
:10FF3000009779F3DC0160E080E09EE22D912032B1
:10FF400099F0883031F49E01260F311DF90190831C
:10FF50006F5F9E01260F311DAD0141505109FA011D
:10FF60004081F90140836F5F8F5F8B3039F7FE016D
:10FF7000E60FF11D1082D7CFCF93DF93EC01CB01B9
:10FF8000E881F981608171810E94827F28813981B5
:10FF9000D901ED91FC91AA81BB818C91908199232B
:10FFA00059F08936C8F4CF010196F9019183808315
:10FFB0008C918F5F8C93EACF893670F48FE28083C7
:10FFC000E881F98180819181019691838083EA8122
:10FFD000FB8180818F5F8083DF91CF9108950F93A4
:10FFE0001F93CF93DF9300D000D01F92CDB7DEB721
:10FFF0009C012F5F3F4F3F832E832FE2FC01208324
:020000021000EC
:1000000081E08D83CE0106969A83898301979C8334
:100010008B8310E00BE18091C514181758F4109FE2
:10002000B00111246A5D7A4ECE0101960E94BC7F18
:100030001F5FF1CF8D818B3558F464E376E1CE01FB
:1000400001960E94BC7F8E819F8101979F838E8342
:10005000EE81FF81108227960FB6F894DEBF0FBEA7
:10006000CDBFDF91CF911F910F910895CF93DF9373
:10007000EC010E94407C1B82DF91CF910895109289
:10008000B2118091D0148F7B8B7F8093D0140E940B
:10009000E3C3882321F084E396E10C94368008952D
:1000A0008091D01482FF0AC080648093D014809124
:1000B000D014877F80628093D01408950E943F807F
:1000C000F6CFCF93DF938091D014877F8093D014A5
:1000D0008091F314882321F080EF94E10E94368010
:1000E0008091D1149091D214DC01ED91FC9101909A
:1000F000F081E02D45E360E0199581110EC00E946A
:1001000018DC8AEF90E20E94B4C78091D01483FF7C
:1001100030C0DF91CF910C94826FC091D114D091F7
:10012000D21461E0CE010E9481F681110BC060E023
:10013000CE010E9481F6811105C00E9414DC86EE7A
:1001400090E2E1CF6BE872E180EF94E10E94CF7A18
:10015000811105C00E9414DC85ED90E2D4CF80911E
:10016000D01488608093D0140E9418DC89EC90E24F
:10017000CACF80911F06882339F06FEF8CEB90E295
:10018000DF91CF910C94EC3CDF91CF91089540E04A
:1001900050E0BA010C94757C0F931F93CF93DF93BB
:1001A000CDB7DEB7EB970FB6F894DEBF0FBECDBF6D
:1001B0008091D01400E010E083FF23C08BE095E134
:1001C0000E94C7808BE1EBE0F5E1DE0191960190A2
:1001D0000D928A95E1F710E000E0BE016F5F7F4F5E
:1001E000CE0181960E94A4F118163CF4CE0101962E
:1001F0000E94A478080F111DF0CFCE0181960E94B5
:10020000D4BFC801EB960FB6F894DEBF0FBECDBFCA
:10021000DF91CF911F910F9108950F931F93CF936B
:10022000DF93CDB7DEB76B970FB6F894DEBF0FBE86
:10023000CDBF8C018BE095E10E94C7808BE1EBE0A4
:10024000F5E1DE01119601900D928A95E1F7B80172
:10025000CE0101960E94D578CE0101960E94D4BFAE
:100260006B960FB6F894DEBF0FBECDBFDF91CF9176
:100270001F910F9108954F925F926F927F92AF926C
:10028000BF92CF92DF92EF92FF920F931F93CF9383
:10029000DF931F92CDB7DEB78C017B015A01C22ECE
:1002A000DB0159968D919C91F801928F818FCB0142
:1002B0000E94C780712CF70180859185A285B38546
:1002C000418952896389748984179507A607B707FE
:1002D00008F052C055E0B695A795979587955A9521
:1002E000D1F7F82FFF70DF2ED70113968C91823053
:1002F00010F480E0DBC041E050E0BE016F5F7F4F53
:10030000C7010E94897E0197A1F7F7018085918539
:10031000A285B3854F96A11DB11D80879187A287C5
:10032000B387F0E2DF9EB00111246955704F61156B
:100330007105F9F2DB018C91882341F0853E09F0CB
:100340004CC0772029F077247394B5CF71100EC07C
:100350008091A7119091A811A091A911B091AA1113
:10036000F80184879587A687B787D08ADB018C91AF
:100370008111E9CF772473948C2D8274823409F033
:10038000B8CF772009F4A2C0F801D08861E0C80195
:100390000E941A7C009709F4ACCF20E2DC011D9288
:1003A0002A95E9F72BE0F501DC0101900D922A95E1
:1003B000E1F721E238E2FC01318B208B40E058E08C
:1003C00057874687338B228B318F208F578B468BF5
:1003D0000E94916F811109C08CCF4BE050E0C501A4
:1003E0000F94773C892B09F066CFF0E2DF9ED001B5
:1003F00011249D012955304FF9018385817121F028
:100400008C2D827109F001C1F801818D928D40918E
:10041000A7115091A8116091A9117091AA11448758
:10042000558766877787D08AFD01E955F04F448864
:100430005588712C612C320155244424D8015596DD
:100440004D925D926D927C925897428D538D70E0E3
:1004500060E0442955296629772955964D935D9387
:100460006D937C935897D9011B962C91287109F0B4
:10047000BEC0848D958DA68DB78DF801818B928B32
:10048000A38BB48B81E083838C2D8F70F8018183E3
:1004900014821582168217821086118612861386A0
:1004A00081E0C4FE03C0C8010E94C9F20F90DF9131
:1004B000CF911F910F91FF90EF90DF90CF90BF9061
:1004C000AF907F906F905F904F900895D7011396F3
:1004D0008C911397823009F40CCF51968D919D9198
:1004E0000D90BC91A02D803E9F4FAF41B10508F00B
:1004F00000CFC7010E941F7B882309F4FACE0E9417
:10050000916F882309F4F5CED7015996ED91FC91AE
:100510005A9714964D905D906D907C901797B2E02D
:100520004B1A510861087108858504C0440C551C9C
:10053000661C771C8A95D2F786859785A089B18934
:10054000480E591E6A1E7B1E81E08093AF114092B7
:10055000A7115092A8116092A9117092AA11E7EA0E
:10056000FFE080E092E0DF019C011D9221503040CD
:10057000E1F7DD24D394D7015996ED91FC91848164
:10058000D816C0F48091B0119091B111DC01ED91B9
:10059000FC910288F389E02D27EA3FE0B301A20134
:1005A0004D0D511D611D711D1995882309F4A1CEB2
:1005B000D394E1CF258580E092E0A0E0B0E004C0D4
:1005C000880F991FAA1FBB1F2A95D2F7F7014189EF
:1005D000528963897489840F951FA61FB71F818B69
:1005E000928BA38BB48B87EA9FE0D12CD6CE20319F
:1005F00061F498012F5E3F4F0E94657A882329F0AD
:1006000084E0D80113968C933FCFD80113961C92A7
:1006100070CE2F923F924F925F926F927F928F9205
:100620009F92AF92BF92CF92DF92EF92FF920F9381
:100630001F93CF93DF93CDB7DEB7C354D1090FB665
:10064000F894DEBF0FBECDBF4C015B016A01222EC4
:1006500019821C821C8E1F8E6115710521F510E018
:10066000CE014C960E94D4BFCE0101960E94D4BF09
:10067000812FCD5BDF4F0FB6F894DEBF0FBECDBF2D
:10068000DF91CF911F910F91FF90EF90DF90CF906E
:10069000BF90AF909F908F907F906F905F904F90A2
:1006A0003F902F900895FC0183818111D8CFFA01EA
:1006B00080818F32A1F18B01CE0101967C013C013A
:1006C00080E2382E2E019CE1490E511C2396EFAE9C
:1006D00023972496FFAE249722963FAE2297219629
:1006E0003FAE21973FAE3EAE3DAE3CAE3BAE3AAEE6
:1006F00039AE38AE3FAA960190E047E0D9018D911E
:10070000882309F447C08F3209F444C08E3209F5BA
:100710004A3009F4A4CF98E04AE09D01EFCFFB01F5
:10072000838182508B01823060F0618D728DCE01A9
:100730004C960E94CF7A8E01045E1F4F882309F4E5
:100740008ECFC6016C010196F60120812F32D1F3C4
:10075000B3CFE8E9F0E22491222321F0319682130D
:10076000FACF7DCF491708F47ACF813208F477CFDA
:100770008F3709F474CF3FE9380F3A3108F420EE8F
:10078000E7E3F0E0EC0FFD1FE90FF11D820F80831E
:100790009F5FC3CF8FA9803209F461CF6901F9014E
:1007A00080812F5F3F4F8F32C9F3882301F121E011
:1007B000AE01495C5F4FB801C7010E943B818823AD
:1007C00009F44DCF0A151B0519F0C8010E943680A7
:1007D000942D852D6E147F0431F023969FAD2397C1
:1007E00024968FAD24978701E92EF82E75CF222D00
:1007F000AE01495C5F4FB801C4010E943B81182FD4
:100800002FCF1F93CF93DF93CDB7DEB76D970FB682
:10081000F894DEBF0FBECDBF1D8E1C8EAC01BE0195
:10082000645E7F4F80E00E947EF510E00097A9F0A3
:1008300019821C826C8D7D8D21E0AC01CE01019668
:100840000E940983182F882321F0CE0101960E946F
:100850003680CE0101960E94D4BF812F6D960FB6CF
:10086000F894DEBF0FBECDBFDF91CF911F910895E9
:10087000EF92FF921F93CF93DF9300D000D000D070
:100880001F92CDB7DEB78091D01483FF0E946180A4
:100890008091D01483FF3CC00E94C2BF811138C038
:1008A0008091C61490E08F969F938F938FE292E28F
:1008B0009F938F93CE0101967C019F938F930F940A
:1008C00024328091D0140F900F900F900F900F90C2
:1008D0000F9083FF1DC0C7010E940184182F882339
:1008E000B9F00E94826FC7010E9446788091C614B9
:1008F0008F5F8093C614812F2A960FB6F894DEBFBF
:100900000FBECDBFDF91CF911F91FF90EF90089563
:100910001092C61410E0EFCF81E08093C6140C94BF
:100920003884CF939091D01493FF23C09091D81422
:1009300091111FC02AE5811121E0C82F46E053E044
:1009400060EF74E185ED94E10E940983811105C097
:1009500086E093E0CF910C943578C1110AC066E02F
:1009600073E084E092E20E940ADC8AE0CF910C946A
:100970008CC7CF910895CF9321E046E053E060EF1C
:1009800074E185ED94E10E940983C82F882321F04A
:1009900085ED94E10E9436808C2FCF910895FF92CF
:1009A0000F931F93CF93DF93CDB7DEB76D970FB63D
:1009B000F894DEBF0FBECDBF2091D01423FF2DC011
:1009C000AC01BE01645E7F4F80E00E947EF58C0129
:1009D000009719F16C8D7D8D19821C8222E0AC018B
:1009E000CE0101960E940983811123C0F12CCE0112
:1009F00001960E94D4BFB801FF2081F183ED91E2FE
:100A00000E940ADC8AE00E948CC71092CC141092DB
:100A1000CD141092CE141092CF146D960FB6F89498
:100A2000DEBF0FBECDBFDF91CF911F910F91FF9021
:100A30000895CE0101960E94C9F28823B9F261E0BF
:100A4000CE0101960E941A7C009781F225EEFC01EE
:100A500020831C820E94916FF82EC9CF8BEB91E20C
:100A60000E940ADC88EB91E20E94B4C7D6CF0E94B4
:100A7000BB84882331F00E94ACBF86E093E00C94E5
:100A8000CF8408950F931F93CF93DF931F921F92EC
:100A9000CDB7DEB72091D01423FF32C08C01BC014A
:100AA00082E00E9433721092C7140E943F80A80116
:100AB000BE016F5F7F4F80E00E947EF58C01009742
:100AC000F9F069817A8126E5AC0184E396E10E9420
:100AD00009838823E1F08091D01481608093D01441
:100AE000C8010E940D811092C414B80184E092E202
:100AF0000E940ADC8AE00E948CC7C8010E9417F598
:100B00000F900F90DF91CF911F910F910895C80121
:100B10000E943578F5CFCF92DF92EF92FF920F933C
:100B20001F93CF93DF931F921F92CDB7DEB7209113
:100B3000D01423FF62C08C01613009F470C008F446
:100B400067C0623009F4CFC00E943F80A801BE0197
:100B50006F5F7F4F81E00E947EF58C01009709F462
:100B60004CC069817A8121E0AC0184E396E10E9466
:100B70000983882309F4BEC08091451690914616DA
:100B8000A0914716B09148168093C8149093C91449
:100B9000A093CA14B093CB141092CC141092CD141D
:100BA0001092CE141092CF14B80180E491E20E940A
:100BB0000ADCC090C814D090C914E090CA14F09018
:100BC000CB1488E391E20E94B4C74AE0C701B601A2
:100BD0000E946F778AE00E948CC789E291E20E94AE
:100BE000B4C7C8010E940D8180912E12882311F094
:100BF0000EE212E1C8010E9417F50F900F90DF91ED
:100C0000CF911F910F91FF90EF90DF90CF900895BB
:100C1000BC0182E00E9433721092C71495CF0E94EB
:100C2000E3C3811105C0B80181E00E9433728CCF0B
:100C30008091C714882391F00E9414DC61E070E079
:100C400089E991E20E947BCA8AE00E948CC740E059
:100C500070E060E088E891E20E94F2DE87E595E0CE
:100C60000E94EF7FE091C71484E0E89FF001112417
:100C7000ED5AFA4F8091CC149091CD14A091CE14DE
:100C8000B091CF1480839183A283B3830E9418DC38
:100C9000B8018FE691E20E940ADC6091C71489E6F0
:100CA000689FB0011124695A7A4F84E691E20E944C
:100CB0000ADCC090CC14D090CD14E090CE14F0900B
:100CC000CF148EE591E20E94B4C74AE0C701B60195
:100CD0000E946F778AE00E948CC78091C7148F5F53
:100CE0008093C71431CF0E9418DC8EE491E20E94F9
:100CF000B4C72ACFC8010E9435787FCF6F927F9208
:100D00008F929F92AF92BF92CF92DF92EF92FF921B
:100D10000F931F93CF93DF93CDB7DEB7C356D1099F
:100D20000FB6F894DEBF0FBECDBF5C018B016DB670
:100D30007EB67E0187E5E80EF11CBE016F5F7F4F36
:100D4000C5010E94A4F118160CF0A4C08C8588710E
:100D5000803109F076C08DB69EB6BE016F5F7F4FC1
:100D6000C7010E94BF780115110509F466C0F8019A
:100D70008081882309F461C001900020E9F7319750
:100D8000CF01801B910B20E0F70101900020E9F7D3
:100D90003197EE19FF09E80FF91F32968DB79EB70C
:100DA0008E1B9F0B0FB6F8949EBF0FBE8DBFEDB785
:100DB000FEB731966F01B801222311F06DE074E0A7
:100DC000C6010F94B63CB701C6010F94A03C6DE07C
:100DD00074E0C6010F94A03C19A21CA221E0A70157
:100DE000B501CE0181960E94098381110AC00E943B
:100DF00018DCB70188EA90E20E940ADC8AE00E94CF
:100E00008CC78BE1FE01B196DE01DC9601900D925C
:100E10008A95E1F7B601CE01CC960E947E86CE017E
:100E2000CC960E94D4BFCE0181960E94D4BF0FB64B
:100E3000F8949EBE0FBE8DBE80CF21E081E090E091
:100E4000A3CFCE0101960E94A478882309F475CF20
:100E5000BE016F5F7F4F81E292E10E94BF78011572
:100E6000110519F0C8010E94347C81E292E10E94D0
:100E7000347C80E20E948CC76D8D7E8D8F8D98A111
:100E80004AE00E946F778DE00E948CC78AE00E9442
:100E90008CC753CF0FB6F8947EBE0FBE6DBECD5932
:100EA000DF4F0FB6F894DEBF0FBECDBFDF91CF91FD
:100EB0001F910F91FF90EF90DF90CF90BF90AF9078
:100EC0009F908F907F906F900895CF93C82F0E942E
:100ED00018DC84E50E948CC78C2F0E9496F180E27A
:100EE0000E948CC786E890E2CF910C94B4C78F9291
:100EF0009F92AF92BF92CF92DF92EF92FF92CF93E9
:100F00006B017C01B42E20E030E0A9010F948D32FA
:100F100087FF07C08DE20E948CC7F7FAF094F7F8BC
:100F2000F094C0E060E070E080E09FE3CB1541F01A
:100F30002DEC3CEC4CEC5DE30F94F332CF5FF6CF3D
:100F4000A70196010F945D396B017C010F94D03A93
:100F50004B015C014AE00E946F77CC2379F1C50117
:100F6000B4010F9492329B01AC01C701B6010F94FA
:100F70005C396B017C018EE20E948CC7C150F0F09D
:100F800020E030E040E251E4C701B6010F94F332B3
:100F90006B017C010F94D03A4B015C014AE00E9446
:100FA0006F77C501B4010F9492329B01AC01C70168
:100FB000B6010F945C396B017C01E0CFCF91FF90BB
:100FC000EF90DF90CF90BF90AF909F908F9008955B
:100FD000EF92FF920F931F93CF937C018B01C2E49A
:100FE0004F3F09F0C4E580E20E948CC78C2F0E941D
:100FF0008CC78AE30E948CC7F7016081718182816E
:10100000938142E00E94778782E790E20E94B4C712
:10101000F801608171818281938142E00E9477872B
:1010200062E070E080E090E0CF911F910F91FF901F
:10103000EF900C94F6731F93CF93DF9300D000D002
:101040001F921F92CDB7DEB7182F60917C1270915E
:101050007D12072E000C880B990B0F9494326D8330
:101060007E838F83988760917A1270917B12072E0E
:10107000000C880B990B0F94943269837A838B83CD
:101080009C834AEFBE016B5F7F4FCE0101960E94A9
:10109000E8876091111270911212072E000C880BD4
:1010A000990B0F9494326D837E838F839887609120
:1010B0000F1270911012072E000C880B990B0F94D1
:1010C000943269837A838B839C834FEFBE016B5F7D
:1010D0007F4FCE0101960E94E887609113121F3F57
:1010E00039F085E11802F0011124EA58FD4E6085BF
:1010F00070E08AE790E20E947BCA6091131270E070
:1011000085E790E20E947BCA28960FB6F894DEBF6E
:101110000FBECDBFDF91CF911F9108952F923F92C7
:101120004F925F926F927F928F929F92AF92BF92F7
:10113000CF92DF92EF92FF920F931F93CF93DF93A3
:10114000CDB7DEB763970FB6F894DEBF0FBECDBF45
:10115000898B81E080932D021A821B821C821D8262
:1011600019861A861B861C861D862CE32E873CE179
:101170003F8746E4488B312C212C50E85A8B8FEB6B
:101180008B8B198291E09887812C912C54010091CE
:10119000111210911212B801012E000C880B990B3C
:1011A0000F9494326B017C01232D322D4A895B8987
:1011B0000F948D32882389F080910F129091101234
:1011C000A989A111E4C0B1E0B983081719070CF08F
:1011D00019823C2C2D2CEA8AFB8A0E9429746B010F
:1011E0007C01DC01CB0129853A854B855C85821B1E
:1011F000930BA40BB50BB7FD2FC0D701C6018851C7
:101200009C4FAF4FBF4F89879A87AB87BC8780E0E1
:101210000E941B8882E890E20E94B4C78114910466
:10122000A104B10409F4DFC0C501B40168577C4EC4
:101230008F4F9F4F6C197D098E099F0928EE33E06F
:1012400040E050E00F94D138CA01B9014AE00E9451
:1012500093C78AE00E948CC780E00E94C3DF0E948F
:10126000297460930512709306128093071290936D
:10127000081260910F1270911012072E000C880B4B
:10128000990B0F9494326E837F838C019B01AC0188
:10129000632D722D8A899B890F945C392B013C0147
:1012A00020E030E0A9010F94BD3B87FF04C077FA2E
:1012B000709477F8709481149104A104B10409F03A
:1012C00096C020E030E040E85FE3C301B2010F9434
:1012D0008D3287FF10C09885812C912C5401992361
:1012E00031F082E8882E86E0982EA12CB12C8C0C4F
:1012F0009D1CAE1CBF1CA981AA2391F12A813B81B0
:101300004C815D81211531054105510541F0D70121
:10131000C601821B930BA40BB50BB7FD21C02E8118
:101320003F81A8016D857E858F8598890F945C39F2
:1013300020E030E040E85FE30F948D3287FD2AC063
:10134000D701C601805A9541AF4FBF4F8A839B8317
:10135000AC83BD839E819D87AF81AE870F87188B3D
:1013600080912D028823B1F081149104A104B1046D
:1013700061F0B8E8CB1AB3E1DB0AE108F108C8185C
:10138000D908EA08FB08F7FE05C0188600CF081741
:1013900019071CF520912D022983222321F0109298
:1013A0002D020E944FF5898163960FB6F894DEBF37
:1013B0000FBECDBFDF91CF911F910F91FF90EF90A6
:1013C000DF90CF90BF90AF909F908F907F906F9065
:1013D0005F904F903F902F9008953C2C2D2CEA8ADF
:1013E000FB8A1982FACE8FE30E948CC732CF20E0AD
:1013F00030E040E450E4C301B2010F94BD3B181645
:101400000CF079CF4601570176CF2F923F924F9241
:101410005F926F927F928F929F92AF92BF92CF9284
:10142000DF92EF92FF920F931F93CF93DF93CDB78D
:10143000DEB765970FB6F894DEBF0FBECDBF8A8BBF
:101440006B8B20915205298B1092520581E080937D
:101450002D021A821B821C821D8219861A861B8607
:101460001C861D863CE33E874CE14F8756E4588B33
:10147000312C212C80E88C8B9FEB9D8B1982A1E075
:10148000A887812C912C540100917C1210917D121F
:10149000B801012E000C880B990B0F9494326B014C
:1014A0007C01232D322D4C895D890F948D32882348
:1014B00089F080917A1290917B12BB89B111E4C0BE
:1014C00021E02983081719070CF019823C2C2D2CD8
:1014D000EC8AFD8A0E9429746B017C01DC01CB013E
:1014E00029853A854B855C85821B930BA40BB50B34
:1014F000B7FD2FC0D701C60188519C4FAF4FBF4FDA
:1015000089879A87AB87BC878A890E941B888EE768
:1015100090E20E94B4C781149104A104B10409F4BB
:10152000E2C0C501B4016053784F8F4F9F4F6C19D3
:101530007D098E099F0928EE33E040E050E00F94CA
:10154000D138CA01B9014AE00E9493C78AE00E94DB
:101550008CC780E00E94C3DF0E942974609305124B
:1015600070930612809307129093081260917A127A
:1015700070917B12072E000C880B990B0F949432FC
:101580006E837F838C019B01AC01632D722D8C894E
:101590009D890F945C392B013C0120E030E0A901CA
:1015A0000F94BD3B87FF04C077FA709477F870946E
:1015B00081149104A104B10409F099C020E030E045
:1015C00040E85FE3C301B2010F948D3287FF10C082
:1015D0009885812C912C5401992331F08AE9882E29
:1015E00082E0982EA12CB12C8C0C9D1CAE1CBF1C33
:1015F000A981AA2391F12A813B814C815D8121152A
:1016000031054105510541F0D701C601821B930BFD
:10161000A40BB50BB7FD21C02E813F81A8016D85BC
:101620007E858F8598890F945C3920E030E040EC0E
:101630005FE30F948D3287FD2AC0D701C601805A1F
:101640009541AF4FBF4F8A839B83AC83BD839E81FF
:101650009D87AF81AE870F87188B80912D028823DD
:10166000B1F081149104A104B10461F0B0EDCB1A82
:10167000B7E0DB0AE108F108C818D908EA08FB0856
:10168000F7FE05C0188600CF0817190734F530910A
:101690002D023983332321F010922D020E944FF541
:1016A000298920935205898165960FB6F894DEBF8B
:1016B0000FBECDBFDF91CF911F910F91FF90EF90A3
:1016C000DF90CF90BF90AF909F908F907F906F9062
:1016D0005F904F903F902F9008953C2C2D2CEC8ADA
:1016E000FD8A1982F7CE8FE30E948CC72FCF20E0AE
:1016F00030E040E450E4C301B2010F94BD3B181642
:101700000CF076CF4601570173CF0F930FB70F93AD
:1017100000916E000B7F00936E0078940F930BB7CF
:101720000F930CB70F921F922F933F934F935F939A
:101730006F937F938F939F93AF93BF93EF93FF9399
:1017400011240E94668CFF91EF91BF91AF919F9100
:101750008F917F916F915F914F913F912F911F904A
:101760000F900CBF0F910BBF0F910460F894009382
:101770006E000F910FBF0F911895209111123091AB
:10178000121221153105E9F080910F12909110127B
:10179000029624503109821793079CF490939B067C
:1017A00080939A060E942974605E70448D4F9F4F0B
:1017B00060939C0670939D0680939E0690939F066F
:1017C000089510929C0610929D0610929E0610920B
:1017D0009F060895CF93DF9310925205C6E7D2E19A
:1017E0001F821E820E9411F118862C98CBE0D2E154
:1017F0001F821E820E94BD8B18868091020180721A
:1018000080930001DF91CF910895EF92FF920F93A3
:101810001F93CF93DF93C82F7B018A0180911F060E
:101820008130A1F40E9414DCC7010E94B4C78AE48D
:101830009FE10E94B4C7C7FD33C08C2F0C2E000C53
:10184000990B0E949DF18AE00E948CC70E94EA8B4E
:10185000A89580917006811132C081E08093700656
:1018600080E880931F060E94EA8BD5E1D150409A10
:10187000E1F069E170E080E090E00E94F673A895E5
:10188000409868E270E080E090E00E94F673A895CE
:1018900068E270E080E090E00E94F673A895E6CFE1
:1018A00086E49FE10E94B4C7CECF6FE37FE1CF3FD4
:1018B00011F063E47FE140E0C8010E94F2DEDF91B5
:1018C000CF911F910F91FF90EF9008950F931F9369
:1018D000CF93DF93809122028F3708F442C08F5755
:1018E00090917E129093A4069923C9F12C9A20918D
:1018F00013122093A30690910201211190959072EA
:10190000909300018F5F809322028091A20691E064
:1019100089278093A20680912102C1E0C80F8530FB
:101920000CF0C0E0823009F4D8C03CF58823D9F12E
:10193000813009F4C6C0C09321020E94EE3280912A
:101940004B0990914C09009729F0019790934C090D
:1019500080934B09DF91CF911F910F9108952C989F
:10196000C6CF9091A406891708F02C989091A306F1
:10197000891740F290910201C2CF843009F4C5C0AA
:101980000CF4BEC08530B9F69091A106911102C049
:101990008093A1068091A10681508093A10688239F
:1019A00051F2C5E0C8CF809120028F5F80311CF4D6
:1019B00080932002C0CF109220028091A006811156
:1019C00013C0809176129091771290937912809340
:1019D000781280910B1290910C1290930E128093BA
:1019E0000D1281E08093A006109277121092761269
:1019F00010920C1210920B12009178121091791221
:101A000080917C1290917D12D1E0181619062CF06D
:101A100080917E12811101C0D0E0809127029091C7
:101A20002802081719073CF444E350E261E470E22D
:101A300080E00E94058CDD2371F080912502909159
:101A40002602801791073CF443E550E260E670E21D
:101A500080E00E94058C8091111290911212D1E0C9
:101A6000181619062CF080911312811101C0D0E0D4
:101A700020910D1230910E128091A6069091A7062A
:101A8000281739073CF444E350E261E470E28FEF39
:101A90000E94058CDD2309F44ECF20910D12309168
:101AA0000E128091230290912402821793070CF06A
:101AB00042CF43E550E260E670E28FEF0E94058C72
:101AC0003ACF88E080937B0085E480937C0080910E
:101AD0007A00806480937A002ECF80917A0086FD10
:101AE00027C02091780030917900809176129091F2
:101AF0007712820F931F90937712809376121BCFE9
:101B000088E080937B0086E4E0CF80917A0086FDB8
:101B100011C0209178003091790080910B12909142
:101B20000C12820F931F90930C1280930B1203CF11
:101B3000C2E001CFC4E0FFCE2F923F924F925F925E
:101B40006F927F928F929F92AF92BF92CF92DF92CD
:101B5000EF92FF920F931F93CF93DF9300D0CDB7F7
:101B6000DEB79B838A836B015A01298318018701A1
:101B700081E090E02F3F11F090E080E025E0289F89
:101B8000F001299FF00D1124E85BFA4F848188232E
:101B900009F48FC0EA81FB811482158216821782B4
:101BA0001086EA81FB8184818230B9F0833009F4A8
:101BB00000C1813009F067C0258136814781508599
:101BC000F60160817181828193810F948D3287FD4E
:101BD0005AC082E0EA81FB818483EA81FB818580AF
:101BE0009680A780B084F601C080D180E280F38027
:101BF000B801110F880B990B0F9494322B013C0103
:101C000080911F028823F9F0F981F1111CC08091A5
